:100000000C94C11E0C94F21E0C94F21E0C94F21E61
:100010000C94F21E0C94F21E0C94F21E0C94F21E20
:100020000C94F21E0C94F21E0C94F21E0C94F21E10
:100030000C94F21E0C94F21E0C94F21E0C94F21E00
:100040000C94F21E0D94580E0C94F21E0C94F21E99
:100050000C94F21E0C94F21E0C94D26F0D94EE1FB1
:100060000C94F21E0C94965B0C948C5B0C94F21E18
:100070000C94F21E0C94F21E0C94F21E0C94F21EC0
:100080000C94FC530C94F21E0C94F21E0C94F21E71
:100090000C94F21E0C94F21E0C94F21E0C94F21EA0
:1000A0000C94F21E0C94F21E0C94CE530C94F21E7F
:1000B0000C94F21E0C94F21E0C94F21E0C94A0539D
:1000C0000C94F21E0C94F21E0C94F21E0C944F74BD
:1000D0000C9425740C94F21E0C94F21E0C94F21ED7
:1000E0000C94F21E8C1FD21FD81FFF1F0C2015204E
:1000F000202007281929F629212A2D362D363C2BB8
:10010000DF2BF5282D362D36CB2D792FB12F2D361F
:10011000AF312D362D3603332D362D369233C53380
:100120002D3685344035C02FC82FEC2F1030443089
:10013000E730FB30143121312E314231C95BCF5BC6
:10014000E15BF15BF95B265CFD5B265C015C055CB9
:10015000265C095C0D5C115C195C265C235C79D41F
:100160007CD480D483D486D4B0D48AD48DD491D492
:1001700094D497D49BD49ED4A1D4B0D4A5D4A8D4DD
:10018000ABD4E1D9E4D9D3D9D7D9DDD91BDAE8D9B1
:10019000ECD9F2D9F6D9FAD900DA04DA08DA1BDA9E
:1001A0000EDA12DA16DA6F018501BD01CD019D016B
:1001B000DB01B9019701A101130239014D019B0136
:1001C000E501DB015F01C901AB01D3015101490127
:1001D000BB0159012F013D01E101F9018101330109
:1001E000ED01B10109022F012B017701CF01084A6E
:1001F000D73B3BCE016E84BCBFFDC12F3D6C74313B
:100200009ABD56833DDA3D00C77F11BED9E4BB4C91
:100210003E916BAAAABE000000803F05A84CCDB25B
:10022000D44EB93836A9020C50B9918688083CA63C
:10023000AAAA2ABE000000803F000C9444300C940F
:100240000EDA0C94CF5B0C9403330C94195C0C9471
:1002500004DA0C94FF1F0D94621F0C94DD720D9450
:10026000801F0C94CB2D0D94351F0C94A5D40C94A9
:1002700021310D946C040C94C5330D94111F0C9412
:10028000E8D90D9482290C94265C0C94E1D90C9445
:10029000235C0D94F31E0C94EC720D9491040C9459
:1002A000DF2B0D94EE1E0C9483D40C9485340C94A7
:1002B000E7300D94071F0C9416DA0C940D5C0D9426
:1002C00000050C9408DA0C9400DA0C9493730C94E7
:1002D00019290C94AF720C9420200C9446730D9441
:1002E0002B030C9415200C94C95B0C94B0D40D9482
:1002F0006C1F0C9440350C94ABD40C940E730C947E
:1003000092330D942B1F0C94212A0D944D030C94C1
:10031000EC2F0C94015C0C94FD5B0C942D360C942A
:10032000FB300C94D3D90C94AF310C94115C0D9428
:10033000FF030C94F6290D94B6040D94B7030C94A6
:1003400086D40D9422040C94C82F0C948AD40C9457
:100350007CD40C9491D40D944A050D9407290C94E7
:10036000F15B0D944E1F0C943C2B0C948DD40C948B
:10037000DDD90D94DC030D94FD1E0D946D030C94DA
:100380001BDA0C9414310C94792F0C94A8D40C948F
:1003900080D40D9425050C949BD40D9492030D9458
:1003A000761F0C949ED40D94E91E0C94F6D90C94EF
:1003B00042310C94F2D90D946E050C94FAD90C9438
:1003C000F95B0D94191F0C94B12F0D94DB040C9460
:1003D000E15B0C9412DA0C942E310D943F1F0C94B7
:1003E000C02F0C94ECD90C9407280C94095C0C9445
:1003F000D81F0D94211F0C9400730C94D21F0C94E1
:10040000E4D90C9497D40C940C200C94A1D40C94A3
:100410008C1F0D94581F0C94D7D90C9410300C9449
:1004200094D40C94055C0D9447040C94F5280C941A
:1004300079D44E414E494E495459494E46CDCCCCC3
:100440003D0AD7233C17B7D13877CC2B329595E6A8
:10045000241FB14F0A000020410000C84200401C88
:100460004620BCBE4CCA1B0E5AAEC59D7400407AD5
:1004700010F35A00A0724E18090010A5D4E800002D
:10048000E87648170000E40B54020000CA9A3B00CB
:100490000000E1F505000080969800000040420F42
:1004A000000000A08601000000102700000000E806
:1004B00003000000006400000000000A00000000CB
:1004C000000100000000002C76D888DC674F08236C
:1004D000DFC1DFAE59E1B1B796E5E3E453C63AE6D2
:1004E00051997696E8E6C28426EB898C9B62ED40B2
:1004F0007C6FFCEFBC9C9F40F2BAA56FA5F4900501
:100500005A2AF75C936B6CF9676DC11BFCE0E40D34
:1005100047FEF520E6B500D0ED902E030094357728
:10052000050080841E080000204E0A000000C80C50
:10053000333333330F986E12831141EF8D211489B9
:100540003BE65516CFFEE6DB18D1844B381BF77C13
:100550001D901DA4BBE424203284725E228100C958
:10056000F124ECA1E53D274D323520500A4D3234BF
:1005700000526573756D650055492050617573654E
:10058000004E6F204D61746368203A004D33303364
:10059000452D31533635433455004D393939004DE9
:1005A0003530320A4D353030004D3330334530531D
:1005B000323135433855000A202A2A2A726563648D
:1005C00061742E646174615B305D203D0047323898
:1005D0000A4731204631303030205A313000556ED4
:1005E000737570706F72746564204F7074696F6E8C
:1005F0002053656C6563746564004D313930533543
:10060000350A4732380A4732390A4D3430300A4DFC
:10061000313034533231350A4732380A4D313039AE
:10062000533231350A4D34323053310A4731583163
:1006300030305931303046353030300A47315A3059
:100640000A4D3530300A4D31313720536574205A08
:10065000204F666673657400473120463130303074
:10066000205A302E30004732380A47312046313088
:100670003030205A302E30004D353030005A204F67
:100680006666736574203A202573004D353030005E
:100690005A204F6666736574203A202573004732EE
:1006A000385A0A473146313530305A302E300047FB
:1006B00032380A473146313530305A302E30004D0D
:1006C000383400473146313030305A302E30004710
:1006D00032380A473146313030305A302E30005AE5
:1006E000204F6666736574203A202573004D3530BF
:1006F00030004D383400426567696E537769746322
:1007000068007265636461742E61646472203D3DAB
:10071000007265636461742E646174615B305D2096
:100720003D3D0077616974776179203D3D000A2085
:100730002A2A2A4E6F7A7A6C6554656D70537461FB
:100740007475735B325D203D00434F4D4D554E49EE
:10075000434154494F4E0044525952554E00455260
:10076000524F525300494E464F004543484F0047B1
:10077000322F47332062616420706172616D65744D
:100780006572730A00536C6565702E2E2E005A2018
:1007900050726F62652050617374204265640A0074
:1007A0005A2050726F6265205061737420426564F4
:1007B00000486F6D652058592046697273740A00AD
:1007C000486F6D65205859204669727374004D3129
:1007D00031372050726F6265206661696C65642EE6
:1007E0000A4732380A0070726F62655F7265776916
:1007F0007065004469736D69737300473239205224
:1008000065747279696E670050726F62696E6720F5
:100810004661696C6564004D313137204265642062
:100820006C6576656C696E67206661696C65642EBF
:100830000A4730205A31300A4D333030205032359B
:1008400020533838300A4D33303020503530205363
:10085000300A4D3330302050323520533838300A8A
:100860004D333030205035302053300A4D33303046
:100870002050323520533838300A4D333030205034
:1008800035302053300A47342053310070726F6284
:10089000655F6661696C6564004D31313720426582
:1008A00064206C6576656C696E6720646F6E652E7A
:1008B00000205A3A200020593A200042656420580E
:1008C0003A20004D65736820706F696E7420636113
:1008D0006E6E6F74206265207265736F6C766564EE
:1008E0000A004D302F3120427265616B2043616CEC
:1008F0006C656400436F6E74696E7565004D302FD2
:100900003120427265616B2043616C6C6564004EFE
:100910006F204D6F76652E00456E642066696C65AC
:10092000206C6973740A00426567696E2066696CA1
:1009300065206C6973740A004469736D6973730090
:10094000526573756D696E6720534400286E6F2081
:1009500066696C65290043757272656E74206669FC
:100960006C653A20002E0A0044656C6574696F6EF0
:10097000206661696C65642C2046696C653A2000CC
:1009800046696C652064656C657465643A005072F4
:10099000696E742074696D653A20000A537461743D
:1009A000733A2046696C616D656E74207573656479
:1009B0003A20002C204C6F6E67657374206A6F625A
:1009C0003A2000546F74616C2074696D653A2000A0
:1009D00053746174733A20002C204661696C65641D
:1009E0003A20002C2046696E69736865643A2000DD
:1009F0005072696E74733A200053746174733A20B4
:100A0000006F6B006F6666006A0765075E07570731
:100A1000490744454255473A004D31313320530090
:100A200042656420436F6F6C696E672E2E2E004204
:100A300065642048656174696E672E2E2E004348F8
:100A4000414D4245525F54454D50455241545552D7
:100A500045004D4F54494F4E5F4D4F444553005450
:100A60004845524D414C5F50524F54454354494FB5
:100A70004E004155544F5245504F52545F53445FBE
:100A80005354415455530050524F4D50545F535599
:100A900050504F525400454D455247454E43595FC3
:100AA00050415253455200434153455F4C494748DA
:100AB000545F4252494748544E45535300544F47A0
:100AC000474C455F4C494748545300534F46545791
:100AD0004152455F504F574552004255494C445F83
:100AE00050455243454E54004C4556454C494E479F
:100AF0005F44415441005A5F50524F4245004155B6
:100B0000544F4C4556454C005052494E545F4A4F45
:100B1000420050524F4752455353004155544F5293
:100B200045504F52545F54454D5000564F4C554D13
:100B3000455452494300454550524F4D0042494E9D
:100B40004152595F46494C455F5452414E534645C8
:100B5000520053455249414C5F584F4E5F584F46E3
:100B600046004649524D574152455F4E414D453A28
:100B70004D61726C696E20322E305F4457342054C0
:100B80004D33442053534D44424220534F5552431A
:100B9000455F434F44455F55524C3A6874747073D7
:100BA0003A2F2F6769746875622E636F6D2F496ED7
:100BB00073616E6974794175746F6D6174696F6E7C
:100BC0002F4D61726C696E2F747265652F4372656B
:100BD000616C6974795F4D61726C696E322E302E72
:100BE000782050524F544F434F4C5F564552534913
:100BF0004F4E3A312E30204D414348494E455F54C7
:100C00005950453A544D33442043522D58204558AD
:100C10005452554445525F434F554E543A32205535
:100C20005549443A63656465326132662D343161F9
:100C3000322D343734382D396231322D63353563F6
:100C400036326633363766660A002F2F200020467C
:100C50006C6F773A200050726F746563746564201E
:100C600050696E0A00206F7574206F662072616E85
:100C700067650A00536572766F20003A20002053A2
:100C80006572766F2000496E76616C6964206578C4
:100C90007472756465720A0020643A0020693A0033
:100CA00020703A0020643A0020693A0020703A002F
:100CB00064697300656E0043290A0061626C6564B3
:100CC00020286D696E2074656D702000436F6C6420
:100CD0002065787472756465732061726520004DBB
:100CE00065736820706F696E742063616E6E6F74D7
:100CF000206265207265736F6C7665640A004D34FE
:100D0000323120696E636F72726563742070617234
:100D1000616D657465722075736167650A004F6661
:100D20006673657473204170706C69656400457208
:100D3000723A20546F6F206661722100546F6F20E9
:100D40006661722066726F6D207265666572656E8F
:100D5000636520706F696E740A00454550524F4DAF
:100D6000204F4B0A00416476616E6365204B003F63
:100D70004B2076616C7565206F7574206F662072EC
:100D8000616E67652028302D3130292E0A003F54CE
:100D90002076616C7565206F7574206F66207261B6
:100DA0006E67652E0A004572726F722077726974E1
:100DB000696E6720746F20454550524F4D210A00DF
:100DC000363726033C3D380E2E303E121A1C1824AE
:100DD000221E08440AFF430809070001627573795F
:100DE0003A2070617573656420666F7220696E7059
:100DF00075740A00627573793A2070617573656461
:100E000020666F7220757365720A00627573793A95
:100E10002070726F63657373696E670A0053544F75
:100E2000505045442E20005072696E7465722073D4
:100E3000746F707065642064756520746F206572CE
:100E4000726F72732E20466978207468652065720F
:100E5000726F7220616E6420757365204D39393967
:100E600020746F20726573746172742E202854652B
:100E70006D70657261747572652069732072657337
:100E800065742E20536574206974206166746572E0
:100E90002072657374617274696E67290A004E6FFF
:100EA00020436865636B73756D2077697468206C87
:100EB000696E65206E756D6265722C204C6173746D
:100EC000204C696E653A20004E6F20436865636B65
:100ED00073756D2077697468206C696E65206E7516
:100EE0006D6265722C204C617374204C696E653A9A
:100EF0002000636865636B73756D206D69736D6148
:100F00007463682C204C617374204C696E653A20C0
:100F1000004C696E65204E756D62657220697320A4
:100F20006E6F74204C617374204C696E65204E7531
:100F30006D6265722B312C204C617374204C696E8C
:100F4000653A20004D31313000776169740A004DF7
:100F5000313137004D3331005344207265616420D4
:100F60006572726F720A00446F6E65207072696EEE
:100F700074696E672066696C650A004B494C4C20A9
:100F800063617573656420627920746F6F206D757D
:100F9000636820696E6163746976652074696D6544
:100FA000202D2063757272656E7420636F6D6D61A4
:100FB0006E643A200024F4D43050C38E20C2A24084
:100FC00017828B7011127A910D816CD90AA861E198
:100FD00008C7586607615143061E4B5D05C145A70A
:100FE000041A411104093D9803713931034036DB7D
:100FF0000265339102D4305402802E1D02632CEE20
:1010000001752AC501B028A001102781018F256430
:10101000012B244B01E0223401AC211F018D200D56
:1010200001801FFC00841EED00971DDF00B81CD25C
:1010300000E61BC600201BBC00641AB200B219A84F
:10104000000A19A0006A189900D117910040178B67
:1010500000B516840031167E00B31579003A157379
:1010600000C7146F0058146A00EE136600881363FB
:101070000025135E00C7125B006C12570015125456
:1010800000C111510070114F0021114B00D61049C1
:10109000008D1047004610440002104200C00F406F
:1010A00000800F3E00420F3C00060F3B00CB0E3885
:1010B00000930E37005C0E3500270E3400F30D321E
:1010C00000C10D3100900D3000600D2E00320D2D4D
:1010D00000050D2C00D90C2B00AE0C2900850C2925
:1010E000005C0C2700350C27000E0C2600E80B24B2
:1010F00000C40B2400A00B23007D0B23005A0B21FE
:1011000000390B2100180B2000F80A1F00D90A1E15
:1011100000BB0A1E009D0A1D00800A1D00630A1CF8
:1011200000470A1B002C0A1B00110A1A00F7091AB3
:1011300000DD091900C4091900AB0919009209174B
:10114000007B091800630917004C091600360916C0
:1011500000200916000A091500F5081500E008141A
:1011600000CC081400B8081400A408140090081358
:10117000007D0812006B0813005808120046081280
:101180000034081100230811001208110001081191
:1011900000F0071000E0071000D0071000C0071093
:1011A00000B0070F00A107100091070E0083070F82
:1011B0000074070F0065070E0057070E0049070E61
:1011C000003B070D002E070E0020070D0013070D32
:1011D0000006070D00F9060C00ED060D00E0060CF8
:1011E00000D4060C00C8060C00BC060C00B0060CAF
:1011F00000A4060B0099060C008D060B0082060B5E
:101200000077060B006C060B0061060A0057060B00
:10121000004C060A0042060A0038060A002E060A9A
:101220000024060A001A060A001006090007060A2A
:1012300000FD050900F4050900EB050900E20509B8
:1012400000D9050900D0050900C7050900BE050938
:1012500000B5050800AD050800A50509009C0508B6
:1012600000940508008C050800840508007C05082A
:1012700000740508006C050700650508005D05079A
:1012800000560508004E0507004705070040050801
:101290000038050700310507002A05070023050768
:1012A000001C050600160507000F050700080506C7
:1012B0000002050700FB040600F5040700EE040623
:1012C00000E8040600E2040700DB040600D504067B
:1012D00000CF040600C9040600C3040600BD0406CE
:1012E00000B7040600B1040500AC040600A604061D
:1012F00000A00405009B0406009504050090040668
:10130000008A04050085040500800406007A0405AF
:101310000075040500700405006B040500660405F3
:1013200000610405005C0405005704050052040533
:10133000004D04050048040500430405003E040474
:10134000003A04050035040500300404002C0405AF
:101350000027040400230405001E0404001A0404EA
:101360000016040500110404000D0404000904051E
:10137000000404040000040400FC030400F8030457
:1013800000F4030400F0030400EC030400E8030489
:1013900000E4030400E0030400DC030400D80304B9
:1013A00000D4030400D0030400CC030400C80303EA
:1013B00000C503030024F404D9201BC40C5C0E9860
:1013C00004C4095F0265077101F405F900FB04B369
:1013D0000048048700C10369005803550003034512
:1013E00000BE023A008402310053022A002902257D
:1013F0000004022000E4011C00C8011900AF01171D
:1014000000980114008401130071011000610110A3
:101410000051010E0043010D0036010B002B010BA2
:101420000020010B00150109000C0109000301084F
:1014300000FB000800F3000800EB000700E40006D2
:1014400000DE000600D8000600D2000600CC000531
:1014500000C7000500C2000500BD000400B900047B
:1014600000B5000400B1000400AD000400A90004B0
:1014700000A5000300A20003009F0004009B0003DE
:101480000098000300950002009300030090000301
:10149000008D0002008B000300880002008600021D
:1014A0000084000300810002007F0002007D000232
:1014B000007B000200790002007700010076000244
:1014C000007400020072000100710002006F00024F
:1014D000006D0001006C0002006A0001006900025A
:1014E0000067000100660001006500010064000261
:1014F000006200010061000100600001005F000265
:10150000005D0001005C0001005B0001005A000169
:101510000059000100580001005700010056000169
:101520000055000100540001005300000053000169
:10153000005200010051000100500001004F000165
:10154000004E0000004E0001004D0001004C000163
:10155000004B0000004B0001004A0001004900015F
:10156000004800000048000100470001004600005C
:101570000046000100450000004500010044000154
:10158000004300000043000100420000004200014F
:10159000004100000041000100400001003F000048
:1015A000003F0001003E0000003E0001003D000041
:1015B000003D0001003C0000003C0000003C000138
:1015C000003B0000003B0001003A0000003A00012F
:1015D0000039000000390001003800000038000028
:1015E000003800010037000000370001003600001D
:1015F0000036000000360001003500000035000014
:101600000035000100340000003400000034000107
:1016100000330000003300000033000100320000FE
:1016200000320000003200010031000000310000F3
:1016300000310001003000000030000000300001E7
:10164000002F0000002F0000002F0000002F0001DD
:10165000002E0000002E0000002E0001002D0000D2
:10166000002D0000002D0000002D0001002C0000C6
:10167000002C0000002C0000002C0001002B0000BA
:10168000002B0000002B0000002B0001002A0000AE
:10169000002A0000002A0000002A000100290000A2
:1016A0000029000000290000002900000029000195
:1016B000002800000028000000280000002800008A
:1016C000002800010027000000270000002700007C
:1016D000002700000027000100260000002600006F
:1016E0000026000000260000002600010025000062
:1016F0000025000000250000002500000025000056
:101700000025000100240000002400000024000047
:10171000002400000024000100230000002300003A
:10172000002300000023000000230000002300002D
:10173000002300010022000000220000002200001F
:101740000022000000220000002200010021000011
:101750000021000000210000002100000021000005
:1017600000210000002100010020000000200000F6
:1017700000200000002000000020000000200000E9
:101780000020000000200001001F0000001F0000DA
:10179000001F0000001F0000001F0000001F0000CD
:1017A000001F0001001E0000001E0000001E0000BF
:1017B000001E000000232C0000B822000056180074
:1017C000003A0F0000B8080000B1040000710200E8
:1017D000003E0100002020506C616E6E6572427503
:1017E0006666657242797465733A200020467265B8
:1017F00065204D656D6F72793A2000436F6D706999
:101800006C65643A204F63742032372032303139AE
:101810000A00204C61737420557064617465643AE9
:1018200020323031392D31302D3035207C2041753A
:1018300074686F723A2054696E794D616368696E9D
:10184000657333440A00322E305F4457340A004D2A
:1018500061726C696E0020536F66747761726520E7
:1018600052657365740A00205761746368646F671A
:101870002052657365740A002042726F776E206F84
:1018800075742052657365740A002045787465721A
:101890006E616C2052657365740A00506F776572D3
:1018A00055700A0073746172740A006175746F2553
:1018B000632E67006572726F722077726974696E49
:1018C0006720746F2066696C650A00446F6E65203E
:1018D000736176696E672066696C652E0A004D3209
:1018E0003900205A3A0020593A0020583A00656ED3
:1018F0006473746F7073206869743A2000473238DB
:10190000585900453120544845524D414C205255BC
:101910004E415741590042454420544845524D419B
:101920004C2052554E4157415900546865726D61C3
:101930006C2052756E617761790045312045727275
:101940003A204D415854454D50004572723A204D51
:10195000415854454D5020424544004D415854454E
:101960004D50207472696767657265640045312067
:101970004572723A204D494E54454D5000457272A1
:101980003A204D494E54454D5020424544004D4962
:101990004E54454D502074726967676572656400E6
:1019A0000A0A0020205A5F4D494E3A002020595F14
:1019B0004D494E3A002020585F4D494E3A004D386F
:1019C0003420582059205A204500202F0020424022
:1019D0003A0020403A00436F6F6C696E672E2E2EDE
:1019E0000048656174696E672E2E2E0045202553D0
:1019F0000020573A0020573A00496E76616C6964BE
:101A00002065787472756465720A00416374697642
:101A1000652045787472756465723A2000486F7469
:101A2000656E6420746F6F20636F6C640A0043619D
:101A30006E6E6F74206F70656E207375626469726C
:101A4000200053442063617264206F6B0A006F7042
:101A5000656E526F6F74206661696C65640A00760A
:101A60006F6C756D652E696E6974206661696C6551
:101A7000640A00534420696E6974206661696C0AC7
:101A8000004D3234004D3233202573005772697493
:101A9000696E6720746F2066696C653A20002E0AB3
:101AA000006F70656E206661696C65642C20466904
:101AB0006C653A20002E0A006F70656E20666169C1
:101AC0006C65642C2046696C653A200046696C653B
:101AD0002073656C65637465640A002053697A65D8
:101AE0003A200046696C65206F70656E65643A2027
:101AF00000667265736800646F696E6700206669CE
:101B00006C653A20004E6F772000454E44205355B7
:101B100042524F5554494E450A002220706F7300BF
:101B20002220706172656E743A2200535542524F02
:101B30005554494E452043414C4C207461726765B1
:101B4000743A2200747279696E6720746F20636141
:101B50006C6C207375622D67636F64652066696CB9
:101B60006573207769746820746F6F206D616E797A
:101B7000206C6576656C732E204D4158206C65761F
:101B8000656C2069733A310A005344207072696EA3
:101B900074696E67206279746520004E6F742053FB
:101BA00044207072696E74696E670A0057616974C7
:101BB000696E6720666F72206865617475702E0AA1
:101BC000004C656176696E6720473236003F53707E
:101BD0006563696669656420582C5920636F6F726C
:101BE00064696E617465206F7574206F6620626F22
:101BF000756E64732E0A003F285229657065617402
:101C00002076616C7565206E6F7420706C617573E1
:101C100069626C653B206D75737420626520617428
:101C2000206C6561737420312E0A003F28522965AB
:101C300070656174206D75737420626520737065C2
:101C4000636966696564207768656E206E6F7420CD
:101C50007573696E6720616E204C43442E0A003F05
:101C6000537065636966696564206E6F7A7A6C6526
:101C70002074656D7065726174757265206E6F7425
:101C800020706C61757369626C652E0A003F537039
:101C9000656369666965642066696C616D656E740B
:101CA0002073697A65206E6F7420706C617573693A
:101CB000626C652E0A003F537065636966696564EE
:101CC000207072696D65206C656E677468206E6F38
:101CD0007420706C61757369626C652E0A003F50E8
:101CE00072696D65206C656E677468206D757374BC
:101CF0002062652073706563696669656420776832
:101D0000656E206E6F74207573696E6720616E203A
:101D10004C43442E0A003F537065636966696564ED
:101D2000206E6F7A7A6C652073697A65206E6F74A5
:101D300020706C61757369626C652E0A003F526594
:101D40007472616374696F6E204D756C7469706C28
:101D5000696572206D7573742062652073706563A8
:101D600069666965642E0A003F5370656369666938
:101D700065642052657472616374696F6E204D757D
:101D80006C7469706C696572206E6F7420706C6120
:101D9000757369626C652E0A003F537065636966EE
:101DA000696564206C61796572206865696768742B
:101DB000206E6F7420706C61757369626C652E0A99
:101DC0000043292E0A003F537065636966696564A4
:101DD000206265642074656D7065726174757265EA
:101DE000206E6F7420706C61757369626C65202859
:101DF00034302D00473236207374617274696E6717
:101E00002E2E2E0A0020746F6F206C6F6E67206577
:101E10007874727573696F6E2070726576656E7412
:101E200065640A0020636F6C642065787472757352
:101E3000696F6E2070726576656E7465640A007CE9
:101E40003C3E5E2B3D3F2F5B5D3B2C2A225C0020FD
:101E500042002050006F6B00526573656E643A203B
:101E60000043616E6E6F74206F70656E20737562D3
:101E700064697220002569730025696D20256973E6
:101E8000002569682025696D20256973002569642E
:101E9000202569682025696D2025697300256979E9
:101EA00020256964202569682025696D20256973CE
:101EB0000023646566696E652044454641554C546F
:101EC0005F0000626564004B6420004B6920004B9A
:101ED000702000504944204175746F74756E652000
:101EE00066696E6973686564212050757420746832
:101EF00065206C617374204B702C204B6920616EDF
:101F000064204B6420636F6E7374616E747320661B
:101F1000726F6D2062656C6F7720696E746F2043FD
:101F20006F6E66696775726174696F6E2E680A00FC
:101F3000504944204175746F74756E6520666169FF
:101F40006C6564212074696D656F75740A00453194
:101F500020544845524D414C2052554E415741590D
:101F60000042454420544845524D414C2052554E64
:101F70004157415900546865726D616C2052756E0D
:101F8000617761790045312048656174696E672029
:101F90004661696C656400426564204865617469E6
:101FA0006E67204661696C65640048656174696E9E
:101FB00067206661696C656400504944204175740E
:101FC0006F74756E65206661696C65642120546567
:101FD0006D706572617475726520746F6F206869C9
:101FE00067680A00204B643A2000204B693A2000C1
:101FF000204B703A20000A20436C617373696320A0
:10200000504944200A00204B643A2000204B693A92
:102010002000204B703A20000A204E6F206F76651A
:102020007273686F6F740A002054753A2000204B59
:10203000753A2000206D61783A2000206D696E3A73
:10204000200020643A200020626961733A20005029
:102050004944204175746F74756E652073746172A4
:10206000740A00504944204175746F74756E652080
:102070006661696C6564212054656D706572617478
:1020800075726520746F6F20686967680A0050492F
:1020900044204175746F74756E65206661696C6566
:1020A00064212042616420657874727564657220D1
:1020B0006E756D6265720A0050726F62696E67209C
:1020C000506F696E740025532025692F2569002EF5
:1020D0000A002F0050726F62696E67206D65736829
:1020E00020706F696E742000202844525952554E5A
:1020F0002900473239204175746F20426564204CB5
:102100006576656C696E67003F20284C2C522C4622
:102110002C4229206F7574206F6620626F756E6483
:10212000732E0A003F2856296572626F7365206C12
:102130006576656C20696D706C61757369626C653C
:102140002028302D34292E0A00426164205A20763E
:10215000616C75650A004E6F2062696C696E65611D
:102160007220677269640A005374616E64617264FC
:1021700020446576696174696F6E3A20002052616F
:102180006E67653A2000204D61783A2000204D6945
:102190006E3A20004D65616E3A200046696E6973A3
:1021A000686564210A002072616E67653A2000202C
:1021B0006D61783A2000206D696E3A2000207369C5
:1021C000676D613A2000206D65616E3A20003A200B
:1021D0007A3A2000206F662000205900476F696E10
:1021E0006720746F3A20580043570A0020646972D0
:1021F0003A0020616E676C653A0053746172742016
:102200007261646975733A00506F736974696F6EB7
:10221000696E67207468652070726F62652E2E2E5D
:102220000A003F4E756D626572206F66206C6567AF
:102230007320696E206D6F76656D656E74206E6FAC
:102240007420706C61757369626C652028302D3163
:1022500035292E0A003F2028582C5929206F7574E3
:10226000206F6620626F756E64732E0A003F5361A3
:102270006D706C652073697A65206E6F7420706C68
:1022800061757369626C652028342D3530292E0AFA
:10229000004D3438205A2D50726F6265205265709F
:1022A0006561746162696C69747920546573740A3C
:1022B000003F2856296572626F7365206C657665EC
:1022C0006C20696D706C61757369626C6520283073
:1022D0002D34292E0A00290A002062797465733B87
:1022E00020637263200053657474696E67732053B2
:1022F000746F726564202800454550524F4D20642C
:1023000061746173697A65206572726F722E0A005A
:10231000290A002062797465733B20637263200090
:102320002073746F7265642073657474696E67736B
:1023300020726574726965766564202800202863C0
:10234000616C63756C6174656429210A0020213D0C
:102350002000454550524F4D20435243206D697334
:102360006D61746368202D202873746F7265642911
:1023700020002053697A653A2000496E6465783AF6
:102380002000204D61726C696E3D563730290A007D
:10239000454550524F4D2076657273696F6E206DC2
:1023A00069736D617463682028454550524F4D3DF7
:1023B00000205A3A0020593A0020436F756E74206D
:1023C000583A0020453A00205A3A0020593A00581D
:1023D0003A0000809D4300009A430000C84300007B
:1023E0000000000000000000000020746F6F206CEF
:1023F0006F6E6720657874727573696F6E20707286
:102400006576656E7465640A0020636F6C64206590
:102410007874727573696F6E2070726576656E740C
:1024200065640A00000000000000000000000000D9
:102430000000484200004842000080405761726E30
:10244000696E673A20486F6D696E672042756D70DE
:102450002044697669736F72203C20310A000202C1
:10246000040000A0400000A0400000004000809D4B
:102470004300009A430000C843FFFFFF0000000133
:10248000000000010000800055555500000040008C
:1024900033333300AAAA2A00499224000000200006
:1024A000C7711C0099991900D145170055551500A1
:1024B0003BB113002449120011111100000010005B
:1024C0000F0F0F00E3380E0043790D00CCCC0C0049
:1024D000C3300C00E8A20B0064210B00AAAA0A007A
:1024E000703D0A009DD80900427B09009224090032
:1024F000DCD30800888808001042080000000800AB
:10250000F0C107008787070075500700711C07009E
:102510003EEB0600A1BC0600699006006666060058
:10252000703E06006118060017F4050074D105001E
:102530005BB00500B29005006272050055550500BC
:1025400078390500B81E0500050505004EEC0400AD
:1025500087D40400A1BD040090A7040049920400A0
:10256000C17D0400EE690400C75604004444040021
:102570005C32040008210400411004000000040043
:102580003FF00300F8E0030026D20300C3C30300BA
:10259000CCB503003AA803000A9B0300388E030061
:1025A000C08103009F750300D0690300505E0300E3
:1025B0001D53030034480300913D030033330300EF
:1025C00016290300381F030097150300300C030081
:1025D000030303000BFA020049F10200BAE802000B
:1025E0005CE002002DD802002DD0020059C8020084
:1025F000B0C0020031B90200DAB10200AAAA02009A
:10260000A0A30200BC9C0200FA9502005C8F0200AD
:10261000DF88020082820200457C020027760200E9
:1026200027700200436A02007C640200D05E020050
:102630003F590200C853020053544F502063616C4D
:102640006C65642062656361757365206F66204206
:102650004C546F756368206572726F72202D207202
:102660006573746172742077697468204D393939E3
:102670000A0053544F502063616C6C65642062659E
:102680006361757365206F6620424C546F75636893
:10269000206572726F72202D20726573746172747E
:1026A0002077697468204D3939390A002F2F61630A
:1026B00074696F6E3A00627574746F6E00656E6453
:1026C0000070726F6D70745F0073686F77004D38C3
:1026D000373620526573706F6E64696E6720505292
:1026E0004F4D50545F00554E4B4E4F574E20535454
:1026F0004154450047434F44455F494E464F004CC7
:1027000043445F50415553455F524553554D450035
:1027100046494C414D454E545F52554E4F55545FBE
:10272000434F4E54494E55450046494C414D454E48
:10273000545F52554E4F5554004D323400436F6E26
:1027400074696E7565005075726765204D6F7265AE
:10275000005061757365640070617573656400484D
:102760006F74656E6420746F6F20636F6C640A0011
:102770004469736D697373005061757365005072BD
:1027800065737320627574746F6E20286F72204DAC
:102790003130382920746F20726573756D650A00B9
:1027A000496E736572742066696C616D656E742024
:1027B000616E6420707265737320627574746F6EDD
:1027C00020286F72204D313038290A00436F6E7413
:1027D000696E75650052656865617420446F6E6549
:1027E00000526568656174696E672E2E2E00526511
:1027F00068656174696E67004865617465725469E3
:102800006D656F7574005265686561740048656137
:1028100074657254696D656F757400507265737379
:1028200020627574746F6E20286F72204D313038BD
:102830002920746F2068656174206E6F7A7A6C65E8
:102840000A004E6F7A7A6C65205061726B65640085
:10285000436F6E74696E7565004E6F7A7A6C652091
:102860005061726B656400486F74656E6420746FAC
:102870006F20636F6C640A00726573756D65640028
:10288000626567696E00436F6E74696E75650050AE
:10289000757267654D6F7265005061757365640090
:1028A0004C6F61642046696C616D656E7400436FA6
:1028B0006E74696E7565004C6F61642046696C6169
:1028C0006D656E74205400496E736572742066697C
:1028D0006C616D656E7420616E64207072657373D7
:1028E00020627574746F6E20286F72204D313038FD
:1028F000290A004469736D69737300526573756DBD
:10290000696E67005A5F53544F505F50494E005AEA
:102910005F535445505F50494E005A5F4D494E5FDA
:1029200050494E005A5F454E41424C455F50494E1A
:10293000005A5F4449525F50494E005A5F43535F0B
:1029400050494E00595F53544F505F50494E005903
:102950005F535445505F50494E00595F4D494E5F9B
:1029600050494E00595F454E41424C455F50494EDB
:1029700000595F4449525F50494E00595F43535FCD
:1029800050494E00585F53544F505F50494E0058C5
:102990005F535445505F50494E00585F4D494E5F5C
:1029A00050494E00585F454E41424C455F50494E9C
:1029B00000585F4449525F50494E00585F43535F8F
:1029C00050494E0053535F50494E00534552564FA5
:1029D000335F50494E00534552564F325F50494E77
:1029E00000534552564F315F50494E0053455256A1
:1029F0004F305F50494E00534453530053445F449B
:102A000045544543545F50494E0053434B5F504932
:102A10004E0052414D50535F44395F50494E005271
:102A2000414D50535F44385F50494E0052414D5024
:102A3000535F4431305F50494E004D4F53495F5012
:102A4000494E004D4F534645545F445F50494E0038
:102A50004D49534F5F50494E004D4158363637353A
:102A60005F53535F50494E004C45445F50494E0000
:102A70004845415445525F4245445F50494E0048E5
:102A800045415445525F305F50494E0046494C5FC6
:102A900052554E4F55545F50494E0046414E315F9E
:102AA00050494E0046414E5F50494E0045315F53FC
:102AB0005445505F50494E0045315F454E41424CB0
:102AC000455F50494E0045315F4449525F50494E81
:102AD0000045315F43535F50494E0045305F5354CA
:102AE00045505F50494E0045305F454E41424C4590
:102AF0005F50494E0045305F4449525F50494E0097
:102B000045305F43535F50494E00455F4D55583245
:102B10005F50494E00455F4D5558315F50494E005A
:102B2000455F4D5558305F50494E00424545504530
:102B3000525F50494E004156525F53535F50494EC9
:102B4000004156525F53434B5F50494E004156522D
:102B50005F4D4F53495F50494E004156525F4D49BA
:102B6000534F5F50494E0054454D505F4245445FBE
:102B700050494E0054454D505F315F50494E00540E
:102B8000454D505F305F50494E0046494C574944CF
:102B900054485F50494E0054584400525844003A3B
:102BA000200020202020434F4D002020206E6F6EFB
:102BB0002D7374616E646172642050574D206D6F87
:102BC000646500202020636F6D7061726520696EFE
:102BD0007465727275707420656E61626C656400F4
:102BE0002020206F766572666C6F7720696E746541
:102BF000727275707420656E61626C6564003A2053
:102C0000002020202054494D534B00423A20002000
:102C10002020205443435200413A2000202020200D
:102C200054434352002020202043533A20002020C8
:102C3000202057474D3A200050574D3A2020253448
:102C4000640050574D3A2020253464004700480066
:102C5000000088008A008C00B300B40000009800D7
:102C60009A009C00A800AA00AC0028012A012C01AF
:102C70002020202054494D455200440045006E005C
:102C8000800081006F00B000B100700090009100E2
:102C90007100A000A10072002001210173002069D1
:102CA0007320616C736F207469656420746F207485
:102CB0006869732070696E0054494D455231430074
:102CC0000A202E002020002020506F72743A20002D
:102CD00020202000202020416E616C6F6720696EEB
:102CE000203D2025356C64003C756E757365642F3E
:102CF000756E6B6E6F776E3E002028412532642919
:102D00002020002533642000257350494E3A2000CE
:102D10004F7574707574203D2000496E7075742075
:102D2000203D2000416E616C6F6720696E203D2060
:102D300025356C640070726F74656374656420007F
:102D400020284125326429202000253364200025D5
:102D50007350494E3A20009B2B0001972B01018AAA
:102D60002B3B007F2B4300742B4500672B44005AFC
:102D70002B32014D2B3301412B3401362B35012BE6
:102D80002B2501202B2801152B2A010A2B2C0100B1
:102D90002B2A01F52A1C01E72A1801DB2A1A01D186
:102DA0002A2C01C62A2201B82A1E01AC2A2401A419
:102DB0002A09019B2A07018C2A02017F2A0A017035
:102DC0002A0801682A0D01592A4201502A3201437A
:102DD0002A07013A2A33012C2A0A011F2A08011264
:102DE0002A09010A2A3401FC293101F7293501ECAD
:102DF000290B01E1290601D6290501CB290401C4CB
:102E0000293501BB293501B1293701A42926019AA9
:102E10002903018F293601842903017B293101719E
:102E2000293D01642938015A290E014F293C0144EA
:102E3000290E013B2928013129300124293E011A9C
:102E40002912010F292E0104291201446F6E652EEB
:102E50000A0066616C7365004641494C3A204E6F2A
:102E60002074726967676572206465746563746550
:102E7000640A004641494C3A204E6F6973652064EC
:102E800065746563746564202D20706C656173657D
:102E90002072652D72756E20746573740A0020644B
:102EA000657465637465642E0A003D20424C546F5E
:102EB000756368207072652056332E3120286F723A
:102EC00020636F6D70617469626C6529003D205AE2
:102ED00020536572766F2050726F6265003D20420C
:102EE0004C546F7563682056332E310020282B2FE9
:102EF0002D20346D73293A20003A2033306D732031
:102F00006F72206D6F72650A002E2050756C7365AC
:102F1000207769647468002A2A20506C65617365A3
:102F200020747269676765722070726F62652077BE
:102F3000697468696E20333020736563202A2A0A19
:102F4000004641494C3A20424C544F554348206575
:102F50006E61626C6564202D20536574207570204D
:102F600074686973206465766963652061732061A4
:102F700020536572766F2050726F62652077697496
:102F80006820494E56455254494E47207365742077
:102F9000746F202774727565272E0A00202044451F
:102FA000504C4F5945442073746174653A204C4F1E
:102FB0005720286C6F676963203029002020444522
:102FC000504C4F5945442073746174653A20484908
:102FD000474820286C6F676963203129003D204DE8
:102FE000656368616E6963616C20537769746368B7
:102FF0002064657465637465640A005741524E49E4
:103000004E473A20494E56455254494E4720736523
:103010007474696E672070726F6261626C7920628D
:1030200061636B77617264732E0A002E20446570B1
:103030006C6F7920262073746F7720342074696D4B
:1030400065730A003D20424C546F75636820436CE1
:10305000617373696320312E322C20312E332C2082
:10306000536D61727420312E302C20322E302C2082
:10307000322E322C20332E302C20332E312064651A
:103080007465637465642E0A002E20436865636B63
:1030900020666F7220424C544F5543480A002E2040
:1030A0005A5F4D494E5F454E4453544F505F494E11
:1030B00056455254494E473A20002E2050726F62B6
:1030C00065205A5F4D494E5F50494E3A20002C20F2
:1030D00073746F7720616E676C653A202020002C36
:1030E000206465706C6F7920616E676C653A2000B2
:1030F000536572766F2070726F62652074657374A9
:103100000A2E207573696E6720696E6465783A20AF
:1031100020004D343320576169742043616C6C6525
:103120006400436F6E74696E7565004D34332057CB
:103130006169742043616C6C6564005761746368F5
:10314000696E672070696E730A0064697300656E4A
:103150000061626C65640A00656E6473746F702050
:103160006D6F6E69746F72200000002100240027CB
:10317000002A002D00300033000101000004010787
:10318000010A0100002200250028002B002E00313A
:1031900000340002010000050108010B01000020BD
:1031A000002300260029002C002F0032000001001F
:1031B00000030106010901050505050705080808C2
:1031C00008020202020A0A080804040404010101B8
:1031D00001010101010303030303030303040707C0
:1031E000070C0C0C0C0C0C0C0C020202020606065E
:1031F00006060606060B0B0B0B0B0B0B0B01021046
:103200002020080810204010204080020102010800
:1032100004020101020408102040808040201008B0
:103220000402018004020180402010080402010809
:103230000402010102040810204080010204081069
:1032400020408000000A0B02090C0D0E0807030441
:10325000010000000000000000000000000000006D
:10326000000000000000000000000000000000124C
:10327000111000000000000000000000000000002D
:1032800000000000000000000050726F62696E676D
:10329000204661696C65640A0050726F62696E67EE
:1032A000204661696C656400205A3A200020593A32
:1032B000200042656420583A2000486F6D65202543
:1032C000732573257320466972737400220A0055B2
:1032D0006E6B6E6F776E20636F6D6D616E643A20FA
:1032E0002200204500205A00205900204D3932206C
:1032F00058004F4646004F4E00205A0020590020EB
:10330000580020204D61783A2000200020204D698F
:103310006E3A2000536F667420656E6473746F702C
:10332000733A20005761726E696E67203A20436CD1
:1033300065616E20436972636C65207265717569A1
:103340007265732058590A004732380020496E765A
:10335000616C696420657874727564657220000A16
:1033600020696E6974207A70726F62655F7A6F6629
:1033700066736574203D2000454550524F4D2049ED
:103380006E697469616C697A65640A004861726487
:10339000636F6465642044656661756C7420536571
:1033A0007474696E6773204C6F616465640A000011
:1033B00000FA430000FA430000204100009642005A
:1033C00000A0420000A0420000C8430000BE42DC52
:1033D000050000DC050000640000004B0000003A1E
:1033E0000A0020204D3630332000546F6F6C2D635F
:1033F00068616E67696E673A0A0020550054312093
:103400004C002055005430204C0046696C616D65BD
:103410006E74206C6F61642F756E6C6F6164206CCC
:10342000656E677468733A0A00204B0020204D399E
:1034300030302054004C696E6561722041647661C1
:103440006E63653A0A00205A0020590020204D384A
:1034500035312058005A2D50726F6265204F6666D4
:103460007365740020440020490020204D3330341F
:1034700020500020440020490020204D33303120CE
:1034800050005049442073657474696E67733A0A3A
:1034900000205A00204A0020204732392057204976
:1034A00000205A0020204D343230205300417574E2
:1034B0006F20426564204C6576656C696E673A0AD8
:1034C00000205A0020590020204D3230362058006C
:1034D000486F6D65206F66667365743A0A00204A0E
:1034E0000020540020530020204D3230352042006F
:1034F000204A3C6A756E635F6465763E004164767F
:10350000616E6365643A20423C6D696E5F73656706
:103510006D656E745F74696D655F75733E20533CB5
:103520006D696E5F66656564726174653E20543CCA
:103530006D696E5F74726176656C5F6665656472F5
:103540006174653E0020540020520020204D32302E
:1035500034205000416363656C65726174696F6EFD
:103560002028756E6974732F7332293A20503C708D
:1035700072696E745F616363656C3E20523C726574
:1035800074726163745F616363656C3E20543C7464
:10359000726176656C5F616363656C3E0A0020450D
:1035A00000205A0020590020204D32303120580090
:1035B0004D6178696D756D20416363656C657261FD
:1035C00074696F6E2028756E6974732F7332293A8F
:1035D0000A00204500205A0020590020204D32309A
:1035E000332058004D6178696D756D20666565649E
:1035F00072617465732028756E6974732F73293A2C
:103600000A0053746570732070657220756E69745A
:103610003A0A0020204D3230302044300A00202069
:103620004D32303020543120440020204D32303093
:103630002044002044697361626C65640A00466935
:103640006C616D656E742073657474696E67733A2E
:103650000020286D6D2900202047323120202020B5
:103660003B20556E69747320696E206D6D00486F44
:103670006D696E67204661696C6564006F70656E88
:1036800000545249474745524544003A20007A5F6A
:103690006D696E00795F6D696E00785F6D696E00AF
:1036A0005265706F7274696E6720656E6473746FB3
:1036B00070207374617475730A00446966663A20F9
:1036C0000046726F6D5374703A0053746570706584
:1036D000723A00556E4C6576656C3A004C657665BD
:1036E0006C65643A005261773A20202020000A4C31
:1036F0006F676963616C3A004361703A00426162CE
:103700007973746570205A0050726F6265204F663D
:1037100066736574205A0050726F6265204F66664A
:103720007365745A3A2000290A0020746F20003F04
:103730005A206F7574206F662072616E676520284D
:1037400000290A0020746F20003F59206F757420F3
:103750006F662072616E676520282D00290A00209F
:10376000746F20003F58206F7574206F662072615F
:103770006E676520282D00205A0020590050726F76
:103780006265204F6666736574205800220A0065E2
:103790006E7175657565696E672022002E0A006F6F
:1037A00070656E206661696C65642C2046696C6585
:1037B0003A2000706F7765726F6666004B494C4C1B
:1037C00045442E20005072696E7465722068616CE9
:1037D0007465642E206B696C6C28292063616C6CA5
:1037E0006564210A00FFFDFCFAF8F6F4F2F0EEEC55
:1037F000EAE9E7E5E3E1E0DEDCDAD9D7D5D4D2D0F7
:10380000CFCDCBCAC8C7C5C3C2C0BFBDBCBAB9B78C
:10381000B6B4B3B2B0AFADACAAA9A8A6A5A4A2A1F4
:10382000A09E9D9C9A99989795949392908F8E8D37
:103830008B8A8988878684838281807F7E7D7B7A5C
:10384000797877767574737271706F6E6D6C6B6A60
:10385000696867666564636261605F5E5D5C5B5A50
:103860005958585756555453525150504F4E4D4C2D
:103870004B4A4A4948474646454443424241403FF5
:103880003E3E3D3C3B3B3A393838373635353433AC
:1038900032323130302F2E2E2D2C2B2B2A29292855
:1038A000272726252524232322212120201F1E1EF1
:1038B0001D1C1C1B1B1A1919181817161615151480
:1038C000131312121111100F0F0E0E0D0D0C0C0B05
:1038D0000A0A090908080707060605050404030380
:1038E0000202010000205400205200416363656C15
:1038F00065726174696F6E3A2050003F4A206F759F
:1039000074206F662072616E67652028302E30311A
:1039100020746F20302E33290A00546F6F6C636857
:10392000616E67653A0020204D32313700205A0021
:10393000205900205800205200205000204500202F
:10394000530050574D3A20202534640050574D3ACB
:1039500020202534640050574D3A2020253464003F
:1039600050574D3A20202534640050574D3A2020BE
:103970002534640050574D3A2020253464005057B8
:103980004D3A20202534640050574D3A20202534EC
:10399000640050574D3A20202534640050574D3A6A
:1039A00020202534640050574D3A202025346400EF
:1039B00050574D3A20202534640050574D3A20206E
:1039C0002534640050574D3A202025346400505768
:1039D0004D3A20202534640050574D3A202025349C
:1039E000640070012C0190012701B0012201C00187
:1039F0001D01F00118011002130130020E016002D6
:103A0000090190020401C002FF000003FA00400314
:103A1000F5008003F000D003EB002004E600700402
:103A2000E100E004DC004005D700C005D2004006FC
:103A3000CD00D006C8008007C3003008BE00F008E3
:103A4000B900C009B400B00AAF00B00BAA00D00C96
:103A5000A500000EA000500F9B00C0109600501251
:103A6000910000148C00C0158700B0178200B019B7
:103A70007D00D01B7800001E730040206E00902255
:103A80006900F024640040275F0090295A00E02B71
:103A90005500102E500020304B0010324600E0330D
:103AA000410090353C001037370070383200A039A3
:103AB0002D00B03A2800A03B2300603C1E00103DC2
:103AC0001900903D1400103E0F00703E0A00C03EE9
:103AD0000500003F0000403FFBFF803FF6FFC03F76
:103AE000F1FF626564002C2073797374656D207337
:103AF000746F7070656421204865617465725F49F8
:103B0000443A20004265642048656174696E67200C
:103B10004661696C65640048656174696E6720661A
:103B200061696C65640042454420544845524D41EA
:103B30004C2052554E4157415900546865726D6191
:103B40006C2052756E61776179004531204865615E
:103B500074696E67204661696C65640048656174CC
:103B6000696E67206661696C656400453120544860
:103B700045524D414C2052554E41574159005468D1
:103B800065726D616C2052756E6177617900202DD0
:103B900020496E76616C696420657874727564651D
:103BA00072206E756D62657220210A001000C902D4
:103BB00010012C014001220170011801B0010E0119
:103BC000F00104015002FA00B002F0003003E600F8
:103BD000D003DC009004D2007005C800A006BE002F
:103BE0000008B400B009AA00D00BA000600E960037
:103BF00060118C000015820020197800C01D6E0035
:103C0000A0226400B0275A00902C500000314600DA
:103C1000E0343C0010383200903A2800603C1E002E
:103C2000A03D1400803E0A00203F000053544F5036
:103C30005045442E20005072696E74657220737472
:103C40006F707065642064756520746F2065727292
:103C50006F72732E204669782074686520657272D1
:103C60006F7220616E6420757365204D393939207B
:103C7000746F20726573746172742E202854656DA0
:103C80007065726174757265206973207265736501
:103C9000742E2053657420697420616674657220E7
:103CA00072657374617274696E67290A006563686E
:103CB0006F3A004572726F723A0042696C696E65C4
:103CC0006172204C6576656C696E67204772696425
:103CD0003A0A00544D33442043522D582052656116
:103CE00064792E005072696E74696E672E2E2E00F4
:103CF0005072696E74205061757365640063616E03
:103D000063656C005072696E742041626F727465F5
:103D100064004469736D6973730055492041626F93
:103D20007274656400726573756D65004D323400A0
:103D30004F46460A004661646520486569676874B5
:103D40002000426564204C6576656C696E672000D2
:103D50004661696C656420746F20656E61626C6594
:103D600020426564204C6576656C696E670A00497F
:103D70006E76616C6964206D6573682E0A0041017E
:103D8000AD0111241FBECFEFD1E2DEBFCDBF00E0F9
:103D90000CBF18E0A0E0B2E0E8EBF5E702E00BBFF3
:103DA00002C007900D92AC33B107D9F72FE1ACE315
:103DB000B8E001C01D92A333B207E1F71EE1C0ECE9
:103DC000DEE100E006C021970109802FFE010F947B
:103DD0000537CF3BD10780E00807A9F70F943820BB
:103DE0000D94CA3A0C9400002F923F924F925F922A
:103DF0006F927F928F929F92AF92BF92CF92DF92FB
:103E0000EF92FF920F931F93CF93DF93CDB7DEB75F
:103E1000A7970FB6F894DEBF0FBECDBF8091090102
:103E2000817091E0982720915B08921781F190931F
:103E30005B08811116C00E942C758091EB1783FFDF
:103E400009C08AED93E00E94355561E080E00E9450
:103E50001CDA1DC060E081E00E941CDA83EF93E071
:103E600014C00091EB1703FB002700F90E94BB74FC
:103E70008091EB17877F8093EB17002341F060E080
:103E800081E00E941CDA8CE094E00E94355580911C
:103E90005A0881110C944D3A809158089091590814
:103EA0009C012F5F3F4F3093590820935808883E5C
:103EB000934010F40C944D3A81E080935A0810928C
:103EC0005908109258088091A818882309F48CC3C7
:103ED0000E94C9A1811188C3809157088F5F809388
:103EE000570880915708853620F010925708109295
:103EF000A818E091A8188E2FEE0F990BAA0BBB0BF8
:103F0000FC013197E730F10508F0A0C08827EE5892
:103F1000FF4F8F4F0D9405370E94C1A1882309F4EC
:103F200095C081E0809370028FE194E00E94355546
:103F300080E190E09093701680936F1685E08093F7
:103F4000631602E80093661684E190E1A0E0B0E019
:103F50008093671690936816A0936916B0936A16BB
:103F60000E9405FA81E09AE59093701680936F168F
:103F700086E390E0909372168093711687E08093A9
:103F800063160093661684E890E0A0E0B0E08093AA
:103F9000671690936816A0936916B0936A160E94EC
:103FA00005FA52C00E94C1A1882309F44FC048C03D
:103FB0008DE294E00E94355581E09AE59093701669
:103FC00080936F1680E490E0909372168093711640
:103FD00007E00093631682E88093661684E890E019
:103FE000A0E0B0E08093671690936816A0936916DE
:103FF000B0936A160E9405FA0093A81827C0809112
:104000005608882319F10E94C1A18823F9F00E9463
:10401000C9A181111BC0EBC20E94C1A18823B1F0CC
:104020000E94C9A1811112C010C30E94C9A18111AF
:104030000DC042E060E070E0CB010E94DFA104C04F
:104040000E94C9A1811102C01092A818809170022B
:10405000882309F4B1C28091A4189091A518892BE6
:1040600009F08FC18091530890915408892B09F071
:104070001EC184E096E09093701680936F1680EADC
:1040800090E8909372168093711617E01093631660
:1040900002E80093661680EA90E0A0E0B0E080932A
:1040A000671690936816A0936916B0936A160E94DB
:1040B00005FA8091130290911402A0911502B0911B
:1040C00016020097A105B10511F510927016109215
:1040D0006F1615E010936316009366168AE890E158
:1040E000A0E0B0E08093671690936816A0936916DD
:1040F000B0936A160E9405FA89E090E090937016DA
:1041000080936F16109363160093661640C0019655
:10411000A11DB11D65E0B695A795979587956A9500
:10412000D1F70197A109B109009721E0A207B105D4
:1041300058F0B0937016A0936F16909372168093F8
:1041400071161093631607C09093701680936F16C4
:1041500085E08093631612E8109366168AE890E172
:10416000A0E0B0E08093671690936816A09369165C
:10417000B0936A160E9405FA88E090E0909370165A
:1041800080936F1685E080936316109366168CE813
:1041900090E1A0E0B0E08093671690936816A0933A
:1041A0006916B0936A160E9405FA809113029091E5
:1041B0001402A0911502B0911602009731E0A307F6
:1041C000B10550F0B0937016A0936F1690937216CD
:1041D0008093711687E005C09093701680936F16D8
:1041E00085E08093631682E88093661688E890E104
:1041F000A0E0B0E08093671690936816A0936916CC
:10420000B0936A160E9405FA8091130290911402ED
:10421000A0911502B0911602BA2FA92F982F8827C6
:104220000097E1E0AE07B10550F0B0937016A0938F
:104230006F16909372168093711687E005C0909365
:10424000701680936F1685E08093631612E81093C2
:10425000661681EA90E0A0E0B0E080936716909344
:104260006816A0936916B0936A160E9405FA8091A9
:10427000D10D882319F082E090E002C083E090E045
:104280009093701680936F1685E080936316109359
:10429000661685E490E1A0E0B0E080936716909305
:1042A0006816A0936916B0936A160E9405FA0091E9
:1042B000530810915408053611057CF410937016BC
:1042C00000936F1685E08093631682E880936616EC
:1042D00080E090E1A0E0B0E011C0C80184569109EF
:1042E0009093701680936F1685E08093631682E832
:1042F0008093661681E090E1A0E0B0E080936716BD
:1043000090936816A0936916B0936A160E9405FAF6
:104310000F5F1F4F1093540800935308093C110579
:1043200064F18BE394E00E94355581E090E0909336
:10433000A5188093A4188093700281E09AE5909369
:10434000701680936F168DE290E0909372168093B2
:10435000711687E08093631682E88093661684E87E
:1043600090E0A0E0B0E08093671690936816A09369
:104370006916B0936A160E9405FA10925A080C94B6
:104380004D3A8091C1159091C215891B8F7009F02B
:10439000DAC10E94CA518111D6C18091EB1782FD0A
:1043A000D2C17DC184E690E09093701680936F1621
:1043B00010936316009366168EE090E1A0E0B0E0E3
:1043C0008093671690936816A0936916B0936A1647
:1043D0000E9405FAC60182539048880F991F909356
:1043E000701680936F1610936316009366168FE015
:1043F00090E1A0E0B0E08093671690936816A093D8
:104400006916B0936A160E9405FA0F941C1A90E080
:104410009093701680936F1685E08093631682E800
:104420008093661686E190E1A0E0B0E08093671685
:1044300090936816A0936916B0936A160E9405FAC5
:1044400020E030E048EC52E46091AA0D7091AB0D91
:104450008091AC0D9091AD0D0F947E300F947A3811
:104460007093701660936F1615E01093631602E850
:104470000093661686E290E1A0E0B0E080936716B4
:1044800090936816A0936916B0936A160E9405FA75
:1044900020E030E0A9016091630970916409809186
:1044A0006509909166090F940E370F947A387093CE
:1044B000701660936F16109363160093661686E36A
:1044C00090E1A0E0B0E08093671690936816A09307
:1044D0006916B0936A160E9405FA60917A09709184
:1044E0007B0980917C0990917D090F947A387093B3
:1044F000701660936F1610936316009366168CE324
:1045000090E1A0E0B0E08093671690936816A093C6
:104510006916B0936A160E9405FA80916709909116
:1045200068099093701680936F161093631600932A
:10453000661684E390E1A0E0B0E080936716909364
:104540006816A0936916B0936A160E9405FA8091C6
:104550007E0990917F099093701680936F16109347
:104560006316009366168AE390E1A0E0B0E08093C2
:10457000671690936816A0936916B0936A160E9406
:1045800005FA00914F0801117FC1809151088111F6
:104590007BC18091560881113CC280911716909181
:1045A0001816A0911916B0911A168C34F0E19F07D5
:1045B000A105B10509F052C283EBC82E86E1D82EC1
:1045C0000AE18DE394E10E940E73E0904408F090BC
:1045D0004508181619060CF09DC31AE1E116F104FE
:1045E00014F40C94403696C3109257087ACC85E0A8
:1045F00096E00E9435558091550890E0A0E0B0E02B
:10460000895B9F4FAE4FB54A21E03AE53093701673
:1046100020936F16909372168093711687E08093A3
:10462000631682E88093661684E890E0A0E0B0E02C
:104630008093671690936816A0936916B0936A16D4
:104640000E9405FA10925608FFCC81E08093700218
:104650001092A81883E196E00E94355581E09AE512
:104660009093701680936F168EE490E0909372167C
:104670008093711687E08093631682E880936616B4
:1046800084E890E0A0E0B0E080936716909368160D
:10469000A0936916B0936A160E9405FAD7CC0091D0
:1046A0007A0910917B0920917C0930917D0908A33A
:1046B00019A32AA33BA360917E0970917F09072E5D
:1046C000000C880B990B0F941F306B017C0120E0CC
:1046D00030E040E050E40F940D3728A139A14AA101
:1046E0005BA10F946E3918160CF433C220E030E051
:1046F000A9016091630970916409809165099091A5
:1047000066090F940E376CA37DA38EA39FA36091BF
:10471000670970916809072E000C880B990B0F949C
:104720001F304B015C0120E030E040E251E40F9487
:104730000D372CA13DA14EA15FA10F946E39181623
:104740000CF407C226C28CE090E090937016809320
:104750006F1605E00093631682E88093661684E185
:1047600090E1A0E0B0E08093671690936816A09364
:104770006916B0936A160E9405FA0F94491820E151
:104780003EE040E050E00F946E362115310511E017
:104790004107510560F05093701640936F163093A7
:1047A00072162093711687E08093631606C03093CB
:1047B000701620936F160093631602E80093661636
:1047C00080E190E1A0E0B0E08093671690936816D6
:1047D000A0936916B0936A160E9405FA0F944918BF
:1047E00020E13EE040E050E00F946E362CE330E0F4
:1047F00040E050E00F946E363093701620936F16A1
:1048000015E0109363160093661682E190E1A0E034
:10481000B0E08093671690936816A0936916B093E2
:104820006A160E9405FA0F941C1A882391F00F94BF
:104830001C1A8F5F80935208C82ED12C833308F046
:10484000B1CDC601880F991F9093701680936F1693
:1048500004C01092701610926F1610936316009396
:1048600066168EE090E1A0E0B0E08093671690932A
:104870006816A0936916B0936A160E9405FA109202
:10488000701610926F16AFCD20E030E0A901609154
:1048900063097091640980916509909166090F948C
:1048A0000E3720E030E048EC52E40F947E306B018C
:1048B0007C016091670970916809072E000C880BD4
:1048C000990B0F941F309B01AC01C701B6010F94E7
:1048D00008380F9481386436710510F064E670E092
:1048E0007093701660936F1695E0A92EA0926316D0
:1048F00022E8B22EB092661684E290E1A0E0B0E029
:104900008093671690936816A0936916B0936A1601
:104910000E9405FA20E030E0A901609163097091DE
:10492000640980916509909166090F940E376B01B7
:104930007C0120E030E04AE253E40F946E3918160F
:104940000CF069C1002309F466C110924F0820E001
:1049500030E040E251E4609147087091480880914E
:10496000490890914A080F947E300F947A387093DA
:10497000701660936F16A0926316B092661684E567
:1049800090E1A0E0B0E08093671690936816A09342
:104990006916B0936A160E9405FA20E030E040E202
:1049A00051E460914B0870914C0880914D089091B2
:1049B0004E080F947E300F947A387093701660937F
:1049C0006F16A0926316B092661688E590E1A0E09B
:1049D000B0E08093671690936816A0936916B09321
:1049E0006A160E9405FA81E296E00E94355581E040
:1049F0009AE59093701680936F1681E490E09093FF
:104A000072168093711687E080936316B0926616D3
:104A100051C18091460801E0080F0093460890E0DC
:104A20009093701680936F1685E08093631682E8EA
:104A30008093661682E490E1A0E0B0E08093671670
:104A400090936816A0936916B0936A160E9405FAAF
:104A50000A3008F4A2CD109246089FCD8A349041C6
:104A6000A105B10509F4A8CD20E030E040E251E411
:104A70006091B90D7091BA0D8091BB0D9091BC0DF4
:104A80000F947E300F947A387093701660936F167F
:104A900015E01093631602E80093661688E490E12F
:104AA000A0E0B0E08093671690936816A093691613
:104AB000B0936A160E9405FA20E030E040E251E42B
:104AC0006091BD0D7091BE0D8091BF0D9091C00D94
:104AD0000F947E300F947A387093701660936F162F
:104AE00010936316009366168AE490E1A0E0B0E0AC
:104AF0008093671690936816A0936916B0936A1610
:104B00000E9405FA20E030E040E251E46091C10DDE
:104B10007091C20D8091C30D9091C40D0F947E30A1
:104B20000F947A387093701660936F161093631613
:104B3000009366168CE490E1A0E0B0E080936716E5
:104B400090936816A0936916B0936A160E9405FAAE
:104B500033CD8DE090E09093701680936F1685E0D2
:104B60008093631682E88093661684E190E1A0E06A
:104B7000B0E08093671690936816A0936916B0937F
:104B80006A160E9405FA8091A718811141C081E040
:104B90003FC020E030E040E050E4C701B6010F9490
:104BA0000E3728A139A14AA15BA10F94183087FDC7
:104BB00010C020E030E040E251E4C501B4010F94A0
:104BC0000E372CA13DA14EA15FA10F94183087FF95
:104BD00037CC84E190E09093701680936F1685E057
:104BE0008093631682E88093661684E190E1A0E0EA
:104BF000B0E08093671690936816A0936916B093FF
:104C00006A160E9405FA8091A718811101C082E0FE
:104C10008093A71815CC6091670970916809072ED9
:104C2000000C880B990B0F941F309B01AC01C7013E
:104C3000B6010F946E396091510887FD4AC0662312
:104C400009F4A7CC062E000C770B8EE297E00F94A8
:104C50002C1710925108109254081092530884E0B7
:104C600090E09093701680936F1685E080936316A2
:104C700002E8009366168EE890E1A0E0B0E0809331
:104C8000671690936816A0936916B0936A160E94EF
:104C900005FA81E09AE59093701680936F1683E58C
:104CA00090E0909372168093711687E0809363165C
:104CB0000093661684E890E0A0E0B0E08093671669
:104CC00090936816A0936916B0936A160E9405FA2D
:104CD00060CC662309F45DCC809153089091540810
:104CE0009C012F5F3F4F309354082093530865E099
:104CF00070E00F94F1369093701680936F1685E0F4
:104D00008093631682E8809366168EE890E1A0E0B7
:104D1000B0E0D4CF1E141F040CF02FCB90911416CA
:104D20008091B316981322C0909115168091B416F5
:104D300098131CC003E0E016F104C4F09091B5167E
:104D4000909313168091B616809316169330D1F473
:104D5000982F9D7F9038B1F49091B7169F3409F049
:104D60005FC09091B8169B3409F05AC08AE1E3EB1A
:104D7000F6E1DF011D928A95E9F71092450810923D
:104D80004408FBCA833809F04BC08091B716909154
:104D9000B816982789279827A0E0B0E080931716C7
:104DA00090931816A0931916B0931A164091B9163D
:104DB00050E060E070E040931B1650931C16609327
:104DC0001D1670931E160AEBA02E06E1B02E80E091
:104DD00090E0DC0184179507A607B70708F04EC0DE
:104DE0006C017D01F694E794D794C79496012A5FED
:104DF0003F4F220F331FF901ED5EF94E7F01F501A0
:104E0000208130E0322F22270181202BF7013183CE
:104E100020830296A11DB11DF2E0AF0EB11CDACFC6
:104E2000813861F58091B71690E0A0E0B0E0809302
:104E3000171690931816A0931916B0931A1680910E
:104E4000B816482F50E060E070E040931B16509376
:104E50001C1660931D1670931E16A9EBB6E1EFE1C8
:104E6000F6E190E020E030E02817390739F04D9165
:104E700050E0419351932F5F3F4FF6CF8AE1E3EB30
:104E8000F6E1DF011D928A95E9F71092450810922C
:104E900044088CE494E00E9435556091A8181616D9
:104EA00064F4062E000C770B83E297E00F942C1726
:104EB0008AE00E942A540C94313660911F1670913A
:104EC000201681E197E00F940E178AE00E942A5481
:104ED00040911716509118166091191670911A1674
:104EE00082E097E00F94FD168AE00E942A54809198
:104EF000171690911816A0911916B0911A16EFE78F
:104F0000F2E000E010E04191519161917191411501
:104F1000510561057105D1F1481759076A077B07EB
:104F200091F5AC01BD01485050416109710945300E
:104F300051056105710568F1AC01BD01477F423340
:104F400050416105710541F18433F0E19F07A105EE
:104F5000B10511F1AC01BD0146545041610971091F
:104F60004730510561057105D0F0AC01BD014455D4
:104F7000504161097109453051056105710588F499
:104F800002E110E00EC00F5F1F4FBDCF0FEF1FEF0C
:104F900008C003E010E005C008E010E002C00FE028
:104FA00010E08A509042A109B109833D9105A10505
:104FB000B10530F00F3F2FEF120721F40C9431367A
:104FC00009E110E0ADE6CA2EA4E0DA2EF6018191E7
:104FD0006F01882319F00E942A54F8CFB801012EDE
:104FE000000C880B990B0E949E540E942F5586EF4F
:104FF00096E00E9435550A31110510F00C942D36BB
:10500000F8018827E758FF4F8F4F0D94053780919F
:105010001F169091201681309105E1F410927002D4
:105020008FEF8093301060E080E00E941CDA0BE785
:1050300014E0D8018D918D01882319F00E942A5423
:10504000F8CF81E09AE59093701680936F168EE208
:1050500090E0AFC08230910509F0B7C081E0809345
:1050600070020F948D1A82EF96E09093B3098093AB
:10507000B2098BE090E09093701680936F1605E074
:105080000093631612E81093661680E092E1A0E0A8
:10509000B0E08093671690936816A0936916B0935A
:1050A0006A160E9405FA1092701610926F160093FD
:1050B0006316109366168EE090E1A0E0B0E0809356
:1050C000671690936816A0936916B0936A160E94AB
:1050D00005FA1092701610926F16009363161093D3
:1050E00066168FE090E1A0E0B0E0809367169093A1
:1050F0006816A0936916B0936A160E9405FA10927A
:10510000701610926F16009363161093661686E160
:1051100090E1A0E0B0E08093671690936816A093AA
:105120006916B0936A160E9405FA62E070E080E0AA
:1051300090E00E94A3A21092701610926F16009336
:1051400063161093661680E190E1A0E0B0E08093D2
:10515000671690936816A0936916B0936A160E941A
:1051600005FA1092701610926F1600936316109342
:10517000661682E190E1A0E0B0E08093671690931C
:105180006816A0936916B0936A160E9405FA05EA9C
:1051900014E0F80181918F01882319F00E942A54AC
:1051A000F8CF81E09AE59093701680936F168DE2A8
:1051B00090E0909372168093711687E08093631647
:1051C00082E8809366160C9476378330910549F512
:1051D00081E0809370020FEC14E0D8018D918D0175
:1051E0008823C9F00E942A54F8CF80911716909115
:1051F0001816A0911916B0911A16823330E1930750
:10520000A105B10509F07AC480911F16909120166E
:10521000009709F036C480911202882309F406C36E
:1052200016C3049711F00C943136109270020C944E
:10523000313680911F169091201681309105D9F456
:105240001092700280911202882319F082E090E09F
:1052500002C083E090E09093701680936F1685E013
:105260008093631682E8809366168EE190E1A0E059
:10527000B0E00C947A378230910519F509EF14E00B
:10528000F80181918F01882319F00E942A54F8CFE8
:1052900081E0809370028091A718843049F081E00A
:1052A0009AE59093701680936F1685E390E081CF16
:1052B00081E09AE59093701680936F1686E390E0F4
:1052C00078CF8330910509F04CC02091120222233F
:1052D00019F19093701680936F1685E08093631692
:1052E00082E8809366168EE190E1A0E0B0E08093C2
:1052F000671690936816A0936916B0936A160E9479
:1053000005FA40E060E070E088EC92E40F94FC1A4B
:10531000109212020C94313682E090E09093701655
:1053200080936F1685E08093631682E880936616FB
:105330008EE190E1A0E0B0E080936716909368164C
:10534000A0936916B0936A160E9405FA40E060E0E7
:1053500070E0CB010F94FC1A81E0809312020C9450
:105360003136049711F00C94313680918D098823E1
:10537000F1F082E090E09093701680936F1685E0D4
:105380008093631682E8809366168FE190E1A0E037
:10539000B0E08093671690936816A0936916B09357
:1053A0006A160E9405FA10928D090C94313683E03A
:1053B00090E09093701680936F1685E0809363164B
:1053C00082E8809366168FE190E1A0E0B0E08093E0
:1053D000671690936816A0936916B0936A160E9498
:1053E00005FA81E080938D090C94313600911F16E7
:1053F00010912016B80180E090E00F941D306B01F1
:105400007C0120E030E040E251E40F94183087FD49
:105410000DC020E030E04AEF53E4C701B6010F941D
:105420006E39181634F0902F812F05C09AE080E075
:1054300002C094EF81E090935102809352020C9449
:1054400031368091171690911816A0911916B091C7
:105450001A168830F0E19F07A105B10509F050C088
:1054600081E09AE59093701680936F168DE290E03C
:10547000909372168093711687E08093631612E8FA
:105480001093661684E890E0A0E0B0E08093671681
:1054900090936816A0936916B0936A160E9405FA55
:1054A0001092701610926F1605E000936316109319
:1054B000661680E190E1A0E0B0E0809367169093DB
:1054C0006816A0936916B0936A160E9405FA1092A6
:1054D000701610926F16009363161093661682E191
:1054E00090E1A0E0B0E08093671690936816A093D7
:1054F0006916B0936A160E9405FA0F948D1A8FC030
:105500008A3000E19007A105B105E1F580911F16F1
:1055100090912016813F910511F00C94313681E075
:105520009AE59093701680936F1686E390E09093BF
:1055300072168093711687E08093631682E88093D9
:10554000661684E890E0A0E0B0E080936716909340
:105550006816A0936916B0936A160E9405FA41E78F
:1055600055E068E775E084E00E941ECE60E080EFC1
:105570009CE30F944E1A87E695E09093B3098093CD
:10558000B2094DC08C309041A105B10509F047C06A
:1055900080911F1690912016019709F040C00F943A
:1055A000D42A1092A71881E0809370028CE090E0DA
:1055B0009093701680936F1685E08093631612E8BF
:1055C0001093661684E190E1A0E0B0E08093671646
:1055D00090936816A0936916B0936A160E9405FA14
:1055E00081E09AE59093701680936F1685E390E0C2
:1055F000909372168093711687E0809363161093D0
:10560000661684E890E0A0E0B0E08093671690937F
:105610006816A0936916B0936A160E9405FA8091E5
:10562000171690911816A0911916B0911A168C3071
:105630009041A105B10511F00C94313680911F16EF
:1056400090912016029711F00C9431360F94D42AC1
:1056500081E0809351081092A718809370021092F5
:1056600054081092530881E09AE590937016809345
:105670006F1682E590E09DCD20911F163091201687
:10568000B90180E090E037FF09C00F941D3020E0A1
:1056900030E040E857E40F940D3702C00F941D30FE
:1056A00020E030E048EC52E40F9408386B017C01B4
:1056B00020E030E040EA51EC0F946E3987FD31C0B4
:1056C00020E030E040EA51E4C701B6010F94183001
:1056D00018163CF1A70196016091AA0D7091AB0DCF
:1056E0008091AC0D9091AD0D0F940D3720E030E01E
:1056F00048EC53E40F947E3090580F947A38CB01E5
:105700000E947DFDC092AA0DD092AB0DE092AC0D2F
:10571000F092AD0D8DEE96E09093B3098093B209AF
:1057200028C020E030E048EC52E46091AA0D70916E
:10573000AB0D8091AC0D9091AD0D0F947E300F9418
:105740007A387093701660936F1685E080936316B5
:1057500082E88093661686E290E1A0E0B0E0809354
:10576000671690936816A0936916B0936A160E9404
:1057700005FA6091AA0D7091AB0D8091AC0D9091DE
:10578000AD0D8E010B5E1F4F23E041E00F94F02A18
:105790009F938F938FED96E09F938F930451110900
:1057A0001F930F930F94B02FC8010E947DA30F90F9
:1057B0000F900F900F900F900F900C9431368091B6
:1057C0001F1690912016009729F481E080937002B3
:1057D0000C94313681309105B1F480911202882306
:1057E00049F081E09AE59093701680936F168CE3F0
:1057F00090E0DFCC81E09AE59093701680936F166D
:105800008BE390E0D6CC82309105F9F2833091059C
:1058100039F58091120240E0882389F060E070E061
:1058200088EC92E40F94FC1A1092120281E09AE53F
:105830009093701680936F1689E390E0BACC60E085
:1058400070E0CB010F94FC1A81E08093120281E09A
:105850009AE59093701680936F168AE390E0A9CC36
:105860008530910599F50F94371B84EB90E00E94E9
:10587000A4A11092440B1092450B1092460B10926B
:10588000470B1092480B0E94C97186E490E00E9479
:10589000C97D84EB90E09093701680936F1605E0BD
:1058A0000093631612E81093661684E390E1A0E07B
:1058B000B0E08093671690936816A0936916B09332
:1058C0006A160E9405FA86E490E035C0863091059C
:1058D000D9F50F94371B80EF90E00E94A4A110929D
:1058E000440B1092450B1092460B1092470B1092EE
:1058F000480B0E94C9718EE690E00E94C97D80EF3E
:1059000090E09093701680936F1605E000936316F5
:1059100012E81093661684E390E1A0E0B0E0809373
:10592000671690936816A0936916B0936A160E9442
:1059300005FA8EE690E09093701680936F160093B0
:10594000631610936616D4C0813F910511F00C9434
:10595000313640E060E070E0CB010F94FC1A41E08A
:1059600060E070E0CB010F94FC1A109212020F94C9
:10597000371B80E090E00E94A4A11092440B10928B
:10598000450B1092460B1092470B1092480B0E9449
:10599000C97180E090E00E94C97D1092701610924B
:1059A0006F1605E00093631612E81093661684E301
:1059B00090E1A0E0B0E08093671690936816A09302
:1059C0006916B0936A160E9405FA61E070E080E003
:1059D00090E00E94A3A21092701610926F1600938E
:1059E0006316109366168AE390E1A0E0B0E080931E
:1059F000671690936816A0936916B0936A160E9472
:105A000005FA61E070E080E090E00E94A3A284E1EA
:105A100090E09093701680936F1600936316109326
:105A2000661684E190E1A0E0B0E080936716909361
:105A30006816A0936916B0936A160E9405FA81E071
:105A40009AE59093701680936F1689E390E0909397
:105A500072168093711687E0809363161093661612
:105A600084E890E0A0E0B0E0809367169093681619
:105A7000A0936916B0936A160E9405FA82E00C940E
:105A80002A3681309105B1F40F94371B80E090E005
:105A90000E94A4A11092701610926F1685E0809358
:105AA000631682E88093661684E390E1A0E0B0E09C
:105AB0000C947A37029711F00C9431361092440B03
:105AC0001092450B1092460B1092470B1092480B08
:105AD0000E94C97180E090E00E94C97D109270160A
:105AE00010926F1685E08093631682E880936616A5
:105AF0008AE390E1A0E0B0E00C947A378433E0E1EF
:105B00009E07A105B105D9F400911F16109120162A
:105B10000F94371BB80180E090E00F941D3020E017
:105B200030E046E953E40F946E39181614F0C801BA
:105B300002C08CE291E00E94A4A10C9431368A3319
:105B40009041A105B10511F00C94313600911F165A
:105B5000109120161092440B1092450B1092460B98
:105B60001092470B1092480B0E94C971B80180E057
:105B700090E00F941D3020E030E04CE053E40F94AF
:105B80006E39181614F0C80102C08CE890E00E942B
:105B9000C97D0C94313680911F1690912016009784
:105BA00009F413CE8130910509F04CC08091D10DDC
:105BB000882319F083E090E002C082E090E09093A7
:105BC000701680936F1685E08093631682E8809349
:105BD000661685E490E1A0E0B0E0809367169093AC
:105BE0006816A0936916B0936A160E9405FA8AE0B7
:105BF00090E09093701680936F1685E08093631603
:105C000082E88093661680E092E1A0E0B0E08093A5
:105C1000671690936816A0936916B0936A160E944F
:105C200005FA0E94C1A1811103C08FEC96E002C069
:105C300083EC96E09093B3098093B20982E080935D
:105C4000A81886C18230910509F0ADC081E080932B
:105C5000700288E0E7E4F8E0DF011D928A95E9F739
:105C600080E090E0A0E2B1E4809347089093480878
:105C7000A0934908B0934A0880934B0890934C082E
:105C8000A0934D08B0934E0884E690E09093701670
:105C900080936F1605E00093631612E81093661662
:105CA00084E590E1A0E0B0E08093671690936816D9
:105CB000A0936916B0936A160E9405FA20E030E0BE
:105CC00040E251E460914B0870914C0880914D087E
:105CD00090914E080F947E300F947A38709370161E
:105CE00060936F16009363161093661688E590E133
:105CF000A0E0B0E08093671690936816A0936916B1
:105D0000B0936A160E9405FA20E030E0A901609184
:105D100063097091640980916509909166090F94F7
:105D20000E370F947A387093701660936F16009345
:105D300063161093661686E390E1A0E0B0E08093CE
:105D4000671690936816A0936916B0936A160E941E
:105D500005FA809167099091680990937016809375
:105D60006F16009363161093661684E390E1A0E02B
:105D7000B0E08093671690936816A0936916B0936D
:105D80006A160E9405FA62E070E080E090E00E94EE
:105D9000A3A281E09AE59093701680936F1681E438
:105DA00090E00C946D378330910509F086C0109215
:105DB000550820E030E040E251E46091B90D709167
:105DC000BA0D8091BB0D9091BC0D0F947E300F9455
:105DD0007A387093701660936F1605E0009363161F
:105DE00012E81093661688E490E1A0E0B0E080939A
:105DF000671690936816A0936916B0936A160E946E
:105E000005FA20E030E040E251E46091BD0D709170
:105E1000BE0D8091BF0D9091C00D0F947E300F94F8
:105E20007A387093701660936F1600936316109310
:105E300066168AE490E1A0E0B0E080936716909344
:105E40006816A0936916B0936A160E9405FA20E0BE
:105E500030E040E251E46091C10D7091C20D80913B
:105E6000C30D9091C40D0F947E300F947A387093C7
:105E7000701660936F1600936316109366168CE489
:105E800090E1A0E0B0E08093671690936816A0932D
:105E90006916B0936A160E9405FA62E070E080E02D
:105EA00090E00E94A3A281E09AE5909370168093FF
:105EB0006F1687E490E00C946D378430910509F4F7
:105EC000D0C68530910549F44EE750E160E070E0BE
:105ED00080E295E00E94C3FAC4C6069709F0C1C6E5
:105EE0008FEB96E09093B3098093B2098BE090E03A
:105EF0002BC280911F1690912016019711F51092D8
:105F0000700281E09AE59093701680936F168FE38C
:105F100090E0909372168093711687E080936316D9
:105F200082E88093661684E890E0A0E0B0E0809379
:105F3000671690936816A0936916B0936A160E942C
:105F400005FA80911F1690912016029709F089C6D4
:105F500081E09AE59093701680936F1680E490E04C
:105F600028C9E0911F16F09120163197EB30F1050A
:105F700008F0E4C18827ED56FF4F8F4F0D94053789
:105F80008091FA1380FFA7C6869580FDA7C6A3C699
:105F90002DEC3CEC4CEC5DE36091AA0D7091AB0DE7
:105FA0008091AC0D9091AD0D0F940E376B017C017B
:105FB00020E030E040EA51EC0F946E3987FDC2C119
:105FC00020E030E040EA51E4C701B6010F941830F8
:105FD00018160CF08AC6B6C12DEC3CEC4CEC5DE317
:105FE0006091AA0D7091AB0D8091AC0D9091AD0DAB
:105FF0000F940D376B017C0120E030E040EA51EC5A
:106000000F946E3987FD9EC120E030E040EA51E4F4
:10601000C701B6010F94183018160CF0DDC692C1F6
:1060200080E00E9447D20E94C1A1811103C086E690
:1060300096E002C088E596E09093B3098093B20998
:1060400082E08093A81881E09AE59093701680937F
:106050006F1684E590E0909372168093711687E036
:106060008093631682E88093661684E890E0A0E04F
:10607000B0E08093671690936816A0936916B0936A
:106080006A160E9405FA5EC183E08093A81883E037
:1060900090E09093701680936F1685E0809363165E
:1060A00082E8809366168DE890E1A0E0B0E08093EE
:1060B000671690936816A0936916B0936A160E94AB
:1060C00005FAE12CF12C00E0DD24D394AA24A3945A
:1060D00075E0972EE5E08E2EF2E87F2EDD2031F080
:1060E000CC24C39465E0B62E10E005C0CC24CA943D
:1060F000BB24BA9414E0DA24B116D1F1802F90E0D9
:106100004897A4F50F5FF701919EE00DF11D112452
:10611000EE0FFF1FEE0FFF1FE459FC4E20E030E0B2
:106120004AE754E460817181828193810F947E30CB
:106130000F947A387093701660936F16809263167E
:1061400070926616802F90E08158974F880F991FA4
:10615000092E000CAA0BBB0B809367169093681650
:10616000A0936916B0936A160E9405FA1C0DC4CF5D
:10617000BFEFEB1AFB0AE5E0EE16F10409F0AECF33
:1061800081E09AE59093701680936F1685E590E014
:10619000909372168093711687E08093631682E85D
:1061A0008093661684E890E0A0E0B0E080936716E4
:1061B00090936816A0936916B0936A160E9405FA28
:1061C0008AEF95E09093B3098093B209BBC042E097
:1061D00060E070E080E890E40E94DFA140E060E0D1
:1061E00070E08DE193E40E94DFA141E060E070E0A7
:1061F0008AE193E413C042E060E070E080E890E45C
:106200000E94DFA140E060E070E080EB91E40E943A
:10621000DFA141E060E070E080EB91E40E94DFA14B
:1062200086E08093A8188EC042E060E070E080E8CD
:1062300090E40E94DFA140E060E070E882E993E42E
:10624000E6CF42E060E070E080E890E40E94DFA1E9
:1062500040E060E070E882E993E40CC042E060E076
:1062600070E080E890E40E94DFA140E060E070E030
:1062700080EB91E40E94DFA141E060E070E08FE8F4
:1062800093E4CCCF8091D10D81111CC083E090E0CC
:106290009093701680936F1685E08093631682E862
:1062A0008093661685E490E1A0E0B0E080936716E5
:1062B00090936816A0936916B0936A160E9405FA27
:1062C00081E01BC082E090E09093701680936F167F
:1062D00085E08093631682E88093661685E490E1FA
:1062E000A0E0B0E08093671690936816A0936916BB
:1062F000B0936A160E9405FA80E00E9447D220E01F
:1063000030E048EC52E46091AA0D7091AB0D8091A1
:10631000AC0D9091AD0D0F947E300F947A38709340
:10632000701660936F1685E08093631682E8809301
:10633000661686E290E1A0E0B0E09BCE8EED95E09F
:106340000E9435558AE090E09093701680936F1606
:1063500085E08093631682E8809366164FC184E0DF
:106360008093A8188091171690911816A09119166D
:10637000B0911A1660911F16709120168834F0E1C2
:106380009F07A105B10509F453C08A3400E19007C5
:10639000A105B10509F455C08C3410E19107A105A0
:1063A000B10509F457C086349041A105B10509F043
:1063B00059C063307105B9F58DEC95E09093B30940
:1063C0008093B20981E08093560880937002109206
:1063D000460881E09AE59093701680936F168AE4E0
:1063E00090E0909372168093711687E08093631605
:1063F00012E81093661684E890E0A0E0B0E0809385
:10640000671690936816A0936916B0936A160E9457
:1064100005FA8AE090E09093701680936F1685E0FD
:1064200080936316E9C0609355081092A81819C4A8
:10643000412C30E8532E3DE9632E33E4732E312C8A
:1064400011C0412C512C2AE9622E23E4722E3324F0
:10645000339408C0412C512C88EC682E83E4782EAC
:1064600092E0392E80E090E00F941D3020E030E083
:1064700040E251E40F9408386B017C0120E030E0E9
:10648000A9010F94183087FF09C01092400810929C
:106490004108109242081092430819C0A3019201CA
:1064A000C701B6010F946E3918164CF0C09240081F
:1064B000D0924108E0924208F092430808C040920E
:1064C00040085092410860924208709243086091DF
:1064D0004008709141088091420890914308432DF3
:1064E0000E94DFA161E070E080E090E00E94A3A242
:1064F00020E030E040E251E46091B90D7091BA0DB6
:106500008091BB0D9091BC0D0F947E300F947A3822
:106510007093701660936F1605E00093631612E88F
:106520001093661688E490E1A0E0B0E080936716CF
:1065300090936816A0936916B0936A160E9405FAA4
:1065400020E030E040E251E46091BD0D7091BE0D5D
:106550008091BF0D9091C00D0F947E300F947A38CA
:106560007093701660936F160093631610936616FF
:106570008AE490E1A0E0B0E08093671690936816FB
:10658000A0936916B0936A160E9405FA20E030E0E5
:1065900040E251E46091C10D7091C20D8091C30D34
:1065A0009091C40D0F947E300F947A3870937016CA
:1065B00060936F1600936316109366168CE490E157
:1065C000A0E0B0E08093671690936816A0936916D8
:1065D000B0936A160E9405FA61E070E080E090E0F6
:1065E0000E94A3A21092A8188AE090E090937016DF
:1065F00080936F16009363161093661680E092E105
:10660000A0E0B0E077C48091171690911816A09181
:106610001916B0911A16863530E19307A105B10518
:1066200009F046C020E030E0A90160916309709153
:10663000640980916509909166090F940E3720E0F6
:1066400030E04AE253E40F94183020911F16309145
:10665000201687FF5AC42530310508F056C48AEA4F
:1066600090E09093701680936F1685E08093631688
:1066700012E81093661680E290E1A0E0B0E080930B
:10668000671690936816A0936916B0936A160E94D5
:1066900005FA65E070E080E090E00E94A3A281E04E
:1066A0009AE59093701680936F1682E490E015C47B
:1066B0008435E0E19E07A105B105B9F460911F168C
:1066C0007091201680E090E00F941D3020E030E0C3
:1066D00040E251E40F9408386093470870934808EB
:1066E0008093490890934A08BCC288359041A1051F
:1066F000B10509F0B6C260911F167091201680E0B6
:1067000090E00F941D3020E030E040E251E40F941F
:10671000083860934B0870934C0880934D08909311
:106720004E089FC260911F167091201687EB95E06E
:106730000F940E1780911F169091201682309105AC
:10674000A1F038F4009771F00197E1F489E495E045
:1067500086C28430910599F058F0059799F48CE839
:1067600095E008C083E395E07AC289EA95E002C02B
:106770008FE995E09093B3098093B20972C28AE9D8
:1067800095E0F8CF8DE595E06AC28CE695E00E9431
:10679000355580911F16909120168130910509F092
:1067A00046C08AE795E00E94355581E00E941BCDE6
:1067B0008DE090E09093701680936F1685E0809343
:1067C000631612E81093661684E190E1A0E0B0E051
:1067D0008093671690936816A0936916B0936A1613
:1067E0000E9405FA83E08093A71881E09AE59093D0
:1067F000701680936F1685E390E0909372168093E5
:10680000711687E0809363161093661684E890E013
:10681000A0E0B0E08093671690936816A093691685
:10682000B0936A160E9405FA10923C081AC2892B8E
:1068300009F017C282E995E00E94355580913C0825
:10684000813039F588EA95E00E94355581E09AE576
:106850009093701680936F168EE290E0909372166C
:106860008093711687E08093631682E880936616A2
:1068700084E890E0A0E0B0E08093671690936816FB
:10688000A0936916B0936A160E9405FA1092A61892
:1068900035C0823069F48CEB95E00E94355581E07B
:1068A0009AE59093701680936F1686E390E00EC081
:1068B000833031F580ED95E00E94355581E09AE511
:1068C0009093701680936F1681E490E09093721607
:1068D0008093711687E08093631682E88093661632
:1068E00084E890E0A0E0B0E080936716909368168B
:1068F000A0936916B0936A160E9405FA1092221F9F
:1069000010923C080F948D1AACC180911F16909183
:1069100020168F3F910531F028F08FEF90E0A0E036
:10692000B0E002C0A0E0B0E08093130290931402A4
:10693000A0931502B0931602809113029091140255
:10694000A0911502B09116020097A105B10509F5B5
:106950001092701610926F1605E00093631612E8FD
:10696000109366168AE890E1A0E0B0E08093671685
:1069700090936816A0936916B0936A160E9405FA60
:1069800089E090E09093701680936F1600936316E1
:106990003DC00196A11DB11D05E0B695A79597953F
:1069A00087950A95D1F70197A109B109009701E0F0
:1069B000A007B10550F0B0937016A0936F16909396
:1069C00072168093711687E005C0909370168093BD
:1069D0006F1685E08093631612E8109366168AE8B6
:1069E00090E1A0E0B0E08093671690936816A093C2
:1069F0006916B0936A160E9405FA88E090E09093B9
:106A0000701680936F1685E0809363161093661658
:106A10008CE890E1A0E0B0E0809367169093681650
:106A2000A0936916B0936A160E9405FA809113022A
:106A300090911402A0911502B0911602BA2FA92FBD
:106A4000982F8827009711E0A107B10550F0B09367
:106A50007016A0936F16909372168093711687E04C
:106A600005C09093701680936F1685E0809363162F
:106A700082E88093661681EA90E0A0E0B0E03AC236
:106A800084EE95E00E9435550E94B5A140911716FD
:106A9000509118166091191670911A16882339F0C2
:106AA000433D20E252076105710509F496C3423D5A
:106AB00050426105710509F0D4C080911F16909174
:106AC0002016019709F0E0C40E94B5A1882309F4BB
:106AD000DBC48091301087FDC4C0A2E18A02C001EE
:106AE000112485519E4E0E94D474C12C90E2D92E5F
:106AF000E12CF12C05E012E81092701610926F163E
:106B00000093631610936616C0926716D0926816AB
:106B1000E0926916F0926A160E9405FABFEFCB1A4E
:106B2000DB0AEB0AFB0AEAE0CE16E0E2DE06E1044D
:106B3000F10411F700913010F2E10F0280011124ED
:106B40000D571F4EF80101900020E9F7C8018E1B78
:106B50009F0B439697FD01967C01F594E7941E14D4
:106B60001F040CF08BC49E012F5F3F4F690184E12D
:106B7000D9011D928A95E9F7A70165EF75E0C90172
:106B80000F94813AB801C6018E0D9F1D0F946C3A87
:106B900040E050E260E070E0C6010E94C3FA62E0AB
:106BA00070E080E090E00E94A3A240E060E070E02E
:106BB0008FE793E40F94FC1A41E060E070E08FE708
:106BC00093E40F94FC1A109212028DE090E09093DF
:106BD000701680936F1685E08093631612E8109309
:106BE000661684E190E1A0E0B0E080936716909390
:106BF0006816A0936916B0936A160E9405FA62E0BF
:106C000070E080E090E00E94A3A281E09AE590937A
:106C1000701680936F1685E390E0909372168093C0
:106C2000711687E0809363161093661684E890E0EF
:106C3000A0E0B0E08093671690936816A093691661
:106C4000B0936A160E9405FA81E0809370028093E7
:106C5000A61883E08093A71804C081E895E00E94FD
:106C6000355580E5E3E1F6E1DF011D928A95E9F70C
:106C70008AE58093141685EA809315160C94BD213D
:106C80008DE394E10E94EC72F701ED54F94E80839C
:106C90008091B3168A3581F01E141F0414F00C94F1
:106CA000E122D601E02F1D92EA95E9F710924508FE
:106CB000109244080C94E12262E070E080E090E0E1
:106CC0000E94A3A2FFEFEF1AFF0AF0924508E0929C
:106CD00044080C94E1228FEA96E002C08EE996E027
:106CE0009093B3098093B2090ACB88E290E00E94A6
:106CF0007DFD2DEC3CEC4CEC5DE36091AA0D7091B8
:106D0000AB0D8091AC0D9091AD0D0F940E376B01D2
:106D10007C0120E030E040EA51EC0F946E3987FDB1
:106D200012C020E030E040EA51E4C701B6010F9400
:106D30001830181644F0C092AA0DD092AB0DE09214
:106D4000AC0DF092AD0D20E030E048EC52E46091E3
:106D5000AA0D7091AB0D8091AC0D9091AD0D0F947B
:106D60007E300F947A387093701660936F1685E0BA
:106D70008093631682E88093661686E290E1A0E035
:106D8000B0E08093671690936816A0936916B0934D
:106D90006A160E9405FA6091AA0D7091AB0D809160
:106DA000AC0D9091AD0D8E010B5E1F4F23E041E0C5
:106DB0000F94F02A9F938F9380E996E09F938F938F
:106DC000045111091F930F930F94B02FC8010E9413
:106DD0007DA38BE896E076C088ED9FEF0E947DFD55
:106DE0002DEC3CEC4CEC5DE36091AA0D7091AB0D89
:106DF0008091AC0D9091AD0D0F940D376B017C011E
:106E000020E030E040EA51EC0F946E3987FD12C06B
:106E100020E030E040EA51E4C701B6010F94183099
:106E2000181644F0C092AA0DD092AB0DE092AC0DB2
:106E3000F092AD0D20E030E048EC52E46091AA0DF4
:106E40007091AB0D8091AC0D9091AD0D0F947E3093
:106E50000F947A387093701660936F1685E0809364
:106E6000631682E88093661686E290E1A0E0B0E0C7
:106E70008093671690936816A0936916B0936A166C
:106E80000E9405FA6091AA0D7091AB0D8091AC0D36
:106E90009091AD0D8E010B5E1F4F23E041E00F94EA
:106EA000F02A9F938F938DE796E09F938F930451E1
:106EB00011091F930F930F94B02FC8010E947DA357
:106EC00088E796E09093B3098093B2090F900F90F2
:106ED0000F900F900F900F9035CA90937216809379
:106EE000711687E0809363161093661684E890E02D
:106EF000A0E0B0E08093671690936816A09369169F
:106F0000B0936A160E9405FAACCE2430310589F49C
:106F100081E00F944F2920914B0830914C0840910B
:106F20004D0850914E080F940E3741E00F942129DF
:106F3000BBC02530310508F4FCC02630310509F40A
:106F400039C108F02BC181E080934F080F94371BA3
:106F50008EEB90E00E94A4A120E030E0A9016091B6
:106F600063097091640980916509909166090F9495
:106F70000E3720E030E048EC52E40F947E306B0195
:106F80007C016091670970916809072E000C880BDD
:106F9000990B0F941F309B01AC01C701B6010F94F0
:106FA00008380F9481386436710510F064E670E09B
:106FB0007093701660936F1605E00093631612E8E5
:106FC0001093661684E290E1A0E0B0E0809367162B
:106FD00090936816A0936916B0936A160E9405FAFA
:106FE00020E030E0A901609163097091640980910B
:106FF0006509909166090F940E370F947A38709353
:10700000701660936F16009363161093661686E3EE
:1070100090E1A0E0B0E08093671690936816A0938B
:107020006916B0936A160E9405FA809167099091DB
:1070300068099093701680936F16009363161093EF
:10704000661684E390E1A0E0B0E080936716909329
:107050006816A0936916B0936A160E9405FA65E057
:1070600070E080E090E00E94A3A281E09AE5909316
:10707000701680936F1684E490E09093721680935C
:10708000711687E0809363161093661684E890E08B
:10709000A0E0B0E08093671690936816A0936916FD
:1070A000B0936A160E9405FA20E030E040E251E415
:1070B00060914708709148088091490890914A086A
:1070C0000F947E300F947A387093701660936F1619
:1070D00005E00093631612E81093661684E590E1CC
:1070E000A0E0B0E08093671690936816A0936916AD
:1070F000B0936A160E9405FA20E030E040E251E4C5
:1071000060914B0870914C0880914D0890914E0809
:107110000F947E300F947A387093701660936F16C8
:10712000009363161093661688E590E1A0E0B0E046
:10713000E1CE2230310579F480E00F944F2920917F
:107140004708309148084091490850914A080F94E7
:107150000E3740E0EBCE2330310570F081E00F9424
:107160004F2920914B0830914C0840914D08509187
:107170004E080F940D37D9CE2130310509F094CF48
:1071800080E00F944F2920914708309148084091A2
:10719000490850914A080F940D37DBCF213F310544
:1071A00009F082CF10924F0861E070E080E090E03B
:1071B0000E94A3A281E09AE59093701680936F16C7
:1071C00081E490E0909372168093711687E080932B
:1071D000631682E88093661659CF82E496E00E9497
:1071E00035558091311090913210992720911F16BA
:1071F000309120168217930708F433CD8DEE95E079
:107200000E94355580911F16815080933010A4ED57
:107210008A2EA0E29A2EA12CB12C05E012E8109241
:10722000701610926F160093631610936616809274
:10723000671690926816A0926916B0926A160E941C
:1072400005FA3FEF831A930AA30AB30A8EED881654
:1072500080E29806A104B10411F780913010A2E1F8
:107260008A02C0011124FC01ED57FF4E7F010190FD
:107270000020E9F7C7018E1B9F0B439697FD0196EF
:107280008C011595079510161106FCF49E012F5FD1
:107290003F4F690184E1D9011D928A95E9F7A80160
:1072A00065EF75E0C9010F94813AB701C601800FFF
:1072B000911F0F946C3A44ED50E260E070E0C6011B
:1072C0000E94C3FA05E012E806C044ED50E260E017
:1072D00070E0C701F5CF1092701610926F160093F0
:1072E0006316109366168092671690926816A092A5
:1072F0006916B0926A160E9405FABFEF8B1A9B0AB4
:10730000AB0ABB0AE6EE8E16E0E29E06A104B104CB
:1073100011F78E010F5F1F4F84E1D8011D928A95EE
:10732000E9F7809132108F93809131108F93809183
:1073300020168F9380911F168F938FEF95E09F9368
:107340008F931F930F930F949B3A4EED50E260E0A2
:1073500070E0C8010E94C3FA62E070E080E090E053
:107360000E94A3A20FB6F894DEBF0FBECDBF31E2DC
:10737000C32E32E1D32EE12CF12C43E1442E40E622
:10738000542E612C712C88248394912CAA24AA94C5
:10739000BA2C75E0272EE2E83E2E0AE010E080913C
:1073A0003110909132108815990594F1B0927016B1
:1073B000A0926F162092631630926616409267165E
:1073C000509268166092691670926A160E9405FAC9
:1073D0001093701600936F16209263163092661603
:1073E000C0926716D0926816E0926916F0926A16FB
:1073F0000E9405FAFFEF8F1A9F0A20E1420E511CEE
:10740000611C711C3FEFC31AD30AE30AF30AC7CF0A
:1074100080911F169091201624E0880F991F2A95BD
:10742000E1F78D5F9F49A0E0B0E020EF37E83093AF
:10743000701620936F1605E00093631612E8109300
:1074400066168093671690936816A0936916B0939A
:107450006A160E9405FA80911F1690912016805E90
:107460009D4EA0E0B0E026E030E03093701620930F
:107470006F1600936316109366163CCD40E050E201
:1074800060E070E0C80189CB80911F1690912016B2
:10749000892B11F40C94E52BE4CBA7960FB6F89446
:1074A000DEBF0FBECDBFDF91CF911F910F91FF9037
:1074B000EF90DF90CF90BF90AF909F908F907F9094
:1074C0006F905F904F903F902F9008952F923F9232
:1074D0004F925F926F927F928F929F92AF92BF92E4
:1074E000CF92DF92EF92FF920F931F93CF93DF9390
:1074F000CDB7DEB7C154D1090FB6F894DEBF0FBEC9
:10750000CDBF22968FAF229720916B082CAF81E0E0
:1075100080936B088091ED138D3409F4BCC38435DE
:1075200011F40C945C4C873411F00C946D4C8091E8
:10753000EB139091EC138A31910509F439C1BCF435
:10754000843091053CF4823091050CF04DC097FFDA
:107550003FC09DC38C30910509F426C1853191054A
:1075600011F40C946F4C049709F091C3DEC08E3176
:10757000910509F47AC144F48C31910509F436C1BE
:107580000CF41AC114E05EC18A35910509F432C2C7
:1075900024F48A9709F4A3C27AC38B35910509F4C0
:1075A0002DC28C35910509F072C308E8202E03E046
:1075B000302E82E5E82E8DE0F82E29EB3DE03DA34C
:1075C0002CA396E9C92E9DE0D92E00E010E056C20A
:1075D00080912902882311F40C946F4C0E9446E29A
:1075E0000E947CC40C946F4C20912902222311F438
:1075F0000C946F4C11E0029709F010E00E9446E2F3
:1076000019821A821B821C821D821E821F8218868A
:1076100082E50E9485CC882309F457C00E9405CCDE
:107620006B017C0120E030E0A9010F941830882321
:1076300009F461C08091B90D9091BA0DA091BB0D74
:10764000B091BC0D88A799A7AAA7BBA78091BD0D33
:107650009091BE0DA091BF0DB091C00D8CA79DA7BC
:10766000AEA7BFA78091850D9091860DA091870D43
:10767000B091880D88AB99ABAAABBBAB8091890D5B
:1076800090918A0DA0918B0DB0918C0D8CAB9DAB20
:10769000AEABBFAB28A939A94AA95BA968A579A552
:1076A0008AA59BA50F94183081110C94934C2CA99A
:1076B0003DA94EA95FA96CA57DA58EA59FA50F9498
:1076C00018308823C1F00C94934C89E40E9485CC37
:1076D000882331F00E9405CC69837A838B839C8355
:1076E0008AE40E9485CC882331F00E9405CC6D830A
:1076F0007E838F83988720E030E0A90169817A81B9
:107700008B819C810F94183081110C94984D20E04E
:1077100030E0A9016D817E818F8198850F941830AA
:1077200081110C94984D0C94AB4D80E50E9485CC52
:10773000882329F00F9446076B017C0103C0C12CFC
:10774000D12C760183E50E9485CC882361F00E94CC
:1077500005CC20E030E04AE754E40F947E300F94EB
:1077600081386B017C010E948CFF8091FB13811199
:1077700005C060E085E897E00F944E1A0F94E21F71
:10778000C60ED71EE81EF91E0F94E21FDC01CB01C6
:107790008C199D09AE09BF09B7FD02C00C946F4C4E
:1077A00080E00E945655F0CF0E942BE50C946F4C60
:1077B0000E94FC7D0C946F4C0E94C8DE81110C94D9
:1077C0006F4C8CE0E7EEF2E0DE01119601900D9235
:1077D0008A95E1F760E070E080E50E9418E5BE015F
:1077E0006F5F7F4F0F94D1180C946F4C8091AE0D4A
:1077F0008770873011F00C94B24D60E08FE40E94E6
:10780000E77D81110C946F4C0C94B24D8091D10D99
:1078100081111DC00E9463B08823F9F0115011F44A
:107820000C948F4F43EF57E06BEF77E085E00E94B9
:1078300065CD61E086EE97E00E94BFCC8EEC97E0CC
:107840000E9472F90E94C8DE882301F306C060E03E
:107850008FE40E94E77D8823E9F20E94D7CC89E972
:1078600098E00E9472F90C946F4C2091A20D309117
:10787000A30D4091A40D5091A50D6091B90D70918B
:10788000BA0D8091BB0D9091BC0D0F940E37AB01DA
:10789000BC0188E50E94ECA369837A838B839C8377
:1078A0002091A60D3091A70D4091A80D5091A90DE2
:1078B0006091BD0D7091BE0D8091BF0D9091C00D76
:1078C0000F940E37AB01BC0189E50E94ECA36D83D8
:1078D0007E838F839887BE016B5F7F4FCE010196B9
:1078E0000F94411B882311F40C946F4C80E00E948C
:1078F00047D20E949AC761E085E40E94E77D182F75
:1079000021E0482FBE016B5F7F4FCE0101960E94A0
:107910006EDF6B017C019B01AC010F94003A811179
:107920005FC089809A80AB80BC8020E030E0A901F4
:10793000C501B4010F94183087FF05C027E137EB6C
:1079400041E558EB04C027E137EB41E558E3C501B9
:10795000B4010F940E37AB01BC018BEB98E00F9490
:107960001B178D809E80AF80B88420E030E0A90195
:10797000C501B4010F94183087FF05C027E137EB2C
:1079800041E558EB04C027E137EB41E558E3C50179
:10799000B4010F940E37AB01BC0186EB98E00F9455
:1079A0001B1720E030E0A901C701B6010F94183081
:1079B00087FF05C067E177EB81E598EB04C067E1DD
:1079C00077EB81E598E3A70196010F940E37AB01A1
:1079D000BC0181EB98E00F941B178AE00E942A54A7
:1079E0000E9481C7113011F40F94910F0E9407CBB0
:1079F0000C946F4C10926A080C946F4C8FE080933B
:107A00006A080C946F4C0E9405CC2B013C0113308A
:107A100049F0F60120813181428153810F940D3765
:107A20002B013C01ACA1BDA12D913D914D915C91EB
:107A3000C301B2010F940D374B015C012DEB37E30D
:107A400046E855EB0F946E3987FD20C02DEB37E3E8
:107A500046E855E3C501B4010F9418301816B4F088
:107A60001F5FB4E0EB0EF11CECA1FDA13496FDA369
:107A7000ECA3F4E0CF0ED11C143039F1D1018D917B
:107A80001D010E9485CC882359F3BDCF133051F4DA
:107A90004092C50D5092C60D6092C70D7092C80DF0
:107AA00001E0DECFA5019401F7016081718182813F
:107AB00093810F940E37D7016D937D938D939C9393
:107AC0001397812F0E94BFC3CBCF002321F085ECF9
:107AD0009DE00E949DFF0E9407CB0C946F4C80910B
:107AE0002902882311F40C946F4C89E40E9485CC00
:107AF000082F882321F00E9401CCE82E01C0E12C40
:107B00008AE40E9485CC182F882321F00E9401CCA2
:107B1000F82E01C0F12C002319F024E02E1528F0D6
:107B2000112349F034E03F1530F483EC98E00F94D2
:107B300067160C946F4C80E1E9EBFDE0A5E8BDE031
:107B400001900D928A95E1F70023F1F020915813EE
:107B5000309159134E2D4203B001439F700D1124F3
:107B60008091350D9091360D680F791F072E000C0E
:107B7000880B990B0F941F306093850D7093860DC1
:107B80008093870D9093880D1123F1F020915A1363
:107B900030915B134F2D4203B001439F700D1124B0
:107BA0008091370D9091380D680F791F072E000CCA
:107BB000880B990B0F941F306093890D70938A0D79
:107BC00080938B0D90938C0D60E080E50E94E77DA3
:107BD0008823C1F10023D1F02091A20D3091A30D93
:107BE0004091A40D5091A50D6091850D7091860D69
:107BF0008091870D9091880D0F940D376093850DBE
:107C00007093860D8093870D9093880D1123D1F08A
:107C10002091A60D3091A70D4091A80D5091A90D6E
:107C20006091890D70918A0D80918B0D90918C0DD2
:107C30000F940D376093890D70938A0D80938B0D8F
:107C400090938C0D40E050E0BA0186E40E94ECA3D2
:107C50006B017C0120E030E0A9010F946E39181609
:107C60004CF420E030E040E752E4C701B6010F9445
:107C7000083803C060E070E0CB0169837A838B83AE
:107C80009C83CE0101960E94B9C70C946F4C0E9450
:107C900090DE0C946F4C8091EB139091EC1386372F
:107CA000910511F40C94B8460CF027C18B34910562
:107CB00009F4C5C40CF095C08A31910509F460C37C
:107CC0009CF58431910509F4DAC27CF48131910587
:107CD00009F4C1C22CF4029708F43AC20C94594C2E
:107CE000429709F4F9C60C94594C8731910509F46F
:107CF000EBC28CF48531910509F4E2C2469711F08C
:107D00000C94594C0E94BB748091EB17877F809331
:107D1000EB170C946F4C8831910509F4EDC249972B
:107D200009F423C30C94594C8032910509F403C41F
:107D30000CF03FC08D31910509F497C394F48B3159
:107D4000910509F42BC34C9711F00C94594C40E069
:107D500060E08091320D9091330D0E9418780C9460
:107D60006F4C8E31910509F487C34F9711F00C9435
:107D7000594C0F9449186C8F7D8F8E8F9F8FBE0149
:107D80006F5F7F4FCE014C960E947CA960E0CE01D0
:107D900001960F94A91A0F945017BE016F5F7F4F81
:107DA0008EE899E00F9439178AE00E942A540C94C7
:107DB0006F4C8B32910509F42BC44CF48132910540
:107DC00009F4EFC38A9709F400C40C94594C80332A
:107DD000910509F421C48934910509F421C40C9456
:107DE000594C8936910509F46DC50CF043C08235B4
:107DF000910509F463C62CF58D34910509F427C467
:107E00000CF421C48E34910509F425C48135910503
:107E100011F00C94594C0E9418720F9445110F9454
:107E20003C010E94D8511092B40D1092B30D1092E3
:107E3000B20D68EE73E080E090E00F9438160C9479
:107E40006F4C8535910509F473C654F4833591055B
:107E500009F43BC68435910509F43EC60C94594C8F
:107E60008C35910509F47DC68836910509F485C4E1
:107E70000C94594C8F36910509F46FC524F58C3656
:107E8000910511F40C946F4CA4F48A36910509F411
:107E90002CC58B36910511F00C94594C6091B80D9E
:107EA00080E50F94841C60E070E00F94E90D0C9461
:107EB0006F4C8D36910509F498C48E36910509F4FE
:107EC0003BC50C94594C8237910509F4D4C65CF437
:107ED0008037910511F40C946F4C8137910509F4AA
:107EE00081C50C94594C8337910509F4C7C6853771
:107EF000910509F42CC70C94594C8E32A1E09A07D5
:107F000011F40C94264A0CF082C08C3C910511F4BB
:107F10000C94AF478CF58C38910509F485C59CF419
:107F20008837910509F461C70CF45CC7893791055E
:107F300009F463C78D37910511F00C94594C0E94D8
:107F400055E40C946F4C883C910509F45DC754F4DA
:107F50008B39910509F48CC58E3B910509F476C5E2
:107F60000C94594C893C910509F4B7C78B3C910599
:107F700009F4D6C70C94594C8D3D910511F40C941D
:107F8000E2472CF5833D910511F40C94CF479CF406
:107F90008D3C910509F4E6C78E3C910511F00C94D7
:107FA000594C58E8C52E53E0D52E65EAE62E69E017
:107FB000F62E10E0E2C7893D910511F40C94D247EA
:107FC0008C3D910511F40C94D5470C94594C823298
:107FD000E1E09E0711F40C941B4964F4823E910584
:107FE00011F40C9438488831914011F40C94844871
:107FF0000C94594C8C3231E0930711F40C941E49C7
:108000008D32914011F40C9433490C94594C853FB6
:10801000A1E09A0711F40C94464B0CF047C082394A
:10802000E1E09E0711F40C94704ADCF4803321E007
:10803000920711F40C94B34914F40C946A4A8039F1
:1080400041E0940711F40C946D4A8139914011F08C
:108050000C94594C81E00F94D90F0E9407CB0C94DB
:108060006F4C853AB1E09B0711F40C94784A7CF48C
:108070008A39F1E09F0711F40C946F4C843A9140D7
:1080800011F00C94594C0F94901C0C946F4C8C3A3A
:1080900031E0930711F40C94E84A843F914011F0C9
:1080A0000C94594C0E94D2BB0C946F4C8B35A2E0BF
:1080B0009A0711F40C94684B5CF5883FE1E09E0749
:1080C00011F40C944C4BACF4863F21E0920711F470
:1080D0000C94494B873F914011F00C94594C61E04E
:1080E00083E50E94E77D91E089270E9444EC0C948F
:1080F0006F4C8C3042E0940711F40C945D4B883542
:10810000924011F00C94594C0E9437E30C946F4C40
:108110008438B3E09B0711F40C94E34B6CF4833583
:10812000F3E09F0711F40C94654B8C36934011F4E7
:108130000C946F4C0C94594C803A33E0930709F43B
:1081400034C2873E934011F40C944B4C0C94594C20
:108150000091320D1091330D80E50E9485CC88236B
:1081600061F00F9446076B017C01BB24B394672B2D
:10817000682B692B31F4B12C04C0B12CC12CD12C4B
:10818000760183E50E9485CC882311F40C94A14FDD
:108190000E9405CC20E030E04AE754E40F947E30A2
:1081A0000F9481386B017C01B1100BC0672B682BD9
:1081B000692B39F40115110521F0D8018C91811139
:1081C00002C0B12C02C0BB24B3940E948CFFB1103A
:1081D00003C081E596E001C0C8010E94C2A31091CE
:1081E0006B0883E080936B0881E08093221F44EF4B
:1081F00058E06DEF78E082E00E9465CD82EE98E075
:108200000E94C2A3C114D104E104F104B1F00F949F
:10821000E21FC60ED71EE81EF91E0F94E21FDC01F6
:10822000CB018C199D09AE09BF09B7FF0EC0809123
:10823000221F81110C94A64F08C08091221F882311
:1082400021F080E00E945655F8CF1092221F109323
:108250006B080C946F4C8091EE1384FF02C00C9459
:10826000AB4F8091F01387FF02C00C94AB4F80910D
:10827000F113837011F00C94AB4F0C94C84F87E24C
:1082800099E00F94671683E395E10E94839B8BE14D
:10829000E3E3F5E1DE01119601900D928A95E1F795
:1082A00060E070E0CE0101960E94BB76CE0101969F
:1082B0000E94B99C88E199E00F9467160C946F4C6A
:1082C0000E942C750C946F4CE091320DF091330D9F
:1082D0008081882329F0803209F410823196F8CF0A
:1082E00040E061E08091320D9091330D0E9418784A
:1082F0001092231F0C946F4C8091CA0B8823E9F0D5
:1083000080E090E0A0EAB1E488A399A3AAA3BBA36C
:108310001C8E1D8E1E8E1F8E19821A821B821C823D
:1083200020E0AE01405E5F4FBE01645E7F4FCE0134
:1083300001960E9425CE0C946F4C0E94CA5188234E
:1083400021F00E94CC740F94951061E085E29DE3CA
:108350000E94BFCC48E359E060E479E085E00E94E8
:108360001ECE0F94D21A0C946F4C8091EB1782FFA3
:1083700003C08B7F8093EB170E9455E40C946F4CE5
:108380008091EB1783FD02C00C946F4C83E50E9433
:1083900085CC81110C94D74F0C946F4C83E40E94D0
:1083A0003CCC8823C1F186E599E00F946716809153
:1083B000DD14882339F1BE016F5F7F4F8AED94E1B0
:1083C0000E944A9A8E010F5F1F4FF80181918F0121
:1083D000882319F00E942A54F8CFCE0101960E94FA
:1083E000EA778091E10F882389F080E20E942A5485
:1083F00001EE1FE0D8018D918D01882339F00E9494
:108400002A54F8CF8CE499E00F9467168AE00E9412
:108410002A540C946F4C83E50E9485CC882309F183
:108420000E94EDCB182F90E0CD970CF01CE3109339
:1084300060080F94E21F6B017C01212F30E0A8EE51
:10844000B3E00F94C236C60ED71EE81EF91EC092C6
:108450005C08D0925D08E0925E08F0925F080C9490
:108460006F4C0E9494740C946F4C8091EB178E7F2C
:108470008093EB170C946F4C8091EB1783FD02C037
:108480000C946F4C0E9440E18091EB1783FD02C079
:108490000C946F4C6091320D7091330DCE014C965F
:1084A0000E947BFC8C01009711F40C946F4C6C8D36
:1084B0007D8D19821C8222E0AC01CE0101960E94C2
:1084C000B3A0811102C0F12C14C0CE0101960E940C
:1084D000E9FB8823C1F361E0CE0101960E942E9A48
:1084E000009789F325EEFC0120831C820E943D9CAD
:1084F000F82ECE0101960E94B99CB801FF2089F0A8
:1085000080E899E00F9439178AE00E942A5410926B
:10851000E7171092E8171092E9171092EA170C94D7
:108520006F4C88E699E00F94391785E699E00F942F
:1085300067160C946F4C8091EB1782FD0E948CFFA4
:108540008091EB1783FD02C00C946F4C60E080E5D6
:108550000E94E77D182F482F61E08091320D9091A5
:10856000330D0E94187883E50E9485CC882381F022
:108570000E94DDCBAB01BC014093E7175093E81795
:108580006093E9177093EA178AED94E10E94449989
:108590000E94CC7411110C946F4C0F9495100C9494
:1085A0006F4C0E945BAA0C946F4C2091320D30915D
:1085B000330D9091EB1792609093EB1740E060E0E1
:1085C000C9010E9418780C946F4C83E50E9485CCF9
:1085D000882311F40C946F4C0E94EDCBF82E6DE0C3
:1085E00070E080E50F94751C8C0197FF02C00C941D
:1085F0006F4CE82E60E089E40E94E77D81110C94C5
:10860000E84F802F0E94995181114FC50C94E84F7B
:108610000E94D5D60C946F4C0E9420AC0C946F4CE9
:1086200080E50E943CCC882311F40C946F4C80911F
:10863000EB1782FF02C00C946F4C0C9401500F9406
:1086400095100C946F4C0F9498180C946F4C0F94D9
:1086500045110C946F4C60E070E083E50F94751C3D
:108660008E34910531F40F94F7110F94D21A0C94B3
:108670006F4C89EF99E00F946716609191097091A2
:10868000920980EF99E00F940E1760919309709111
:10869000940983EE99E00F940E17609191097091FF
:1086A00092098091930990919409681B790B8091AC
:1086B000AD18815021E030E0823010F020E030E051
:1086C000621B730B88ED99E00F940E178AE00E94ED
:1086D0002A5480ED99E00F94671680919509909146
:1086E0009609A0919709B09198098C8F9D8FAE8FB4
:1086F000BF8FBE016F5F7F4FCE014C960E947CA959
:10870000BE016F5F7F4F83EC99E00F943917809122
:10871000990990919A09A0919B09B0919C098C8F1D
:108720009D8FAE8FBF8FBE016F5F7F4FCE014C9686
:108730000E947CA9BE016F5F7F4F83EB99E00F948D
:10874000391720E030E04AE754E460919D097091C8
:108750009E0980919F099091A0090F940838AB0160
:10876000BC018BE999E00F941B178DE60E942A54F7
:108770008AE00E942A540C946F4C8091A20B83FFD4
:1087800002C00C946F4C0E940DE3182F87FF02C0AB
:108790000C946F4C83E50E9485CC882311F10E94D4
:1087A00005CC0F947A387B01212F110F330BF9017F
:1087B000EE0FFF1FE556F44F718360834091B80DB3
:1087C00050E02417350711F00C946F4CCB010E9438
:1087D000A4A1F6E5EF16F10424F40F9445110F94CB
:1087E000D21A0F94A42A0C946F4C8091A20B83FF91
:1087F00002C00C946F4C0E940DE3082F87FF02C04B
:108800000C946F4C83E50E9485CCF82E811107C033
:1088100082E50E9485CC182F882309F447C00E9466
:1088200005CC0F947A38402F002E000C550BFA011E
:10883000EE0FFF1FE556F44F718360832091B80D52
:1088400030E04217530711F00C946F4CCB010E949B
:10885000A4A10E9405CC20E030E04AEA52E40F9443
:108860001830181614F40C940C500F9445110F94F2
:10887000D21A6091670970916809072E000C880B65
:10888000990B0F941F302091630930916409409136
:108890006509509166090F946E39181614F40C94FA
:1088A0001050FF2011F40C94105011E00F94A42AE2
:1088B000112311F40C946F4C6F2D802F0E94146AB9
:1088C0000C946F4C0E940DE3182F87FF02C00C948C
:1088D000764C81E09AE00F946716812F0E941E6803
:1088E0008AE00E942A540C94764C6091B80D80E581
:1088F0000F94841C182F823010F00C946F4C81E47C
:108900000E943CCC882341F0E091B80DF0E0E055A6
:10891000F24F608170E002C06FEF70E083E50E946B
:1089200018E58F3F910519F010F08FEF90E0BC0132
:10893000812F0F94E90DD3C78EE40E9485CC882344
:1089400009F4CDC70E94DDCB60932E0D70932F0DDF
:108950008093300D9093310DC2C783E50E943CCCCB
:10896000882331F060E083E50F94841C8093A20B90
:108970000F94501782E19AE00F9467168091A20B32
:10898000882369F1B8E0EB2EBAE0FB2E00E010E09E
:1089900020E08091A20B90E0A0E0B0E0002E04C0A7
:1089A000B695A795979587950A94D2F780FF0EC044
:1089B000DD24D394D20E222319F08CE20E942A5493
:1089C000F701859194910F9467162D2D0F5F1F4F1E
:1089D00032E0E30EF11C05301105D9F617CD84E025
:1089E0009AE012CD83E50E9485CC882371F00E9425
:1089F000EDCB282F30E02D3331051CF4809300029D
:108A00006EC78CE3809300026AC70F9450174091A1
:108A1000000250E060E070E089E19AE00F94FD16FA
:108A20008AE00E942A545BC78091A20B83FD57C73E
:108A300083E50E9485CC882309F451C70E9405CCA8
:108A40000F947A38CB010E94C97D49C78091A20B4F
:108A500083FD45C783E50E9485CC182F81110C94B6
:108A6000155082E50E9485CC81110C94155037C7B2
:108A700083E50E9485CC882309F431C70E94EDCBA1
:108A8000182F90E0CD970CF01CE3109365080F941D
:108A9000E21F6B017C01212F30E0A8EEB3E00F94C0
:108AA000C236C60ED71EE81EF91EC0926108D092CB
:108AB0006208E0926308F092640811C780916A0826
:108AC0008F7D806180936A080AC780916A088F7ED3
:108AD000806280936A0803C783E50E9485CC88235F
:108AE00099F00E9405CC20E030E04AE754E40F946E
:108AF0007E300F948138609301027093020280935C
:108B0000030290930402EBC68091EE1384FF02C02F
:108B10000C944A508091F01387FF02C00C944A5085
:108B20008091F113837011F00C944A500C947B5097
:108B300083E50E943CCC882309F4D1C60E9405CC71
:108B400020E030E04AE754E40F947E300F948138FF
:108B5000609366087093670880936808909369082B
:108B6000BEC60E940DE387FDBAC69091EE1394FD38
:108B700004C09091F01397FF0AC0F8E8CF2EF3E0FD
:108B8000DF2EA3E5EA2EABE0FA2E10E009C09091AB
:108B9000F113937091F7682F81E00E9459E99FC605
:108BA000D6018D916D010E9485CC882309F459C0AE
:108BB000133009F04FC00E9405CC4B015C0120E04E
:108BC00030E040EA51E40F94183087FF3AC0A50125
:108BD00094016091730B7091740B8091750B90915F
:108BE000760B0F9408382B013C019B01AC0160917E
:108BF000830B7091840B8091850B9091860B0F9461
:108C00007E306093830B7093840B8093850B9093DD
:108C1000860B6091740C7091750C8091760C90911C
:108C2000770C0F941D30A30192010F947E300F94A6
:108C300081386093740C7093750C8093760C9093CC
:108C4000770C8092730B9092740BA092750BB0927C
:108C5000760B07C00E9405CCF701648B758B868B61
:108C6000978B1F5FF4E0EF0EF11C143009F098CFE2
:108C70000E9468FF34C60E9411F831C682E69BE06C
:108C80000F94671660E082E59BE00E94F7F760E0D2
:108C90008DE39BE00E94F7F761E086E39BE00E9492
:108CA000F7F761E08BE29BE00E94F7F761E08BE170
:108CB0009BE00E94F7F760E082E19BE00E94F7F7FB
:108CC00061E088E09BE00E94F7F761E08EEF9AE0B8
:108CD0000E94F7F761E086EF9AE00E94F7F761E003
:108CE00088EE9AE00E94F7F761E08AED9AE00E9430
:108CF000F7F760E08BEC9AE00E94F7F760E08DEB0D
:108D00009AE00E94F7F760E087EA9AE00E94F7F79E
:108D100061E086E99AE00E94F7F761E087E89AE06F
:108D20000E94F7F761E082E79AE00E94F7F761E0BE
:108D30008FE59AE00E94F7F760E082E59AE00E94F2
:108D4000F7F760E08EE39AE00E94F7F7C8C58091DC
:108D5000320D9091330D009741F0DC012C912223CC
:108D600021F060E00F94A91ABAC50F94D21AB7C5C2
:108D70000091320D1091330D94E0F12C40E09150B0
:108D800021F1F8018081282F2B7F213421F42181CA
:108D90002133D9F407C08035C1F4818180538A30F2
:108DA00048F013C0813421F0853421F441E002C041
:108DB000FF24F39498012E5F3F4F89012F5F3F4FAF
:108DC000F80180818032C9F3DACF41110F94501736
:108DD000FF2021F08AE49CE00F946716C8010E94EE
:108DE00035557DC50E9419EA7AC581E08093A209B4
:108DF0008093A1090E9469EA72C51092A20910929B
:108E0000A1090E9469EA6BC50E940DE3182F87FD36
:108E100066C584E40E943CCC882309F45BC00E94B0
:108E200005CC6B017C0101E020E030E0A9010F944A
:108E30001830811101C000E00093341820E030E0C8
:108E4000A901C701B6010F941830882309F442C064
:108E50000E9405CC24E01202F0011124E35CF74EDD
:108E6000608371838283938320E030E0A901609165
:108E70003D1870913E1880913F18909140180F94C2
:108E8000183081110CC080E090E0A0EEBFE3809329
:108E90003D1890933E18A0933F18B093401820E0DF
:108EA00030E0A901609141187091421880914318F7
:108EB000909144180F94183081110CC080E090E01C
:108EC000A0EEBFE38093411890934218A0934318FB
:108ED000B09344180F948B0202C50E940DE387FDE6
:108EE000FEC4E8E8EE2EE3E0FE2E03E51BE0D7012A
:108EF0008D917D010E943CCC882359F00E9405CCC5
:108F00000F948138F80160837183828393830E9478
:108F1000F1FE0C5F1F4FFBE003361F0741F7DFC474
:108F20000E940DE387FDDBC478E8E72E73E0F72E9F
:108F300003E51BE0D7018D917D010E943CCC882385
:108F400039F00E9405CCF80164A375A386A397A30A
:108F50000C5F1F4FFBE003361F0761F7C0C40F947F
:108F6000D006BDC40F945607BAC41F5FF4E0EF0EDD
:108F7000F11C133011F40C946B3DD6018D916D01F1
:108F80000E943CCC882389F30E9405CCF7016083C2
:108F9000718382839383812F0E94BFC3E6CF0E9497
:108FA0006AE89DC40F94FA059AC483E50E9485CCB3
:108FB000882309F494C40E9401CC909352028093B8
:108FC00051028DC40E940DE3F82E87FD88C483E50D
:108FD0000E9485CC0F2D0F2C000C110B882369F1FA
:108FE0000E9401CCF801EE0FFF1FE15AFD4F918363
:108FF0008083000F111F000F111F9801285B3D4F48
:109000007901BC01990F880B990B0F941F302AE04E
:1090100037ED43E25CE30F947E30F801EB5CF74EF2
:1090200020813181428153810F947E30D7016D932D
:109030007D938D939C93139752C40F94501785E49E
:109040000E942A5480E38F0D0E942A54F801EE0FEB
:10905000FF1FE15AFD4F608171818EE49CE00F9407
:109060002C1785E20E942A548AE00E942A5437C4B1
:1090700080E50E943CCC882309F431C460E070E0B4
:1090800080E50F94751CF82E6FEF7FEF83E50F944A
:10909000751C8C010196039708F021C4F7FC1FC4CE
:1090A0008F2D0E949951882339F00F944C1786E533
:1090B0009CE00F94671613C40E948CFF60E08F2D14
:1090C0000E940AE20F3FBFEF1B0731F0013011058C
:1090D00071F000E010E00DC08F2D0E94B2E131E090
:1090E00020E0892B09F030E0032F122F02C001E0AD
:1090F00010E08F2D0E94B2E18017910709F4EFC3B1
:1091000080E00E945655F5CF80E50E943CCC882334
:1091100009F4E5C30E9401CC8C01892B09F07FC0C2
:1091200083E50E943CCC882389F00E9401CC8F3FCC
:10913000EFEF9E0729F48BEB95E10E94E251CFC33C
:10914000BC018BEB95E10E94B252C9C30F9450173A
:1091500060E070E08EE79CE00F942C178091BD15C5
:1091600028E532E06901C81AD10887FDD394CC0CF8
:10917000DD1CCC0CDD1C0D2C000CEE08FF088091D2
:10918000BC1528E830E04901881A910887FD9394BE
:10919000880C991C880C991C092C000CAA08BB0887
:1091A0008091BB158F3FC1F090E0FC01EE0FFF1FD7
:1091B0008E0F9F1FFC01E25BFA4E2181328113E08A
:1091C000220F331F1A95E1F704E0369527950A958B
:1091D000E1F72E5F3F4F02C020E030E02F5F3F4FAE
:1091E000C901330FAA0BBB0B9C01AD01281939092A
:1091F0004A095B09A4EBB0E00F94AF36A7019601D2
:10920000281939094A095B090F949036B9018BE78F
:109210009CE00F942C178AE00E942A5460C30F949C
:109220004C17B80184E79CE00F942C1785E69CE06E
:109230000F94671654C30E9487F351C364E071E032
:1092400083E50E9418E58C0168EE73E080E50E94DA
:1092500018E58938F3E19F0710F088E893E1B80139
:109260000F94EF193CC360E085E40F94841C8111D6
:1092700073C080E50E943CCC882351F00E9405CC4D
:1092800060936A0970936B0980936C0990936D09E0
:1092900089E40E943CCC882381F00E9405CC2CEA12
:1092A00035EC47E25EE30F947E3060936E09709375
:1092B0006F09809370099093710984E40E943CCCFB
:1092C000882381F00E9405CC2CEA35EC47E25EE36E
:1092D0000F9408386093720970937309809374092E
:1092E000909375090F94501740916A0950916B093A
:1092F00060916C0970916D0980EA9CE00F941B17D6
:109300002CEA35EC47E25EE360916E0970916F09DB
:1093100080917009909171090F940838AB01BC01DC
:109320008CE99CE00F941B172CEA35EC47E25EE3D6
:109330006091720970917309809174099091750917
:109340000F947E30AB01BC0188E99CE00F941B17A1
:109350008AE00E942A54C3C20F944C1786E89CE00E
:109360000F946716BCC280E50E943CCC882351F064
:109370000E9405CC609381097093820980938309D0
:109380009093840989E40E943CCC882381F00E9458
:1093900005CC2CEA35EC47E25EE30F947E30609317
:1093A000850970938609809387099093880984E4DE
:1093B0000E943CCC882381F00E9405CC2CEA35EC3D
:1093C00047E25EE30F9408386093890970938A0935
:1093D00080938B0990938C090F94501740918109C9
:1093E0005091820960918309709184098CEA9CE014
:1093F0000F941B172CEA35EC47E25EE36091850978
:109400007091860980918709909188090F94083896
:10941000AB01BC0188EA9CE00F941B172CEA35ECE9
:1094200047E25EE36091890970918A0980918B0916
:1094300090918C090F947E30AB01BC0184EA9CE0D2
:109440000F941B178AE00E942A5449C283E50E94A8
:109450003CCC182F882371F00E9405CC0F947A38E9
:10946000709343026093420221E0672B09F020E0F1
:109470002093A10B80E50E943CCC882359F02091D9
:10948000420230914302232B11F00E94D77D80933A
:10949000A10B25C2111123C20F9450178CEC9CE034
:1094A0000F9467168091A10B882319F084EB9CE040
:1094B00002C080EB9CE00F946716609142027091AD
:1094C00043028BEB9CE00F942C1787EB9CE00F94EE
:1094D000671605C20E9403A402C20E948CFFFFC14E
:1094E00080E00F94D90F0F94910F0E9407CBF7C122
:1094F0006FEF7FEF89E40F94751CF82E6FEF7FEF0D
:109500008AE40F94751CE82E8AE50E943CCC182F43
:10951000811105C081E50E943CCCB82E01C0B12C60
:10952000F7FC06C0E7FC04C0111109C0B11007C068
:109530000F944C178EEF9CE00F946716D0C124E077
:109540002F1510F02E1538F40F944C178FED9CE06A
:109550000F946716C4C1CF2C0F2C000CDD080E2D04
:109560000E2C000C110B0E9405CCBB2099F025E0BD
:109570002C9DF0012D9DF00D1124E00FF11FEE0F39
:10958000FF1FEE0FFF1FE459FC4E20813181428105
:10959000538103C020E030E0A9010F940E379B01F6
:1095A000AC0185E08C9DF0018D9DF00D1124E00F44
:1095B000F11FEE0FFF1FEE0FFF1FE459FC4E20833B
:1095C0003183428353836E2D8F2D0E94BEA287C1AB
:1095D0000E94C8DE811183C104E214E289EB9DE0A0
:1095E0009DA38CA3DE0111961D0159E7C52E54E2FF
:1095F000D52E7D01F8016591759185919491ECA12D
:10960000FDA181909190A190B190FDA3ECA3A50143
:1096100094010F940D372B013C01D7016D937D937D
:109620008D939C93139720E030E040EA51EC0F9427
:109630006E3987FD0AC020E030E040EA51E4C30102
:10964000B2010F94183018162CF4F60184911816F4
:109650000CF454C5D7018D909D90AD90BD907D01C7
:1096600020E030E040EA51ECC501B4010F946E39BE
:1096700087FD4EC520E030E040EA51E4C501B40169
:109680000F94183018160CF055C542C50E9484EF8F
:1096900026C10E9483EA23C181E0809353130E9474
:1096A000CFB510925313882309F419C10F945017A2
:1096B0008AE59DE00F94671612C18091EB1782FF37
:1096C0000EC180648093EB170AC10E94DBF007C1D2
:1096D0000E940DE3082F87FD02C185E50E943CCC66
:1096E0008823B1F1E02E002E000CFF080E9405CC6B
:1096F0004B015C0120E030E0A9010F946E3987FF37
:1097000004C0B7FAB094B7F8B094C70133E0880F3B
:10971000991F3A95E1F79C01245A3C4E7901D901F1
:109720008D929D92AD92BC92139720E030E04AEF6B
:1097300053E4C501B4010F946E3918164CF480E05F
:1097400090E0AAEFB3E4F70180839183A283B3830F
:109750008CE40E943CCC882309F4C1C0002E000C8C
:10976000110B0E9405CC6B017C0120E030E0A901C7
:109770000F946E3987FF04C0F7FAF094F7F8F0946D
:1097800023E0000F111F2A95E1F7045A1C4ED8015F
:109790001496CD92DD92ED92FC92179720E030E086
:1097A0004AEF53E4C701B6010F946E3918160CF056
:1097B00096C080E090E0AAEFB3E4F801848395833B
:1097C000A683B7838CC06091B80D70E084E50F94D8
:1097D000751C8C01823028F08EE89DE00F9467168E
:1097E0007EC08BE40E9485CC882349F10E9405CC81
:1097F0006B017C0120E030E0A9010F946E3987FDF8
:1098000019C020E030E040E251E4C701B6010F94F6
:10981000183018167CF00E948CFFF801FF27EE0F1D
:10982000FF1FEE0FFF1FE058F34FC082D182E2828C
:10983000F38255C08FE69DE00F94671650C00F94D9
:10984000501785E69DE00F94671600E81CE0C12CD8
:10985000D12C760180E20E942A54C701B6010E94F1
:109860009E548DE30E942A54D8016D917D918D9173
:109870009D918D0142E00E94BA54BFEFCB1ADB0AE2
:10988000EB0AFB0AE2E0CE16D104E104F10411F484
:109890000C940642DFCF81E08093290210923B14A2
:1098A00060E083E50E94E77D811119C00E9480ABD2
:1098B00016C00E9490DE13C01091EB138091B80D7A
:1098C000181729F060E083E50E94E77D01C081E080
:1098D000682F812F0E94956B02C00E9490DE229615
:1098E000FFAD2297F11102C00E942BAB2CAD20934B
:1098F0006B08CF5BDF4F0FB6F894DEBF0FBECDBF56
:10990000DF91CF911F910F91FF90EF90DF90CF905B
:10991000BF90AF909F908F907F906F905F904F908F
:109920003F902F90089520E030E0A901C701B601D3
:109930000F941830881F8827881F181709F4F3C060
:1099400080E090E0A0E8BFEB88AF99AFAAAFBBAFD3
:1099500028A539A54AA55BA568A979A98AA99BA9C3
:109960000F940D372B013C012CA53DA54EA55FA5FD
:109970006CA97DA98EA99FA90F940D376CA37DA317
:109980008EA39FA3A3019201C301B2010F947E3065
:109990004B015C012CA13DA14EA15FA1CA01B901FF
:1099A0000F947E309B01AC01C501B4010F940E37BA
:1099B0000F94BC394B015C0120E030E040E05FE3F4
:1099C0000F947E3021966CAF7DAF8EAF9FAF219705
:1099D000A7019601C701B6010F947E306B017C018F
:1099E00021962CAD3DAD4EAD5FAD2197CA01B901B9
:1099F0000F947E309B01AC01C701B6010F940D3767
:109A00000F94BC396B017C018CA19DA1AEA1BFA1BB
:109A1000B0588CA39DA3AEA3BFA32DEB37E346E8BC
:109A200055EBC501B4010F946E3987FD0AC02DEBCB
:109A300037E346E855E3C501B4010F941830181612
:109A40005CF4A501940160E070E080E89FE30F946E
:109A500008384B015C0103C0812C912C5401A501F5
:109A60009401C301B2010F947E3028AD39AD4AADE7
:109A70005BAD0F947E30A70196010F947E302B01D1
:109A80003C0128A939A94AA95BA968A579A58AA595
:109A90009BA50F940E3720E030E040E05FE30F9489
:109AA0007E309B01AC01C301B2010F940E3728A593
:109AB00039A54AA55BA50F940D3769837A838B83FB
:109AC0009C83A50194016CA17DA18EA19FA10F94FF
:109AD0007E3028AD39AD4AAD5BAD0F947E30A70125
:109AE00096010F947E306B017C012CA93DA94EA9F3
:109AF0005FA96CA57DA58EA59FA50F940E3720E0CC
:109B000030E040E05FE30F947E309B01AC01C70181
:109B1000B6010F940E372CA53DA54EA55FA50F9459
:109B20000D370C94773B80E090E0A0E8BFE30CCFCA
:109B3000412FBE016F5F7F4F85E89DE00E942DF4AD
:109B40000F94E21F6093F2137093F3138093F41356
:109B50009093F513C4CE0F944C178FE697E00F94B3
:109B60006716BDCE0E948CFF9091D10D9CAB80E01A
:109B70000E9447D20E949AC781E08093A2090E9466
:109B800069EA88E50E943CCC182F89E50E943CCC0C
:109B9000082F8AE50E943CCC1013BFC1181711F0A2
:109BA000012FBBC101E011E091E09CA780E1E9EB4E
:109BB000FDE0A5E8BDE001900D928A95E1F782E510
:109BC0000E9485CC882361F00E9405CC6B017C014A
:109BD00020E030E0A9010F941830882369F106C015
:109BE000C12CD12C20E8E22E20E4F22E111103C06A
:109BF000002309F4FCC0C0928D0DD0928E0DE0922E
:109C00008F0DF092900DA70196016091C10D70919A
:109C1000C20D8091C30D9091C40D0F94183087FF31
:109C20000BC019821A821B821C82BE016F5F7F4F9C
:109C30008DE89DE00E9426C9112309F4D3C00023BA
:109C400009F4CDC01092B90D1092BA0D1092BB0D4F
:109C50001092BC0D1092BD0D1092BE0D1092BF0D52
:109C60001092C00D0E94D9C9E9E7F4E2A491A8AF0F
:109C7000EDE6F4E2C590D590E590F490E1E7F4E2EA
:109C800085909590A590B490A5019401C701B60167
:109C90000F946E3918162CF4A7019601C501B40172
:109CA00004C0A5019401C701B6010F9408382B0127
:109CB0003C01E4E3F4E285919591A591B4918CA3E4
:109CC0009DA3AEA3BFA3E0E3F4E285919591A59196
:109CD000B49188A799A7AAA7BBA79C01AD016CA1C5
:109CE0007DA18EA19FA10F946E39181634F428A47B
:109CF00039A49AA598AB1BA505C02CA03DA0AEA188
:109D0000A8AB1FA1A3019201C301B2010F947E3041
:109D100020E030E040E85FE30F940E370F94BC3949
:109D2000910148A9512F0F947E3068A379A38AA38B
:109D30009BA3EAE7F4E2149120E030E040EC5FE31B
:109D4000C501B4010F947E304B015C01612F110FEE
:109D5000770B880B990B0F941F309B01AC01C50149
:109D6000B4010F947E3069837A838B839C8320E0D7
:109D700030E040EC5FE3C701B6010F947E306B0129
:109D80007C01B8AD6B2FBB0F770B880B990B0F9431
:109D90001F309B01AC01C701B6010F947E306C8F60
:109DA0007D8F8E8F9F8FAE01405E5F4FBE016F5FD4
:109DB0007F4FCE014C960E9404C90E9478EA10920F
:109DC000B90D1092BA0D1092BB0D1092BC0D1092ED
:109DD000BD0D1092BE0D1092BF0D1092C00D80E00F
:109DE0000E94DBC9002319F081E00E94DBC9ECA5C9
:109DF000EE2309F484C080E00E94CBD18091FA1355
:109E00008370833051F060E080EC97E00F944E1A3D
:109E10000F94501781EB97E06EC00E94D9C98090D3
:109E2000C10D9090C20DA090C30DB090C40D2091B3
:109E3000A20D3091A30D4091A40D5091A50D60E0AD
:109E400070E088E492E40F940D376093850D709371
:109E5000860D8093870D9093880D2091A60D3091EB
:109E6000A70D4091A80D5091A90D60E070E08CE81D
:109E700092E40F940D376B017C016093890D709310
:109E80008A0D80938B0D90938C0D2091AA0D3091AB
:109E9000AB0D4091AC0D5091AD0DC501B4010F94C7
:109EA0000D3760938D0D70938E0D80938F0D909371
:109EB000900DB701A60185E89DE00F945C1E8823F4
:109EC00089F019821A821B821C82AE014F5F5F4F9C
:109ED00069E87DE085E89DE00E9404C982E00E9477
:109EE000DBC90BC060E080EA97E00F944E1A0F9434
:109EF00050178EE897E00F9467160F94910F0E9409
:109F0000D9C98091A1098093A2098CA90E9447D246
:109F10000E9481C70E9407CBE2CC8CA747CE61E0AC
:109F20008CE898E00E94BFCC87E198E00E9472F92B
:109F300061E08DEF9CE30E94BFCC88E098E00E9436
:109F400014FBB1100C94E1400C94DA4080E00E94C4
:109F500056550C940D4188E50E943CCC81115F98C8
:109F600089E50E943CCC81118A988AE50E943CCC0C
:109F7000882329F08091080181708093060185E48F
:109F80000E943CCC882309F4AACC12984798A7CC0D
:109F900060E08FE099E00F944E1A5F988A98809164
:109FA00008018170809306011298479898CC0E940E
:109FB000DDCBAB01BC014093E7175093E8176093EA
:109FC000E9177093EA178AED94E10E94449987CCCF
:109FD00061E0802F0E940AE26F2D802F0E94DBE15A
:109FE0006F2D70E0802F0F94C01EA7E0EA1203C00F
:109FF000F092B10D74CCB9E0EB1271CCF092B00DCF
:10A000006ECC0E94EDCB90E08536910514F084E68D
:10A0100090E08093231F63CC0F9495100C943944E7
:10A02000802F0E94F4670C9455440E9405CC0F9435
:10A030007A38CB010E94C97D0E9405CC20E030E037
:10A0400040EA50E40F946E39181614F40F949510EA
:10A0500060917E0970917F09072E000C880B990B87
:10A060000F941F3020917A0930917B0940917C092F
:10A0700050917D090F946E3918161CF48FE29AE006
:10A0800002C080E29AE060E00F944E1A812F0E9495
:10A09000956825CC0E948CFF88E50E943CCC8823E3
:10A0A00031F05F9A8091FA138E7F8093FA1389E5DD
:10A0B0000E943CCC882331F08A9A8091FA138D7FDC
:10A0C0008093FA138AE50E943CCC882359F0809152
:10A0D000080180958170809306018091FA138B7F2F
:10A0E0008093FA1385E40E943CCC882309F4F7CBD3
:10A0F0000E949651F4CB0F943C01F1CBB7FAB09487
:10A10000B7F8B094F70180829182A282B382A2CA8A
:10A110000F944C178CE39DE00F94671661E08EE27C
:10A120009DE00F944E1A68E270E088EC90E00F9486
:10A13000EF19D5CB0C5F1F4FFFEFCF1ADF0A24E2D8
:10A140000033120709F056CA45EAE42E49E0F42E1E
:10A1500010E0F10181919191A191B1911F01F7015D
:10A1600081939193A193B1937F01812F0E94BFC3EB
:10A170001F5F133071F70E9407CB60E08EE19DE016
:10A180000F944E1A63E972E084E690E00F94EF19A1
:10A190006AEB72E084E690E00F94EF19A0CBCF92C7
:10A1A000DF92EF92FF920F931F93CF93DF936C0197
:10A1B0008B017A01EC01C258D74F888187FF04C018
:10A1C000FB011182108224C02CE02C9DC0012D9D2A
:10A1D000900D11242881AC01420F511D27FD5A9585
:10A1E0002091BA1530E04217530794F42881AC014E
:10A1F000420F511D27FD5A959A01FA01EE0FFF1FDC
:10A200002E0F3F1FF901E25BFA4E208127FD19C096
:10A2100088818F5F88832CE02C9DC0012D9D900D3F
:10A2200011242881AC01420F511D27FD5A95209120
:10A23000BA1530E042175307BCF428812C3044F1A2
:10A2400013C02881820F911D27FD9A95FC01EE0F06
:10A25000FF1F8E0F9F1FFC01E25BFA4E808160E0C2
:10A260008F770E94DBE1D4CFF80180819181049641
:10A2700080349C4918F480E49CE904C0F801808192
:10A2800091810496F701918380838FEF888345C085
:10A29000F801408151812881BC01620F711D27FDA9
:10A2A0007A959B01FB01EE0FFF1F2E0F3F1FF90157
:10A2B000E25BFA4E21813281240F351FF701318391
:10A2C00020832881AC01420F511D27FD5A959A0128
:10A2D000FA01EE0FFF1F2E0F3F1FF901E25BFA4E4E
:10A2E000208127FF1AC02881820F911D27FD9A9592
:10A2F000FC01EE0FFF1F8E0F9F1FFC01E25BFA4E69
:10A30000808161E08F77DF91CF911F910F91FF9056
:10A31000EF90DF90CF900C94DBE1DF91CF911F9114
:10A320000F91FF90EF90DF90CF900895129A479A87
:10A330000895FF920F931F93CF93DF931F92CDB792
:10A34000DEB7F82E00EC1DE041E050E0B801CE0190
:10A3500001960F94522F89818F1102C081E007C0AE
:10A360000F5F1F4F8DE00C3D180771F780E00F90D5
:10A37000DF91CF911F910F91FF90089580918108F7
:10A38000811107C00E9484EF882319F081E0809337
:10A39000810808959091EB1793FB882780F993FF2C
:10A3A00006C081E09091DD14911101C080E0089514
:10A3B00060E070E080E00F94E90D60E070E081E023
:10A3C0000D94E90DDC01EC91F0E0CF01880F991FAD
:10A3D000E80FF91FE25BFA4E80818F778083089542
:10A3E0008F929F92AF92BF92CF92DF92EF92FF92A5
:10A3F0000F93CF93DF931F92CDB7DEB75C016B0154
:10A400007A014901F501808191810F944836898351
:10A41000002311F0F6018083BE016F5F7F4FC401FE
:10A420000E94ABFAF501808191810196918380832E
:10A43000FFEFCF1ADF0A81E0E81AF10819F780E090
:10A440000F90DF91CF910F91FF90EF90DF90CF9021
:10A45000BF90AF909F908F9008957F928F929F9220
:10A46000AF92BF92CF92DF92EF92FF920F931F9322
:10A47000CF93DF931F92CDB7DEB77C0159018B01DB
:10A480006B01C40ED51E0C151D0559F1F701808016
:10A490009180F80171908F017982C4010F94483640
:10A4A000781691F0672DC4010F945036C4010F94B3
:10A4B00048369981891741F00F94501786EA9DE03C
:10A4C0000F94671681E00EC0BE016F5F7F4FC5011C
:10A4D0000E94ABFAF701808191810196918380837C
:10A4E000D2CF80E00F90DF91CF911F910F91FF901D
:10A4F000EF90DF90CF90BF90AF909F908F907F9024
:10A500000895009781F41092900082E0809391006A
:10A510001092950010929400C19A8091710082600F
:10A520008093710008958130910569F41092A00024
:10A5300082E08093A1001092A5001092A40089BB34
:10A54000809372000895029761F41092200182E0D6
:10A550008093210110922501109224018ABB8093DF
:10A56000730008957F928F929F92AF92BF92CF9285
:10A57000DF92EF92FF920F931F93CF93DF93FC0133
:10A580009081943208F0CEC06B017F01892F90E05A
:10A59000FC01EE0FFF1F8E0F9F1FFC01E25BFA4EC6
:10A5A000808161E08F770E940AE2F70111821282B6
:10A5B00080816CE00F94D136FCE08F9FB0011124B4
:10A5C00040E050E09B01240F351FF901EE0FFF1F03
:10A5D0002E0F3F1FF901E25BFA4E908197FD08C0F4
:10A5E0004F5F5F4F4C30510569F790E00E948152F8
:10A5F000F7017080C72DD0E08E01000F111FF80108
:10A60000EC0FFD1FE25BFA4E80818068808377FC4F
:10A6100089C0F0E2CF16F2E0DF060CF041C0F7018E
:10A62000828128E532E0281B310987FD3395220F0E
:10A63000331F220F331F032E000C440B550B818157
:10A6400068E870E04B01881A910887FD9394880CA4
:10A65000991C880C991C092C000CAA08BB08D7FC73
:10A660000BC0B601653B710514F064EB70E0072E7A
:10A67000000C880B990B03C060E070E0CB01281937
:10A6800039094A095B090F945E3624EB30E040E05B
:10A6900050E00F949036820E931EA41EB51E01C08A
:10A6A0004601F3E2F71558F1F701218188E890E0BF
:10A6B000821B910927FD9395880F991F880F991F79
:10A6C0008816990684F0F701228188E592E0821BC2
:10A6D000910927FD9395880F991F880F991F881658
:10A6E00099060CF4C40102972FB7F894C00FD11F3C
:10A6F000C25BDA4E880F991F9A8389832FBF62E36A
:10A7000070E080E090E0DF91CF911F910F91FF907A
:10A71000EF90DF90CF90BF90AF909F908F907F9001
:10A720000D943816DF91CF911F910F91FF90EF900C
:10A73000DF90CF90BF90AF909F908F907F900895C3
:10A740001F920F920FB60F9211240BB60F922F93F8
:10A750003F934F935F936F937F938F939F93AF93A9
:10A76000BF93EF93FF9348E251E064E271E082E02F
:10A7700090E00E94CF50FF91EF91BF91AF919F91D8
:10A780008F917F916F915F914F913F912F910F909A
:10A790000BBE0F900FBE0F901F9018951F920F9237
:10A7A0000FB60F9211240BB60F922F933F934F9336
:10A7B0005F936F937F938F939F93AF93BF93EF9329
:10A7C000FF9348EA50E064EA70E081E090E00E9484
:10A7D000CF50FF91EF91BF91AF919F918F917F915A
:10A7E0006F915F914F913F912F910F900BBE0F9002
:10A7F0000FBE0F901F9018951F920F920FB60F92D9
:10A8000011240BB60F922F933F934F935F936F9347
:10A810007F938F939F93AF93BF93EF93FF9348E9F9
:10A8200050E064E970E080E090E00E94CF50FF913A
:10A83000EF91BF91AF919F918F917F916F915F91B8
:10A840004F913F912F910F900BBE0F900FBE0F9025
:10A850001F9018959091C00095FFFCCF8093C60083
:10A8600008958F929F92AF92BF92EF92FF920F93B3
:10A870001F93CF93DF93CDB7DEB7A0970FB6F894B1
:10A88000DEBF0FBECDBF611571058105910591F148
:10A8900000E0842E912CA12CB12C102FEE24E394F7
:10A8A000F12CEC0EFD1EE00EF11C07FDFA94A50143
:10A8B00094010F946E36F7016083B901CA010F5FEE
:10A8C000611571058105910541F71F3F31F1E1E007
:10A8D000F0E0EC0FFD1FE10FF11D17FDFA958081EF
:10A8E0008A3010F097E301C090E3890F0E942A5448
:10A8F0001150EBCF80E3A0960FB6F894DEBF0FBEE9
:10A90000CDBFDF91CF911F910F91FF90EF90BF903E
:10A91000AF909F908F900C942A54A0960FB6F89405
:10A92000DEBF0FBECDBFDF91CF911F910F91FF9082
:10A93000EF90BF90AF909F908F900895CF92DF924D
:10A94000EF92FF926B017C0197FF0BC08DE20E949A
:10A950002A54F094E094D094C094C11CD11CE11C02
:10A96000F11C4AE0C701B601FF90EF90DF90CF9055
:10A970000C9431548F929F92AF92BF92CF92DF92FC
:10A98000EF92FF92CF936B017C01B42E20E030E078
:10A99000A9010F94183087FF07C08DE20E942A5446
:10A9A000F7FAF094F7F8F094C0E060E070E080E02F
:10A9B0009FE3CB1541F02DEC3CEC4CEC5DE30F94A8
:10A9C0007E30CF5FF6CF9B01AC01C701B6010F947B
:10A9D0000E376B017C010F9481384B015C014AE01A
:10A9E0000E943154CC2389F1C501B4010F941D306C
:10A9F0009B01AC01C701B6010F940D376B017C01BF
:10AA00008EE20E942A5420E030E040E251E4C70187
:10AA1000B6010F947E304B015C010F947A386B01C4
:10AA2000770FEE08FF08C701B6010E949E54C701C8
:10AA3000B6010F941F309B01AC01C501B4010F9406
:10AA40000D376B017C01C150F1F6CF91FF90EF9073
:10AA5000DF90CF90BF90AF909F908F9008958DE042
:10AA60000E942A548AE00C942A54CF93DF93EC017D
:10AA70008991882319F00E942A54FACFDF91CF914F
:10AA80000C942F558091AA0C9091AB0C981759F00B
:10AA9000E92FF0E0E655F34F82819F5F9F77909317
:10AAA000AB0C90E008958FEF9FEF08952F923F92A7
:10AAB0004F925F926F927F928F929F92AF92BF92CE
:10AAC000CF92DF92EF92FF920F931F93CF93DF937A
:10AAD000CDB7DEB728970FB6F894DEBF0FBECDBF57
:10AAE000E82E0E94F41E0F94E21F4B015C0180913E
:10AAF0000002882359F180916B08882339F1409135
:10AB000082085091830860918408709185089501AE
:10AB10008401041B150B260B370B37FD2AC083302D
:10AB200079F03CF4813094F00F9450178BE09EE064
:10AB30000BC0843059F40F9450178CED9DE004C085
:10AB40000F94501784EF9DE00F9467162091000238
:10AB500030E0A8EEB3E00F94C236860E971EA81E12
:10AB6000B91E8092820890928308A0928408B092C5
:10AB700085088091350B843008F07FC20F94E21F66
:10AB80004B015C018091350B81111DC08091AA0C95
:10AB90009091AB0C891B8F77B1F48091EB08909169
:10ABA000EC08A091ED08B091EE08A5019401281BD6
:10ABB000390B4A0B5B0BDA01C901885E9340A1098E
:10ABC000B109B7FF61C560E6F62E8091350B843080
:10ABD00008F036C18091AA0C9091AB0C891B8F773D
:10ABE00009F42EC10E944255AC0197FDEECF209191
:10ABF0002C0D30912D0D8A3019F08D3009F0E8C000
:10AC00001092EA082115310519F40F94D009DDCF0F
:10AC1000F901E657F74F108210922D0D10922C0D6E
:10AC20000AE818E0F8018191803211F48F01FACF1F
:10AC30008E3409F07AC00115110509F476C064E478
:10AC40007FE0C8010F94962F6C01892B41F06EE4D0
:10AC500070E0C80104960F94613A009709F4C801A6
:10AC60004AE050E060E070E001960F940E2D609392
:10AC7000860870938708809388089093890840908D
:10AC80002E0D50902F0D6090300D7090310D3FEFD4
:10AC9000431A530A630A730A6415750586059705F6
:10ACA00031F0CD2821F460E081E19FE0C7C06AE285
:10ACB00070E0C8010F94903A9C01009709F1982F19
:10ACC000901BD12C992339F09150F801E90FF11D17
:10ACD0008081D826F7CF4AE050E060E070E0C901FB
:10ACE00001960F940E2D4D2C512C612C712C641556
:10ACF00075058605970541F060E082EF9EE09EC0F5
:10AD000060E088EC9EE09AC0809186089091870868
:10AD1000A0918808B091890880932E0D90932F0DF3
:10AD2000A093300DB093310D12C08091EB1780FFCE
:10AD30000EC06EED78E1C8010F94962F009709F4CC
:10AD40007AC0FC01838180538A3008F474C08091FA
:10AD5000290281111CC067E470E0C8010F94613AB8
:10AD60000097A9F04AE050E060E070E001960F948F
:10AD70000E2D643071058105910548F487E29EE04F
:10AD80000F94671660E08DE19EE00F944E1A80925A
:10AD9000EB089092EC08A092ED08B092EE0880913A
:10ADA0008A088B3309F411CF8091350B843008F079
:10ADB0000CCF8091B109F89EC00111246AE878E0B7
:10ADC0008C54964F0F946C3A81E00E9494F0FDCE23
:10ADD0002F3531050CF0F9CE8C35C1F40E94425567
:10ADE00097FDF3CE2091EA082111EFCE20912C0D92
:10ADF00030912D0DA9014F5F5F4F50932D0D409362
:10AE00002C0DF901E657F74F8083DFCE8B3321F409
:10AE100081E08093EA08D9CE8091EA088111D5CEED
:10AE2000C901019690932D0D80932C0DF901E657E1
:10AE3000F74F4083CACE60E08EE99EE00E949CAB53
:10AE40008091EB1782FF19C18091350B811102C0EF
:10AE50001092F008DD24D3944091E7175091E81741
:10AE60006091E9177091EA178091E3179091E417C8
:10AE7000A091E517B091E617481759076A077B07B5
:10AE800008F4D12C00E010E0CC24C39430E6B32EBB
:10AE900044E6A42E59E6952E8091350B843008F0B7
:10AEA000ECC0D110EAC08091F0088111E6C0809119
:10AEB000E2149091E314A091E414B091E51480930E
:10AEC000E7179093E817A093E917B093EA1741E0CA
:10AED00050E0BE016F5F7F4F8AED94E10E94299D93
:10AEE000019719F4898190E002C08FEF9FEFF82E4F
:10AEF0004090E7175090E8176090E9177090EA17B4
:10AF00004091E3175091E4176091E5177091E617AF
:10AF1000DD24D394441655066606770608F4D12C32
:10AF20004416550666067706B0F4019609F461C02A
:10AF30002AE0F21609F46EC03DE0F31609F46AC087
:10AF400043E2F41619F05AE3F5127CC08091EF0841
:10AF5000811178C054C00E948CFF8AED94E10E9458
:10AF6000B09C8091E217882339F181508093E217D9
:10AF7000989EC001112441E061E08153944F0E94EA
:10AF80001878E091E21764E0E69FF0011124E553A0
:10AF9000F44F40815181628173814093E717509350
:10AFA000E8176093E9177093EA178AED94E10E941D
:10AFB00044990E94CC7416C00E94BB740F943C014B
:10AFC0000F9445110F9449186D3371058105910552
:10AFD00018F48FE49FE002C084E59FE00E94C5ABB7
:10AFE000A092231F8091EB1782FD0DC087E69FE0A2
:10AFF00004C00F944C1788E59FE00F94671673E226
:10B00000F71208C005C053E2F5124BC300E010E090
:10B01000C092F0081092EF080115110519F40F9471
:10B02000D0090DC08091B109B89E000D111D1124E9
:10B03000F801EC54F64F108280E00E9494F000E09A
:10B0400010E02ACF0F35110508F026CF8BE3F81258
:10B0500003C0C092EF0820CF8091EF0881111CCF70
:10B060008091B109F801B89EE00DF11D1124EC5456
:10B07000F64FF0820F5F1F4F0FCF0F94E21F4B016F
:10B080005C01409166085091670860916808709172
:10B090006908411551056105710529F18091F21387
:10B0A0009091F313A091F413B091F513840F951FB1
:10B0B000A61FB71F95018401081B190B2A0B3B0B18
:10B0C00037FD11C00F944C176091B60D7091B70DFC
:10B0D0008BE79FE00F9439178AE00E942A5480E0A2
:10B0E00090E00E9414FB4091010250910202609195
:10B0F000030270910402411551056105710509F4BF
:10B100004EC09091C1158091C215981759F00F94B7
:10B11000E21F6093F2137093F3138093F4139093F0
:10B12000F5133DC08091CA0B811137C0E11035C0C5
:10B130008091F2139091F313A091F413B091F51351
:10B14000840F951FA61FB71FA5019401281B390B5B
:10B150004A0B5B0B57FD21C08091010981111FC073
:10B1600081E0809301095F9A8091FA138E7F80932A
:10B17000FA138A9A8091FA138D7F8093FA13809143
:10B18000080180958170809306018091FA138B7F6E
:10B190008093FA130E94965102C010920109809187
:10B1A000FD089091FE08A091FF08B0910009B5013B
:10B1B000A401481B590B6A0B7B0B77FDABC1909127
:10B1C000C1158091C215609122023091230298131B
:10B1D0000FC08091B00D869F80011124B801660FC9
:10B1E000672F661F770B7195062F8091B10D17C0E1
:10B1F0008091C21554E6859FC00111248E54974E4C
:10B20000FC01EE59FF4F2081269FB0011124660FEB
:10B21000672F661F770B7195062F31968081839F6C
:10B22000B0011124660F672F661F770B7195162FDB
:10B23000002331F10F94E21FC090F508D090F6087A
:10B24000E090F708F090F808DC01CB01C114D104BC
:10B25000E104F10469F48C599F4FAF4FBF4F8093C5
:10B26000F5089093F608A093F708B093F80806C085
:10B270008C199D09AE09BF09B7FF0AC00FEF08C0BE
:10B280001092F5081092F6081092F7081092F8083C
:10B29000602F70E089E00F94C01E112331F10F94EC
:10B2A000E21FC090F908D090FA08E090FB08F090F7
:10B2B000FC08DC01CB01C114D104E104F10469F400
:10B2C0008C599F4FAF4FBF4F8093F9089093FA0866
:10B2D000A093FB08B093FC0806C08C199D09AE0929
:10B2E000BF09B7FF0AC01FEF08C01092F9081092FB
:10B2F000FA081092FB081092FC08612F70E087E0BA
:10B300000F94C01E80914E0B882309F4F6C0E09084
:10B310006702F09068020091690210916A026091E0
:10B320006709709168096E5F7F4F072E000C880BCC
:10B33000990B0F941F309701A8010F94183087FDC7
:10B34000DCC03090C215212C1A821B821C82809195
:10B35000C115831509F467C0832D90E064E6689FEA
:10B36000F001699FF00D1124EE54F74E458956897E
:10B370006789708D452B462B472B89F4418D528D63
:10B38000638D748D452B462B472B49F4458D568D87
:10B39000678D70A1452B462B472B09F43FC074E6FF
:10B3A000789F9001799F300D1124C9018E54974EDA
:10B3B0006C01FC0161817281838194810F94BC399D
:10B3C0002B013C01F60161A172A183A194A10F940C
:10B3D0001D306D837E838F839887F60165A176A1EA
:10B3E00087A190A50F941D309B01AC016D817E81DA
:10B3F0008F8198850F940838A30192010F947E30B5
:10B400003B016C01222D3A814B815C810F946E3996
:10B41000181624F4262C7A82CB82DC8281E0830DFC
:10B420008F70382E94CF20916B0230916C02409136
:10B430006D0250916E02622D7A818B819C810F94F6
:10B440007E309701A8010F940E373B016C012090CC
:10B4500063023090640240906502509066029B0146
:10B46000AC01B701C8010F946E3918166CF0910148
:10B47000A201B301C6010F946E3918161CF47101B4
:10B48000820102C0730186014090F1085090F208D9
:10B490006090F3087090F4089701A801C301B2010D
:10B4A0000F946E391816C4F420E037ED43EA5CE3DC
:10B4B000B701C8010F947E306B017C0128E431EEA6
:10B4C0004AE75FE3C301B2010F947E30A701960102
:10B4D0000F940E377B018C01C701D8018093F108CE
:10B4E0009093F208A093F308B093F408B701C80151
:10B4F0000F947A38CB010E94A4A1F4E68F0E911C20
:10B50000A11CB11C8092FD089092FE08A092FF0839
:10B51000B09200090F94D0098091AD18813009F0E4
:10B520006EC00F94E21F6B017C018091060990911F
:10B530000709A0910809B091090997018601081B24
:10B54000190B2A0B3B0B37FD3AC08090AE18909038
:10B55000AF18A090B018B090B1180F94491860932C
:10B56000AE187093AF188093B0189093B1180091F3
:10B570009509109196092091970930919809081919
:10B5800019092A093B09DC01CB01800F911FA21F79
:10B59000B31F8093950990939609A0939709B09350
:10B5A0009809D701C601805F984DAF4FBF4F809378
:10B5B000060990930709A0930809B093090980919F
:10B5C000020990910309A0910409B0910509A7010E
:10B5D0009601281B390B4A0B5B0B57FD10C030E856
:10B5E000C30E3EEED31EE11CF11CC0920209D092A4
:10B5F0000309E0920409F09205090F941F110F94BA
:10B60000671980916508882391F00F94E21F0091DB
:10B610006108109162082091630830916408DC0190
:10B62000CB01801B910BA20BB30BB7FF3DC00F9456
:10B63000E21F6B017C0120916008222309F453C0B2
:10B6400080915C0890915D08A0915E08B0915F08C0
:10B65000B701A601481B590B6A0B7B0B77FD43C052
:10B6600030E0A8EEB3E00F94C236C60ED71EE81E37
:10B67000F91EC0925C08D0925D08E0925E08F092DC
:10B680005F080E9494742FC089E49FE00F946716AE
:10B690008092EB089092EC08A092ED08B092EE0830
:10B6A00092CA1092EF08BBCC0F94E21F6B017C0191
:10B6B0002091650830E0A8EEB3E00F94C236C60EC4
:10B6C000D71EE81EF91EC0926108D0926208E0926F
:10B6D0006308F09264088091B80D0E941E688AE0A9
:10B6E0000E942A54A4CF28960FB6F894DEBF0FBE4E
:10B6F000CDBFDF91CF911F910F91FF90EF90DF9021
:10B70000CF90BF90AF909F908F907F906F905F9001
:10B710004F903F902F9008951F920F920FB60F9267
:10B7200011240F900FBE0F901F9018951F920F922B
:10B730000FB60F9211240BB60F920F931F932F93F6
:10B740003F934F935F936F937F938F939F93AF93A9
:10B75000BF93CF93DF93EF93FF930091AB0CD09106
:10B76000AA0C11E01D0F1F77C091C60090917D08B3
:10B77000492F092E000C550B660B770B41315105F3
:10B7800008F064C0FA018827E256FF4F8F4F0D94EE
:10B790000537CD3449F0CE34B9F481E006C0CA3360
:10B7A00038F0CD3409F043C082E080937D0876C044
:10B7B000C03308F073C0C03209F470C0CD32B9F59F
:10B7C0006DC0C13351F018F4C03289F567C0C4337D
:10B7D00031F0C83361F58BE0E8CF83E0E6CF88E055
:10B7E000E4CFC03321F0C13311F586E0DECF84E031
:10B7F000DCCFC833E1F485E0D8CFC233C1F487E0B1
:10B80000D4CFC133A1F489E0D0CFC03381F48AE032
:10B81000CCCFC73361F48CE0C8CFC63341F48DE0A0
:10B82000C4CFC032D9F1C33511F48EE0BECF80E170
:10B83000BCCF80ED8C0F8A3088F59FE090937D0817
:10B8400080937C082BC0CA3049F526C0CA3031F538
:10B850008091D116882301F1973089F03CF495301E
:10B86000D9F4109221021092221F16C09A3059F07A
:10B870009F3091F480917C080E941BCD0DC081E027
:10B880008093661809C00F9492010E948CFF8EEF7E
:10B890000E946BC90E94D9C910927D08011731F02E
:10B8A000ED2FF0E0E655F34FC283D12FD093AA0CD1
:10B8B000FF91EF91DF91CF91BF91AF919F918F91C8
:10B8C0007F916F915F914F913F912F911F910F91B8
:10B8D0000F900BBE0F900FBE0F901F9018958EBD4E
:10B8E0000DB407FEFDCF08958FEF8EBD0DB407FE9A
:10B8F000FDCF8EB50895909164009B7F9093640076
:10B90000982F906A96959CBD80FD03C091E086308B
:10B9100009F490E09DBD08952F923F924F925F925F
:10B920006F927F928F929F92AF92BF92CF92DF924F
:10B93000EF92FF920F931F93CF93DF93CDB7DEB7B4
:10B9400062970FB6F894DEBF0FBECDBF8FEF9FEFAB
:10B9500090938900809388002AE02A8B212C312C37
:10B96000789480915A0990915B09A0915C09B091FB
:10B970005D09892B8A2B8B2B09F0D7C1809149183F
:10B980008823E1F010924918809147189091481847
:10B99000892B09F4CAC1109212091092481810920A
:10B9A00047189091C1158091C215981709F4BDC12F
:10B9B0008091C2158F5F8F708093C2158091471858
:10B9C00090914818892B09F4B0C1409156095091C3
:10B9D00057096091580970915909809152099091C5
:10B9E0005309A0915409B09155090091490910E0FB
:10B9F00020E030E0841B950BA60BB70B0817190746
:10BA00002A073B0710F4D901C801E82F840F951FBE
:10BA1000A61FB71F8093560990935709A093580902
:10BA2000B09359092091840030918500225E3F4FE8
:10BA300040911E0950911F096091200970912109C0
:10BA400080912E0990912F09A0913009B091310970
:10BA5000840F951FA61FB71F80932E0990932F095F
:10BA6000A0933009B0933109B7FD1CC0889A80912A
:10BA70000A09082E000C990BAA0BBB0B4091561813
:10BA8000509157186091581870915918840F951F4C
:10BA9000A61FB71F8093561890935718A093581855
:10BAA000B0935918409122095091230960912409BB
:10BAB000709125098091320990913309A091340940
:10BAC000B0913509840F951FA61FB71F80933209C7
:10BAD00090933309A0933409B0933509B7FD1CC086
:10BAE0008E9A80910B09082E000C990BAA0BBB0BA8
:10BAF00040915A1850915B1860915C1870915D18D4
:10BB0000840F951FA61FB71F80935A1890935B1838
:10BB1000A0935C18B0935D184091260950912709B5
:10BB2000609128097091290980913609909137090F
:10BB3000A0913809B0913909840F951FA61FB71F2E
:10BB40008093360990933709A0933809B093390947
:10BB5000B7FD21C080910B01809588708093090109
:10BB600080910C09082E000C990BAA0BBB0B40917D
:10BB70005E1850915F186091601870916118840F81
:10BB8000951FA61FB71F80935E1890935F18A09310
:10BB90006018B093611840913A0950913B09609147
:10BBA0003C0970913D0980912A0990912B09A0913F
:10BBB0002C09B0912D09840F951FA61FB71F8093E4
:10BBC0003A0990933B09A0933C09B0933D09B7FD16
:10BBD0003AC040910D09042E000C550B660B770BF3
:10BBE000C0906218D0906318E0906418F0906518C7
:10BBF0004C0D5D1D6E1D7F1D4093621850936318A0
:10BC0000609364187093651840911A0950911B094C
:10BC100060911C0970911D09841B950BA60BB70B35
:10BC200080933A0990933B09A0933C09B0933D0956
:10BC30009091A3098091470993FF02C0815001C0F0
:10BC40008F5F8093470980918400909185008217CF
:10BC50009307C8F380912E0990912F09A091300984
:10BC6000B0913109B7FD15C040911A0950911B09D7
:10BC700060911C0970911D09841B950BA60BB70BD5
:10BC800080932E0990932F09A0933009B093310926
:10BC900088988091320990913309A0913409B0912C
:10BCA0003509B7FD15C040911A0950911B096091E3
:10BCB0001C0970911D09841B950BA60BB70B809373
:10BCC000320990933309A0933409B09335098E98C3
:10BCD0008091360990913709A0913809B0913909BE
:10BCE000B7FD19C040911A0950911B0960911C09B8
:10BCF00070911D09841B950BA60BB70B8093360919
:10BD000090933709A0933809B093390980910B01BA
:10BD1000887080930901E15041F0809184009091F6
:10BD2000850082179307C8F381CE80910E0290910F
:10BD30000F02A0911002B0911102892B8A2B8B2B3C
:10BD400009F0ADC080914809882309F453C0809060
:10BD5000560990905709A0905809B0905909C09081
:10BD60004309D0904409E0904509F090460940917C
:10BD70004709C814D904EA04FB0480F48091170928
:10BD80009091180920911509309116092817390743
:10BD900028F4415040934709019714C08C149D0426
:10BDA000AE04BF04E0F48091170990911809209126
:10BDB0001309309114098217930788F44F5F409359
:10BDC00047090196909318098093170940910A0238
:10BDD00050910B0260910C0270910D020EC08FEF1A
:10BDE0009FEFDC0180930A0290930B02A0930C0258
:10BDF000B0930D024FEF5FEFBA01000000000000AA
:10BE0000909147098091190997FD06C0811102C0E0
:10BE1000169A07C0439805C0811102C0169801C048
:10BE2000439A0000000000008091840090918500FA
:10BE30004E9620914709222351F120911909211191
:10BE400002C0149A01C0419A20918400309185006B
:10BE500028173907C8F32091470927FF02C02F5F31
:10BE600001C021502093470920911909211102C0D6
:10BE7000149801C04198209147092223D1F22091C2
:10BE800084003091850028173907C8F3D1CF40933B
:10BE90000E0250930F026093100270931102809172
:10BEA0005A0990915B09A0915C09B0915D09892BB9
:10BEB0008A2B8B2B11F00C94A565A0914718B0919B
:10BEC0004818109711F40C94BC6780905609909014
:10BED0005709A0905809B0905909409152095091C2
:10BEE0005309609154097091550984169506A60668
:10BEF000B706D8F0109212091092481810924718FD
:10BF00009091C1158091C215981711F40C94BC67DB
:10BF10008091C2158F5F8F708093C21540EDC42E43
:10BF200047E0D42EE12CF12C1CC440914E095091D5
:10BF30004F096091500970915109481559056A05DA
:10BF40007B0508F4ABC140914A0950914B096091BF
:10BF50004C0970914D09D6960D911D912D913C91F2
:10BF6000D997401751076207730708F078C1411548
:10BF700051056105710549F480900E0990900F09F3
:10BF8000A0901009B090110965C1E12CF980842EB0
:10BF9000952F862F0A811B81FD81EE813F812885A7
:10BFA0009C80E091F21EE89D912CFF273091F31EBA
:10BFB000389D900CF11D1090F41E189CF00DE99F17
:10BFC000900CF11D399FF00DE89FF00D092D1F2FEA
:10BFD000099DE12D332722270F9FE00D311D2E1DD6
:10BFE000199DE00D311D2E1D1F9F300D211D032FAA
:10BFF000122F099DF12C332722270F9FF00C311DA2
:10C000002E1D199DF00C311D2E1D1F9F300D211D61
:10C01000032F122FEE2780900E0990910F09809127
:10C020001009009078080E2809F484C03091740833
:10C03000309FE1198E089E098E0920917508209F76
:10C04000E01981089E098E09F0907608F09E80180C
:10C0500091098E09319FE01981089E098E09219F5F
:10C06000801891098E09F19E90198109099DF12C82
:10C07000332722270F9FF00C311D2E1D199DF00C28
:10C08000311D2E1D1F9F300D211D032F122F3091AA
:10C090007008309FE10D8E1C9E1D8E1D2091710831
:10C0A000209FE00D811C9E1D8E1DF0907208F09E59
:10C0B000800C911D8E1D319FE00D811C9E1D8E1DDB
:10C0C000219F800C911D8E1DF19E900D811D099D5B
:10C0D000F12C332722270F9FF00C311D2E1D199DA7
:10C0E000F00C311D2E1D1F9F300D211D032F122F0F
:10C0F00030916C08309FE1198E089E098E092091BD
:10C100006D08209FE01981089E098E09F0906E0845
:10C11000F09E801891098E09319FE01981089E09CF
:10C120008E09219F801891098E09F19E901981092D
:10C130000C941C6130917408309FE10D8E1C9E1D83
:10C140008E1D20917508209FE00D811C9E1D8E1D67
:10C15000F0907608F09E800C911D8E1D319FE00DB1
:10C16000811C9E1D8E1D219F800C911D8E1DF19E98
:10C17000900D811D099DF12C332722270F9FF00C74
:10C18000311D2E1D199DF00C311D2E1D1F9F300DD0
:10C19000211D032F122F30917008309FE1198E0856
:10C1A0009E098E0920917108209FE01981089E093F
:10C1B0008E09F0907208F09E801891098E09319FC7
:10C1C000E01981089E098E09219F801891098E0926
:10C1D000F19E90198109099DF12C332722270F9F89
:10C1E000F00C311D2E1D199DF00C311D2E1D1F9FB1
:10C1F000300D211D032F122F30916C08309FE10D5F
:10C200008E1C9E1D8E1D20916D08209FE00D811CAF
:10C210009E1D8E1DF0906E08F09E800C911D8E1D4F
:10C22000319FE00D811C9E1D8E1D219F800C911D54
:10C230008E1DF19E900D811D11249C82F9820A832E
:10C240001B83FD83EE833F832887912C992AA12CA1
:10C25000B12CA82A85EB97E121E0298B14C0D29656
:10C260008D909D90AD90BC90D597F4CFB694A79447
:10C2700097948794D988DD0CD98A049627E1813D6B
:10C28000920709F4DDC4FC010591159125913491C3
:10C29000081519052A053B0548F3D2C44090430907
:10C2A000509044096090450970904609481459041B
:10C2B0006A047B0408F0C4C180914209811121C045
:10C2C000FD01EE5BFF4FE080F180028113817896E3
:10C2D0002081318142815381D2966D917D918D91E2
:10C2E0009C91D5970F94980EDD24D394D092420957
:10C2F000E0914718F091481882A993A9A4A9B5A97B
:10C300008FC140913E0950913F0960914009709161
:10C310004109DA960D911D912D913C91DD974017C1
:10C3200051076207730708F074C141155105610593
:10C33000710549F480910E0990910F09A09110099F
:10C34000B09111096DC1F0E0E985842F352F262FBA
:10C35000AA857B856C855D85BE854F859889B09162
:10C36000F21EB89F612D55274091F31E489F600D26
:10C37000511D1090F41E189E500DB39F600D511D5D
:10C38000439F500DB29F500DA62F752FA69FB12D24
:10C3900044279927A59FB00D411D9F1F769FB00D83
:10C3A000411D9F1F759F400D911DA42F792FA69FA2
:10C3B000E12D44279927A59FE00D411D9F1F769FE2
:10C3C000E00D411D9F1F759F400D911DA42F792FDA
:10C3D000BB2780910E0930910F0920911009009020
:10C3E00078080F2A09F484C0409174084A9FB11953
:10C3F0008F0B3F0B2F0B909175089A9FB0198109F5
:10C400003F0B2F0BE0917608EA9F801931092F0B23
:10C41000479FB01981093F0B2F0B979F8019310956
:10C420002F0BE79F30192109A69FE12D442799275B
:10C43000A59FE00D411D9F1F769FE00D411D9F1F91
:10C44000759F400D911DA42F792F409170084A9F30
:10C45000B10D8F1F3F1F2F1F909171089A9FB00D34
:10C46000811D3F1F2F1FE0917208EA9F800D311D33
:10C470002F1F479FB00D811D3F1F2F1F979F800DBE
:10C48000311D2F1FE79F300D211DA69FE12D442751
:10C490009927A59FE00D411D9F1F769FE00D411D2F
:10C4A0009F1F759F400D911DA42F792F40916C08FF
:10C4B0004A9FB1198F0B3F0B2F0B90916D089A9FDC
:10C4C000B01981093F0B2F0BE0916E08EA9F80198C
:10C4D00031092F0B479FB01981093F0B2F0B979FF5
:10C4E000801931092F0BE79F301921090C94FA624A
:10C4F000409174084A9FB10D8F1F3F1F2F1F9091CD
:10C5000075089A9FB00D811D3F1F2F1FE09176087F
:10C51000EA9F800D311D2F1F479FB00D811D3F1FCA
:10C520002F1F979F800D311D2F1FE79F300D211D5D
:10C53000A69FE12D44279927A59FE00D411D9F1F30
:10C54000769FE00D411D9F1F759F400D911DA42FEB
:10C55000792F409170084A9FB1198F0B3F0B2F0B19
:10C56000909171089A9FB01981093F0B2F0BE091B0
:10C570007208EA9F801931092F0B479FB019810972
:10C580003F0B2F0B979F801931092F0BE79F301915
:10C590002109A69FE12D44279927A59FE00D411D64
:10C5A0009F1F769FE00D411D9F1F759F400D911DA0
:10C5B000A42F792F40916C084A9FB10D8F1F3F1F08
:10C5C0002F1F90916D089A9FB00D811D3F1F2F1F47
:10C5D000E0916E08EA9F800D311D2F1F479FB00D1F
:10C5E000811D3F1F2F1F979F800D311D2F1FE79F1C
:10C5F000300D211D1124E987AA877B876C875D8711
:10C60000BE874F87988B90E0932BA0E0B0E0A22BE1
:10C6100007C0A65ABF4F8D919D910D90BC91A02D42
:10C6200025EB37E141E0498BF90145915591659141
:10C630007491481759076A077B0708F48BC399C39D
:10C64000809147098823E1F0FD01E85BFF4F4081BD
:10C65000518160E070E000910A0210910B0220917C
:10C660000C0230910D02401751076207730741F029
:10C6700010920E0210920F021092100210921102EC
:10C6800040910602509107026091080270910902E0
:10C6900077FF5FC0AE5ABF4FCD90DD90ED90FC901C
:10C6A00085EB97E121E0FC014591559165917491ED
:10C6B0004C155D056E057F0550F4F694E794D7940C
:10C6C000C794220F049637E1813D930761F72093C9
:10C6D000490940E2C416D104E104F10428F460E2FF
:10C6E000C62ED12CE12CF12C90E2C91AD108E10818
:10C6F000F108C114A8E0DA06E104F10408F4F5C376
:10C70000B4E0DB9EC00111248B549C4EFC01329698
:10C7100025913491EC2D6627E39FA001E29F410D06
:10C72000561F0694461F561F112460E070E0FC015E
:10C7300025913491C901A0E0B0E0841B950BA60BB4
:10C74000B70B8093060290930702A0930802B09360
:10C750000902C0900602D0900702E0900802F09013
:10C7600009028091471890914818892B09F0E5C17A
:10C770000F941E0F9093481880934718892B09F443
:10C78000DCC1E0914718F0914818808183FF3EC0DA
:10C79000858D968DA78DB0A1418D528D638D748D41
:10C7A000058916892789308D0093561810935718DC
:10C7B000209358183093591840935A1850935B1887
:10C7C00060935C1870935D1880935E1890935F1867
:10C7D000A0936018B093611881A192A1A3A1B4A104
:10C7E0008093621890936318A0936418B0936518AF
:10C7F0009091C1158091C215981709F4B9CF809115
:10C80000C2158F5F8F708093C215B2CFC588D6884E
:10C81000E788F08C81E0C114D104E104F10409F44B
:10C8200080E0018D128D238D348D011511052105B8
:10C83000310509F08260458D568D678D70A14115D7
:10C8400051056105710509F0846080931209109209
:10C850003E0910923F09109240091092410910922E
:10C860004A0910924B0910924C0910924D0985A16A
:10C8700096A1A7A1B0A58093520990935309A093C4
:10C880005409B0935509882499245401881A990AA7
:10C89000AA0ABB0A80922E0990922F09A092300911
:10C8A000B09231098092320990923309A0923409F2
:10C8B000B09235098092360990923709A0923809D2
:10C8C000B092390980923A0990923B09A0923C09B2
:10C8D000B0923D0981A092A0A3A0B4A0880C991C9D
:10C8E000AA1CBB1CCC0CDD1CEE1CFF1CC0921E093C
:10C8F000D0921F09E0922009F0922109000F111F28
:10C90000221F331F00932209109323092093240927
:10C9100030932509440F551F661F771F4093260942
:10C9200050932709609328097093290980922A0956
:10C9300090922B09A0922C09B0922D09880F991F73
:10C94000AA1FBB1F80931A0990931B09A0931C096F
:10C95000B0931D0910925609109257091092580968
:10C960001092590982A593A5A4A5B5A580934E0957
:10C9700090934F09A0935009B093510986A597A5AC
:10C98000A0A9B1A98093430990934409A0934509B4
:10C99000B093460981A580931909909105028917E2
:10C9A00021F01092180910921709DF01A95BBF4FFF
:10C9B0002C9120934809222339F115962D913C9111
:10C9C0001197309316092093150912972D913C91D8
:10C9D0001197309314092093130910920E021092AC
:10C9E0000F02109210021092110212972D913C9199
:10C9F000A90160E070E040930A0250930B0260933B
:10CA00000C0270930D020CC088248A94982C540157
:10CA100080920A0290920B02A0920C02B0920D0238
:10CA2000EA5BFF4F20813091A309231302C08917CD
:10CA300031F02093A309809305020F94EA0E0E941F
:10CA4000ACE92FEF3FEFA9012093060230930702D4
:10CA50004093080250930902E0914718F09148185A
:10CA6000DF01DE96ED90FD900D911C9122A933A976
:10CA700044A955A9EA5AFF4F60817181828193814F
:10CA80000F94980E10924209E0914718F0914818BF
:10CA9000EA5AFF4F80809180A280B38085EB97E1B6
:10CAA00021E0FC0145915591659174914815590516
:10CAB0006A057B0558F4B694A79497948794220F3F
:10CAC0000496A1EDB7E1A817B90759F720934909D2
:10CAD000B0E28B169104A104B10428F4B0E28B2ECD
:10CAE000912CA12CB12C30E2831A9108A108B10835
:10CAF000811448E09406A104B10408F41AC254E079
:10CB0000959EC00111248B549C4EFC0132962591B8
:10CB10003491782D6627739FA001729F410D561F97
:10CB20000694461F561F1124FC01C590D490E12C99
:10CB3000F12CC41AD50AE108F108C0925A09D09222
:10CB40005B09E0925C09F0925D0900915A0910912D
:10CB50005B0920915C0930915D0940910E02509172
:10CB60000F026091100270911102F02E198BF22FBA
:10CB7000E32F401751076207730720F4F42E598BF7
:10CB8000F62FE72F8F2D9989AF2FBE2F0097E1E069
:10CB9000AE07B10520F08FEF9FEFA0E0B0E0081BDB
:10CBA000190B2A0B3B0B00935A0910935B09209336
:10CBB0005C0930935D094F3FFFEF5F076F077F0709
:10CBC00061F0481B590B6A0B7B0B40930E0250938C
:10CBD0000F026093100270931102F8942091840068
:10CBE00030918500205F3F4F4A8941504A8B442352
:10CBF00041F0280E391E2216330610F40C94B05C56
:10CC000001C01901309289002092880078946296C0
:10CC10000FB6F894DEBF0FBECDBFDF91CF911F914D
:10CC20000F91FF90EF90DF90CF90BF90AF909F90CB
:10CC30008F907F906F905F904F903F902F900895CE
:10CC400089898093490990E289169104A104B1046D
:10CC500028F430E2832E912CA12CB12C30E2831ADF
:10CC60009108A108B108811488E09806A104B104D4
:10CC700020F1E4E09E9EC00111248B549C4EFC01E7
:10CC8000329625913491F82DEE27F39F7001F29F93
:10CC9000E10CFE1E0694EE1EFE1E1124FC01C59042
:10CCA000D490860120E030E0480159018E189F0899
:10CCB000A108B1087501640122C09501840136956F
:10CCC000279517950795F801EC7FCF018B54904F6E
:10CCD000FC01C590D490FC01329625913491E82D49
:10CCE000E770E29FC001E39F900D112423E0969529
:10CCF00087952A95E1F7C81AD90AE12CF12C4C0D39
:10CD00005D1D6E1D7F1D40934A0950934B09609332
:10CD10004C0970934D0990914809809147099923D6
:10CD200009F474C0882309F41CCDA85BBF4F8D9112
:10CD30009C91A0E0B0E040910A0250910B026091FA
:10CD40000C0270910D0284179507A607B70709F02A
:10CD500060C007CDB695A795979587954989440FEB
:10CD6000498B2C5F3F4FE1EDF7E1E217F30709F044
:10CD70005BCCD988D092490980329105A105B105D3
:10CD800020F480E290E0A0E0B0E08097A109B10932
:10CD9000811558E09507A105B10508F443C074E07A
:10CDA000979F900111242B543C4EF90132964591E6
:10CDB0005491EE27859FB001849F610D7E1F0694DC
:10CDC0006E1F7E1F1124F901C590D490E12CF12C27
:10CDD000C61AD70AE108F10880913E0990913F09EF
:10CDE000A0914009B09141098C0D9D1DAE1DBF1D44
:10CDF00080933E0990933F09A0934009B093410965
:10CE000080914809811130C080914709882309F435
:10CE1000A8CC10920E0210920F02109210021092E3
:10CE200011029FCCAC01BD0176956795579547954A
:10CE3000FA01EC7F9F012B54304FF901C590D4903B
:10CE4000F9013296459154918770849F9001859F96
:10CE5000300D1124F3E036952795FA95E1F7C21AC3
:10CE6000D30AE12CF12CB8CF8989480E511C611CE2
:10CE7000711C8091471890914818481459046A040D
:10CE80007B04D8F420914709222309F46ACCFC01E1
:10CE9000E85BFF4F20813181A90160E070E00091E3
:10CEA0000A0210910B0220910C0230910D024017E2
:10CEB00051076207730709F454CC10920E021092C6
:10CEC0000F021092100210921102FC01E85BFF4F5A
:10CED00080819181A0E0B0E080930A0290930B02E0
:10CEE000A0930C02B0930D023CCCD701C601B695BD
:10CEF000A79597958795FC01EC7FCF018B54904FB8
:10CF0000FC0125913491FC013296459154916C2D90
:10CF10006770649FC001659F900D112453E0969542
:10CF200087955A95E1F7281B390BC901A0E0B0E0BD
:10CF300008CCD501C401B695A79597958795FC01B6
:10CF4000EC7FCF018B54904FFC01C590D490FC0135
:10CF5000329625913491482D4770429FC001439FDE
:10CF6000900D1124A3E096958795AA95E1F7C81A2C
:10CF7000D90AE12CF12CE1CD80EDC82E87E0D82E26
:10CF8000E12CF12CF5CBEF92FF920F931F93CF93EF
:10CF90007C018B014F3F11F4C2E401C0C4E580E283
:10CFA0000E942A548C2F0E942A548AE30E942A54F9
:10CFB000F701608171818281938142E00E94BA54BD
:10CFC000F80140815181628173818AEC99E10F946B
:10CFD0001B1762E070E080E090E0CF911F910F910D
:10CFE000FF90EF900D94A81F6091670970916809F8
:10CFF000072E000C880B990B0F941F3020916309AA
:10D000003091640940916509509166090F946E3919
:10D0100018161CF086ED99E102C081EE99E19F930C
:10D020008F938CEE99E19F938F931F920E9463FDE3
:10D030000F900F900F900F900F9008951F93CF9324
:10D04000DF93CDB7DEB728970FB6F894DEBF0FBEDB
:10D05000CDBF182F6091670970916809072E000CE9
:10D06000880B990B0F941F306D837E838F83988775
:10D0700020E030E0A901609163097091640980911A
:10D080006509909166090F940E3769837A838B83C3
:10D090009C834CEFBE016B5F7F4FCE0101960E94D7
:10D0A000C36760917E0970917F09072E000C880B81
:10D0B000990B0F941F306D837E838F8398878091A7
:10D0C0007A0990917B09A0917C09B0917D098983AF
:10D0D0009A83AB83BC834FEFBE016B5F7F4FCE0162
:10D0E00001960E94C3671F3F19F46091800907C031
:10D0F00087E11802F0011124E15AF64F628570E0D1
:10D1000082ED99E10F942C176091800970E08DEC0D
:10D1100099E10F942C1728960FB6F894DEBF0FBE36
:10D12000CDBFDF91CF911F9108952F923F924F92E3
:10D130005F926F927F928F929F92AF92BF92CF92A7
:10D14000DF92EF92FF920F931F93CF93DF93CDB7B0
:10D15000DEB763970FB6F894DEBF0FBECDBF898BE5
:10D1600081E0809321021A821B821C821D82198613
:10D170001A861B861C8619821D862CE32E873CE1AD
:10D180003F8746E4488B312C212C50E85A8B8FEB9B
:10D190008B8B91E09887812C912C540160917E09B2
:10D1A00070917F09072E000C880B990B0F941F308C
:10D1B0007B018C019B01AC01632D722D8A899B89B7
:10D1C0000F941830882361F160917A0970917B097E
:10D1D00080917C0990917D09A989A1110EC0B1E0CF
:10D1E000B9839701A8010F946E3918160CF01982B3
:10D1F0003E2C2F2C0A8B1B8B13C09701A8010F9478
:10D200006E39181644F480912102882309F4F1C084
:10D210000F94D21AEEC03E2C2F2C0A8B1B8B198236
:10D220000F94E21F6B017C01DC01CB0129853A855B
:10D230004B855C85821B930BA40BB50BB7FD34C0EB
:10D24000D701C60188519C4FAF4FBF4F89879A873E
:10D25000AB87BC878091B80D0E941E6885EF99E16D
:10D260000F94671681149104A104B104B9F0D5019B
:10D27000C401805F984DAF4FBF4FBC01CD016C1909
:10D280007D098E099F0928EE33E040E050E00F94BD
:10D290006E36CA01B9010E949E5403C08FE30E94FA
:10D2A0002A548AE00E942A5480E00E9456550F9426
:10D2B000E21F6093F2137093F3138093F41390932F
:10D2C000F51390917A099E83A0917B09AF83009119
:10D2D0007C0910917D09292F3A2FA801632D722D09
:10D2E0008A899B890F940D372B013C0120E030E0A7
:10D2F000A9010F946E3987FF04C077FA709477F80C
:10D30000709481149104A104B104B1F420E030E0E0
:10D3100040E85FE3C301B2010F94183087FF18C0E3
:10D32000B88546015701BB2399F020E1820E27E220
:10D33000921EA11CB11C0CC020E030E040E450E47F
:10D34000C301B2010F946E39181614F44601570147
:10D3500039813323A9F18A819B81AC81BD81892BDD
:10D360008A2B8B2B61F0D701C6012A813B814C812E
:10D370005D81821B930BA40BB50BB7FD21C02E81E1
:10D380003F81A8016D857E858F8598890F940D3723
:10D3900020E030E040EC5FE30F94183087FD33CF9E
:10D3A000D701C601805A9541AF4FBF4F8A839B83F7
:10D3B000AC83BD839E819D87AF81AE870F87188B1D
:10D3C00080912102882309F41ECF81149104A104C5
:10D3D000B10411F41886E2CEB0E1CB1AB7E2DB0A51
:10D3E000E108F108C818D908EA08FB08F7FCF2CFF1
:10D3F0000ACF8091210263960FB6F894DEBF0FBE6C
:10D40000CDBFDF91CF911F910F91FF90EF90DF90F3
:10D41000CF90BF90AF909F908F907F906F905F90D4
:10D420004F903F902F9008952F923F924F925F928E
:10D430006F927F928F929F92AF92BF92CF92DF9224
:10D44000EF92FF920F931F93CF93DF93CDB7DEB789
:10D4500064970FB6F894DEBF0FBECDBF898B6A8B81
:10D4600081E0809321021A821B821C821D82198610
:10D470001A861B861C8621E0288719821D863CE3BC
:10D480003E874CE14F8756E4588B312C212C80E8A5
:10D490008B8B9FEB9C8B812C912C540160916709A5
:10D4A00070916809072E000C880B990B0F941F30A0
:10D4B0007B018C019B01AC01632D722D8B899C89B2
:10D4C0000F941830882361F16091630970916409A9
:10D4D0008091650990916609AA89A1110EC0B1E0F9
:10D4E000B9839701A8010F946E3918160CF01982B0
:10D4F0003E2C2F2C0B8B1C8B13C09701A8010F9473
:10D500006E39181644F480912102882309F4F2C080
:10D510000F94D21AEFC03E2C2F2C0B8B1C8B198230
:10D520000F94E21F6B017C01DC01CB0129853A8558
:10D530004B855C85821B930BA40BB50BB7FD33C0E9
:10D54000D701C60188519C4FAF4FBF4F89879A873B
:10D55000AB87BC8789890E941E6881EF99E10F948F
:10D56000671681149104A104B104B9F0D501C40176
:10D57000805F984DAF4FBF4FBC01CD016C197D0945
:10D580008E099F0928EE33E040E050E00F946E369C
:10D59000CA01B9010E949E5403C08FE30E942A541D
:10D5A0008AE00E942A5480E00E9456550F94E21FA0
:10D5B0006093F2137093F3138093F4139093F51325
:10D5C00020E030E0A90160916309709164098091C5
:10D5D0006509909166090F940E376E837F838C01E5
:10D5E0009B01AC01632D722D8B899C890F940D37A3
:10D5F0002B013C0120E030E0A9010F946E3987FF38
:10D6000004C077FA709477F8709481149104A1049F
:10D61000B104B1F420E030E040E85FE3C301B201BF
:10D620000F94183087FF18C0988546015701992339
:10D6300099F0A0E18A0EA7E29A1EA11CB11C0CC0B1
:10D6400020E030E040E450E4C301B2010F946E39B1
:10D65000181614F446015701B981BB2391F12A81B0
:10D660003B814C815D81211531054105510541F01A
:10D67000D701C601821B930BA40BB50BB7FD21C0CC
:10D680002E813F81A8016D857E858F8598890F94B5
:10D690000D3720E030E040EC5FE30F94183087FD59
:10D6A00032CFD701C601805A9541AF4FBF4F8A8311
:10D6B0009B83AC83BD839E819D87AF81AE870F879F
:10D6C000188B80912102882309F41DCF81149104C5
:10D6D000A104B10411F41886E1CEB0E1CB1AB7E28F
:10D6E000DB0AE108F108C818D908EA08FB08F7FCCA
:10D6F000F2CF09CF8091210264960FB6F894DEBF75
:10D700000FBECDBFDF91CF911F910F91FF90EF9092
:10D71000DF90CF90BF90AF909F908F907F906F9051
:10D720005F904F903F902F9008952F923F924F928D
:10D730005F926F927F928F929F92AF92BF92CF92A1
:10D74000DF92EF92FF920F931F93CF93DF93CDB7AA
:10D75000DEB72A970FB6F894DEBF0FBECDBFF82E06
:10D76000762E0E948CFF81E08F1598F40F9450174D
:10D7700084E50E942A546F2D70E080E090E00E94C2
:10D780009E5480E20E942A5489EF99E10F94671613
:10D790000DC2711008C08091AE0D8770772473940C
:10D7A000873009F4712C9090B80D81E08725898726
:10D7B000882389F08824839420E030E0A9016091D7
:10D7C000A30B7091A40B8091A50B9091A60B0F94C5
:10D7D0001830811101C0812C8091A20B83FD69C199
:10D7E0008091A10B811165C1209167093091680971
:10D7F0008091420290914302281739070CF059C1D9
:10D80000882049F00F9450178DE19AE10F94671624
:10D81000F092B80DCBC1662463948091D10D8A87B4
:10D8200080E00E9447D2F91409F431C120905B02D4
:10D8300030905C0240905D0250905E0280915702F1
:10D8400090915802A0915902B0915A0280935B02C4
:10D8500090935C02A0935D02B0935E0280E00E9410
:10D8600060C781E00E9460C782E00E9460C780E1DB
:10D87000E9EBFDE0A5E8BDE001900D928A95E1F7A6
:10D880008985882309F472C02091B70B3091B80BB9
:10D890004091B90B5091BA0B6091C10D7091C20DBE
:10D8A0008091C30D9091C40D0F940E376093C10DFC
:10D8B0007093C20D8093C30D9093C40DA0903E024F
:10D8C000B0903F02C0904002D0904102A601950165
:10D8D0000F946E39181644F4A092C10DB092C20D87
:10D8E000C092C30DD092C40D80917F0B9091800B9C
:10D8F000A091810BB091820B89839A83AB83BC8307
:10D90000CE0101960E9424C88091B30B9091B40B74
:10D91000A091B50BB091B60B4091AF0B5091B00BED
:10D920006091B10B7091B20B4093B90D5093BA0D49
:10D930006093BB0D7093BC0D8093BD0D9093BE0D95
:10D94000A093BF0DB093C00DA12CB12C6501E92CA3
:10D950000BE512E025EC3DE041EC5DE06DEB7DE098
:10D9600089EB9DE00F9427020E948CFFF092B80D86
:10D9700020E030E0A9016091B90D7091BA0D80915D
:10D98000BB0D9091BC0D0F940E376093B90D709341
:10D99000BA0D8093BB0D9093BC0D20E030E0A9013F
:10D9A0006091BD0D7091BE0D8091BF0D9091C00D25
:10D9B0000F940E376093BD0D7093BE0D8093BF0D15
:10D9C0009093C00D20E030E0A9016091C10D7091ED
:10D9D000C20D8091C30D9091C40D0F940E376093CA
:10D9E000C10D7093C20D8093C30D9093C40D0E941E
:10D9F000D9C9711044C080912902882309F43FC01D
:10DA0000892D90E0FC01E156F44F2091B00D208368
:10DA10006F2D70E0FB01E156F44F20812093B00D93
:10DA20002091670930916809880F991FFC01E5561C
:10DA3000F44F31832083660F771FFB01E556F44FC7
:10DA400080819181009761F02817390749F00E9481
:10DA5000A4A180E00E94F46760E080E00E94146A64
:10DA6000811053C085E89DE00E94DFC3898588232B
:10DA700031F06FE77BE08DE89DE00E9426C920929F
:10DA80005B0230925C0240925D0250925E020E9404
:10DA90008CFF0F9450176091B80D70E08BE09AE105
:10DAA0000F942C178AE00E942A548A850E9447D23C
:10DAB0007DC0882041F16091AD0B7091AE0B072EB7
:10DAC000000C880B990B0F941F3020E030E040E7EA
:10DAD00052E40F9408386D837E838F8398878091FA
:10DAE000A30B9091A40BA091A50BB091A60BB058DD
:10DAF00089839A83AB83BC83BE016B5F7F4FCE016A
:10DB000001960E9492CC612C88CE6110ABCF6091BF
:10DB1000AB0B7091AC0B072E000C880B990B0F947C
:10DB20001F3020E030E040E752E40F94083869836A
:10DB30007A838B839C83BE016F5F7F4F83EA9BE078
:10DB40000E9492CC80E090E0A0E4B0E489839A83C4
:10DB5000AB83BC83BE016F5F7F4F87EA9BE00E946F
:10DB600092CC0E948CFF20E030E040E050E46091D5
:10DB7000C50D7091C60D8091C70D9091C80D0F9481
:10DB80000D376093C50D7093C60D8093C70D9093AC
:10DB9000C80D6093910D7093920D8093930D9093A7
:10DBA000940D81E99DE00E949DFF5CCF2A960FB6FF
:10DBB000F894DEBF0FBECDBFDF91CF911F910F91C3
:10DBC000FF90EF90DF90CF90BF90AF909F908F909D
:10DBD0007F906F905F904F903F902F900895EF92BD
:10DBE000FF920F931F93CF93DF93809128028F377B
:10DBF000A0F08F57909169099093C90B992311F068
:10DC00002C9A01C02C98209180092093C80B9091E8
:10DC10000201222369F090950BC09091C90B8917DE
:10DC200008F02C989091C80B891728F09091020168
:10DC30009072909300018F5F809328029091C70BA0
:10DC400081E089278093C70B8091270285301CF4DF
:10DC500011E0180F01C010E0823009F4B9C054F48B
:10DC6000882301F1813009F0E8C088E080937B00CF
:10DC700085E4C5C0843009F4CAC00CF4BCC085304A
:10DC800009F0DBC09091C60B911102C08093C60BC6
:10DC90008091C60B81508093C60B882309F4CDC0B8
:10DCA00015E0CBC0809126028F5F80311CF48093F9
:10DCB0002602C3C01092260280914F0B811113C01F
:10DCC00080915F0990916009909362098093610946
:10DCD00080917609909177099093790980937809DA
:10DCE00081E080934F0B1092600910925F091092AF
:10DCF000770910927609E0906109F0906209F19439
:10DD0000E194F108809167099091680901E0181683
:10DD100019062CF080916909811101C000E0809101
:10DD20001B0290911C029195819591098E159F057A
:10DD30003CF44AE359E16BE579E180E00F94840912
:10DD4000002389F08091190290911A029195819592
:10DD50009109E816F9063CF44DE659E16EE879E1DF
:10DD600080E00F94840980917E0990917F0901E001
:10DD7000181619062CF080918009811101C000E06D
:10DD8000209178093091790980918E0990918F09BD
:10DD9000821793073CF04AE459E16BE579E18FEF94
:10DDA0000F948409002309F448C020917809309128
:10DDB0007909809117029091180228173907ECF120
:10DDC0004DE759E16EE879E18FEF0F94840935C092
:10DDD00080917A0086FD2EC0809178009091790024
:10DDE00020915F0930916009820F931F9093600921
:10DDF00080935F0922C088E080937B0086E4809353
:10DE00007C0080917A00806480937A0016C08091B3
:10DE10007A0086FD11C08091780090917900209160
:10DE2000760930917709820F931F90937709809339
:10DE3000760903C012E001C014E01093270220917C
:10DE4000F6133091F7132115310509F43DC0F8940C
:10DE50009091090192708091080181708093060170
:10DE600000000000000080910B01121613060CF058
:10DE7000809582708093090100000000000080916D
:10DE80000B01809588708093090184E08A950000D9
:10DE9000E9F780910B0188708093090180910B0153
:10DEA0009111809582708093090178948091F61386
:10DEB0009091F7131216130614F4019701C00196FE
:10DEC0009093F7138093F6138091500B882309F4F5
:10DED0004DC0809125028E5F8F778093250281113E
:10DEE00045C08CB185FB882780F9C82F80E0D82FEA
:10DEF0008091030181FDC2604B99C4600091C40B05
:10DF00001091C50B0C271D270115110579F100FF94
:10DF100007C0BE016170772785EB99E10F942C173C
:10DF200001FF08C06C2F6695617070E08CEA99E182
:10DF30000F942C1702FF08C0C2FB662760F970E03F
:10DF400083EA99E10F942C1780EA99E10F94671600
:10DF50001091C30B612F70E08DE00F94C01E1095DF
:10DF60001093C30BD093C50BC093C40B0E94ACE9B4
:10DF70008091510B9091520B009769F0019790930B
:10DF8000520B8093510B892B31F48EEB99E19093D6
:10DF9000B3098093B209DF91CF911F910F91FF9048
:10DFA000EF9008950F930FB70F9300916E000B7FC2
:10DFB00000936E0078940F930BB70F930CB70F92EA
:10DFC0001F922F933F934F935F936F937F938F9302
:10DFD0009F93AF93BF93EF93FF9311240E94EF6D34
:10DFE000FF91EF91BF91AF919F918F917F916F9131
:10DFF0005F914F913F912F911F900F900CBF0F9108
:10E000000BBF0F910460F89400936E000F910FBF47
:10E010000F9118952F923F924F925F926F927F923D
:10E020008F929F92AF92BF92CF92DF92EF92FF9228
:10E030000F931F93CF93DF93CDB7DEB729970FB61A
:10E04000F894DEBF0FBECDBF1C017B836A8329839A
:10E050001F830E83FD82EC8227FD10C0022E000C70
:10E06000330B39872887398185E03802F001112484
:10E07000E75BF44F84818823E1F008C08091480B6E
:10E08000882399F0E1E0F0E0F987E887F101148254
:10E09000E885F985EE0FFF1FEE0FFF1FE554F44FE3
:10E0A00010821182128213822EC021E030E0398763
:10E0B0002887FA01C080D180E280F3800885198525
:10E0C000000F111F000F111F0554144FA7019601D7
:10E0D000F80160817181828193810F9418308823C7
:10E0E00091F0F801C082D182E282F38211E020E057
:10E0F00030E0A901C701B6010F946E3918160CF073
:10E1000010E0F1011483F10184818230F9F0833051
:10E1100009F401C1813009F023C1E885F985EE0FCA
:10E12000FF1FEE0FFF1FE554F44F20813181428124
:10E130005381EA81FB8160817181828193810F9497
:10E14000183087FD0DC182E0F101848380912402A3
:10E15000882309F493C0F981F7FD90C08F2FFF0F3A
:10E16000990B8C011816190614F401E010E0F8015F
:10E17000E055F24F2081222371F1EA81FB81C080BA
:10E18000D180E280F380880F991F880F991FFC01CE
:10E19000E554F44F80809180A280B3802C813D8132
:10E1A000B90180E090E00F941D302B013C0120E08C
:10E1B00030E040E85EE30F947E309B01AC01C50186
:10E1C000B4010F940D379B01AC01C701B6010F9448
:10E1D0006E3987FD05C0F801EE5DFD4F80E81AC07D
:10E1E00023E830EC4AEA5EE3C301B2010F947E30CB
:10E1F0009B01AC01C501B4010F940D379B01AC012B
:10E20000C701B6010F946E390E5D1D4F87FD04C026
:10E2100080E6F801808332C020E030E040E05FE338
:10E22000C301B2010F947E309B01AC01C501B40162
:10E230000F940D379B01AC01C701B6010F946E39E5
:10E2400087FD02C080E4E5CF2DEC3CEC4CE45FE3BD
:10E25000C301B2010F947E309B01AC01C501B40132
:10E260000F940D379B01AC01C701B6010F946E39B5
:10E2700087FD02C080E2CDCFF801108208851985A4
:10E28000000F111F000F111F98012554344F3987BB
:10E290002887EC81FD81BF0180E090E00F941D3064
:10E2A0009B01AC01E885F985608171818281938150
:10E2B0000F940D379B01AC01EA81FB816081718174
:10E2C000828193810F946E3987FD14C00F94E21FF1
:10E2D0006B017C012E813F81A8EEB3E00F94C23622
:10E2E000C60ED71EE81EF91EF101C082D182E2825D
:10E2F000F38236C00F94E21FF10100811181228167
:10E300003381DC01CB01801B910BA20BB30BB7FD5A
:10E3100027C083E08483F981FF3F19F043E059E18E
:10E3200002C046E159E16AE279E1898129960FB696
:10E33000F894DEBF0FBECDBFDF91CF911F910F913B
:10E34000FF90EF90DF90CF90BF90AF909F908F9015
:10E350007F906F905F904F903F902F900D94840925
:10E3600029960FB6F894DEBF0FBECDBFDF91CF91D7
:10E370001F910F91FF90EF90DF90CF90BF90AF90E3
:10E380009F908F907F906F905F904F903F902F90D5
:10E390000895CF92DF92EF92FF9260917E09709183
:10E3A0007F0961157105C1F0C0907A09D0907B0991
:10E3B000E0907C09F0907D0966507109072E000CF1
:10E3C000880B990B0F941F309B01AC01C701B6015C
:10E3D0000F94183087FD09C01092400B1092410B2A
:10E3E0001092420B1092430B1EC020E030E040E040
:10E3F00050E4C701B6010F940E370F948138709323
:10E400003F0B60933E0B0F94E21FDC01CB01805E5B
:10E410009044AD4FBF4F8093400B9093410BA0931E
:10E42000420BB093430BFF90EF90DF90CF90089595
:10E43000CF93DF9310924E0B80E090E00E94A4A156
:10E44000C6E7D9E0198618860E94C97180E090E07D
:10E450000E94A4A1109269092C98198618861A8620
:10E4600080910201807280930001DF91CF91089525
:10E47000CF92DF92EF92FF92CF93DF93C091670923
:10E48000D0916809209701F120E030E0A901609166
:10E4900063097091640980916509909166090F94F0
:10E4A0000E376B017C01BE0166507109072E000C0E
:10E4B000880B990B0F941F309B01AC01C701B6016B
:10E4C0000F94183087FD09C010923A0B10923B0B45
:10E4D00010923C0B10923D0B1EC020E030E040E05B
:10E4E00050E4C701B6010F940E370F948138709332
:10E4F000390B6093380B0F94E21FDC01CB01805B7A
:10E500009C43AF4FBF4F80933A0B90933B0BA0932C
:10E510003C0BB0933D0BDF91CF91FF90EF90DF90DC
:10E52000CF900895CF93DF93CFE5D9E060E08A8163
:10E530009B810F9497086C837D838E839F83C6E7AE
:10E54000D9E08A819B810F94FE076C837D838E8343
:10E550009F83A89510924F0BDF91CF910895CF9292
:10E56000DF92EF92FF920F931F93CF93DF936C0193
:10E570007A018B01C0E0D0E0CE15DF0581F0D80133
:10E580006D918D01D601ED91FC910190F081E02D0E
:10E59000C6011995892B11F02196EECF7E01C70196
:10E5A000DF91CF911F910F91FF90EF90DF90CF906F
:10E5B0000895089580E090E00895FC01538D448D06
:10E5C000252F30E0842F90E0821B930B541710F01E
:10E5D000CF96089501970895FC01918D828D98172B
:10E5E00061F0828DDF01A80FB11D5D968C91928D37
:10E5F0009F5F9F73928F90E008958FEF9FEF089534
:10E60000FC01918D828D981731F0828DE80FF11DFC
:10E61000858D90E008958FEF9FEF0895FC01918D17
:10E62000228D892F90E0805C9F4F821B91098F7310
:10E63000992708958DE394E10E940E7321E0892BC0
:10E6400009F420E0822F0895FC01848DDF01A80FDA
:10E65000B11DA35ABF4F2C91848D90E001968F730A
:10E660009927848FA689B7892C93A089B1898C9129
:10E67000837080648C93938D848D981306C0028878
:10E68000F389E02D80818F7D80830895EF92FF9242
:10E690000F931F93CF93DF93EC0181E0888F9B8DC5
:10E6A0008C8D981305C0E889F989808185FD26C085
:10E6B000F62E0B8D10E00F5F1F4F0F731127E02E0A
:10E6C0008C8DE8120CC00FB607FCFACFE889F989E7
:10E6D000808185FFF5CFCE010E942473F1CF8B8D11
:10E6E000FE01E80FF11DE35AFF4FF0829FB7F89447
:10E6F0000B8FEA89FB89808180620AC09FB7F894FA
:10E70000EE89FF896083E889F9898081837080645C
:10E7100080839FBF81E090E0DF91CF911F910F91A7
:10E72000FF90EF900895CF93DF93EC01888D8823BD
:10E73000C9F0EA89FB89808185FD05C0A889B9896E
:10E740008C9186FD0FC00FB607FCF5CF808185FF49
:10E75000F2CFA889B9898C9185FFEDCFCE010E94B7
:10E760002473E7CFDF91CF91089580E090E0892B6B
:10E7700041F080E090E0892B21F00E94000081119F
:10E7800021C080E090E0892B41F080E090E0892B6F
:10E7900021F00E940000811118C080E090E0892BD8
:10E7A00021F00E941A73811113C080E090E0892B40
:10E7B000A1F080E090E0892B81F00E94000081119F
:10E7C0000AC008950E940000DCCF0E940000E5CF3F
:10E7D0000E940000EACF0C94000008950F94203AA4
:10E7E000CF93DF93EC01CB01E881F98160817181E6
:10E7F0000E944A9A88819981DC01ED91FC912081E7
:10E80000AA81BB81222369F02C91293650F43196DC
:10E81000DC01ED93FC93EA81FB8180818F5F808333
:10E82000E9CF8C91893670F48FE28083E881F98199
:10E8300080819181019691838083EA81FB8180812F
:10E840008F5F8083DF91CF9108951F920F920FB653
:10E850000F9211240BB60F922F933F934F935F9318
:10E860006F937F938F939F93AF93BF93EF93FF9398
:10E870008DE394E10E942473FF91EF91BF91AF91DA
:10E880009F918F917F916F915F914F913F912F91C8
:10E890000F900BBE0F900FBE0F901F9018951F92F8
:10E8A0000F920FB60F9211240BB60F922F938F93E6
:10E8B0009F93EF93FF93E0914D14F0914E1480815C
:10E8C000E0915314F091541482FD12C09081809114
:10E8D00056148F5F8F7320915714821751F0E09177
:10E8E0005614F0E0E35CFB4E958F8093561401C004
:10E8F0008081FF91EF919F918F912F910F900BBE8F
:10E900000F900FBE0F901F9018958BE1E3E3F5E198
:10E91000A8E1B5E101900D928A95E1F78091EB179E
:10E9200080628093EB1708958091EB1782FF1FC0E0
:10E9300089E89BE10F9467166091E7177091E817DB
:10E940008091E9179091EA174AE00E9431548FE2D2
:10E950000E942A546091E3177091E4178091E517A3
:10E960009091E6174AE00E9431540C942F558BE9A0
:10E970009BE10D9467161092CA0B8091EB178F7B69
:10E980008B7F8093EB170E94CA51882321F08AED78
:10E9900094E10C94B09C08958091EB1783FF03C021
:10E9A00084608093EB170895CF92DF92EF92FF92ED
:10E9B0000F931F93CF93DF93CDB7DEB7EDB6FEB6BF
:10E9C000DC010D900020E9F79D01281B390B2C5F1D
:10E9D0003F4F4DB75EB7421B530B0FB6F8945EBF67
:10E9E0000FBE4DBF0DB71EB70F5F1F4F9F938F9385
:10E9F00085E89AE19F938F931F930F930F94B02F05
:10EA0000680154E0C50ED11C0F900F900F900F902D
:10EA10000F900F90F6018081882349F0082E000C9A
:10EA2000990B0F94253AF60181936F01F3CFC8013A
:10EA30000E94A9F081E89AE10E94C5AB0FB6F89454
:10EA4000FEBE0FBEEDBEDF91CF911F910F91FF90E3
:10EA5000EF90DF90CF9008958F929F92AF92BF92E8
:10EA6000CF92DF92EF92FF92CF938091EB17877F47
:10EA70008093EB1780913615882321F083E395E18D
:10EA80000E94B09C109217151092141585E3809384
:10EA900013150F94E21F6B017C0120EDC20E27E0DD
:10EAA000D21EE11CF11CA89561E0809113150E9413
:10EAB000DBE161E0809113150E940AE2209A289A16
:10EAC000219A2398229A81E00E947B5C85E08093C2
:10EAD00015150E947B5CCAE08FEF0E946F5CC150ED
:10EAE000D9F7A89520E030E0A90160E083E195E145
:10EAF0000E94909B80931615813061F00F94E21F65
:10EB0000DC01CB018C199D09AE09BF09B7FDEACF25
:10EB100081E062C0A8952AEA31E040E050E068E078
:10EB200083E195E10E94909B853011F481E00AC059
:10EB3000C4E00E94745C80931615C150D1F78A3AE4
:10EB400061F482E080931715A895809117158230A3
:10EB500081F0812C912C540111C00F94E21FDC0133
:10EB6000CB018C199D09AE09BF09B7FDD4CF82E056
:10EB700033C0812C912CA12C80E4B82E20E030E011
:10EB8000A90167E383E195E10E94909BA5019401AF
:10EB900069E283E195E10E94909B8093161588239A
:10EBA00061F00F94E21FDC01CB018C199D09AE09C5
:10EBB000BF09B7FDE3CF8AE00FC0809117158230FF
:10EBC00021F520E030E0A9016AE383E195E10E94AC
:10EBD000909B882361F088E08093141583E195E190
:10EBE0000E94889B0F94501783E79AE122C00E94ED
:10EBF000745C807C803C19F483E0809317150E943C
:10EC0000745C0E94745C0E94745C83E195E10E94D4
:10EC1000889B1092151581E00E9461DC81110CC067
:10EC200080E00E9461DC811107C00F944C178FE5D2
:10EC30009AE10F9467161AC065EF74E183E395E1DA
:10EC40000E94DB99811105C00F944C178EE49AE164
:10EC5000F0CF8091EB1788608093EB170F945017DB
:10EC600082E49AE10F9467160E94BE51CF91FF9003
:10EC7000EF90DF90CF90BF90AF909F908F900C94CB
:10EC80008574FC0180818823E1F0853ED1F08E32CD
:10EC9000C1F08091E10F8E32A1F09385892F8A70A7
:10ECA00081F4987121E0903109F020E08091EB1718
:10ECB00020FB84F98093EB17903141F080858734F5
:10ECC00011F080E0089581858E37D9F381E00895B1
:10ECD0000F931F93CF93DF93CDB7DEB7EB970FB6AC
:10ECE000F894DEBF0FBECDBF88E195E10E94839B03
:10ECF0008BE1E8E1F5E1DE01919601900D928A95B4
:10ED0000E1F700E010E041EE5FE0BE016F5F7F4F92
:10ED1000CE0181960E94459E18163CF4CE010196C4
:10ED20000E944176080F111DEECFCE0181960E9400
:10ED3000B99CC801EB960FB6F894DEBF0FBECDBFED
:10ED4000DF91CF911F910F910895FC0120E03EE2E9
:10ED5000DB014C91403241F0283011F43083319680
:10ED6000DB014C91408331962F5F6F5F7F4F2B30DB
:10ED700079F7108208956F927F928F929F92AF924F
:10ED8000BF92CF92DF92EF92FF920F931F93CF9398
:10ED9000DF93CDB7DEB7C356D1090FB6F894DEBF07
:10EDA0000FBECDBF5C018B016DB67EB67E0187E5DF
:10EDB000E80EF11C41EE5FE0BE016F5F7F4FC501C1
:10EDC0000E94459E18160CF0AFC08C85887180316A
:10EDD00009F06CC08DB69EB6BE016F5F7F4FC70154
:10EDE0000E94A5760115110521F0F801808181119D
:10EDF00091C021E081E090E0F70101900020E9F767
:10EE00003197EE19FF09E80FF91F32968DB79EB7BB
:10EE10008E1B9F0B0FB6F8949EBF0FBE8DBFEDB734
:10EE2000FEB731966F01211102C0B80102C066EA37
:10EE300076E0C6010F946C3AB701C6010F94563ABA
:10EE400066EA76E0C6010F94563A19A21CA221E0A8
:10EE5000A701B501CE0181960E94B3A081110AC01D
:10EE60000F945017B7018EE29AE10F9439178AE098
:10EE70000E942A548BE1FE01B196DE01DC960190DE
:10EE80000D928A95E1F7B601CE01CC960E94BB7631
:10EE9000CE01CC960E94B99CCE0181960E94B99C6D
:10EEA0000FB6F8949EBE0FBE8DBE84CFCE010196E4
:10EEB0000E944176882309F47DCFBE016F5F7F4FAA
:10EEC00083E290E10E94A5760115110529F483E201
:10EED000C82E80E1D82E09C06801F60181916F012A
:10EEE0008823A9F30E942A54F8CFF60181916F017B
:10EEF000882319F00E942A54F8CF80E20E942A54F5
:10EF00006D8D7E8D8F8D98A14AE00E9431540E94B4
:10EF10002F5550CFF80101900020E9F73197CF012C
:10EF2000801B910B20E068CF0FB6F8947EBE0FBE19
:10EF30006DBECD59DF4F0FB6F894DEBF0FBECDBF0B
:10EF4000DF91CF911F910F91FF90EF90DF90CF90C5
:10EF5000BF90AF909F908F907F906F900895EF92A9
:10EF6000FF920F931F93CF93DF93CDB7DEB7A09798
:10EF70000FB6F894DEBF0FBECDBF7C018B0141EE12
:10EF80005FE0BE016F5F7F4FC7010E94459E18166C
:10EF9000A4F4CE0101960E944176882381F3BE013C
:10EFA0006F5F7F4F83E290E10E94A57663E270E19C
:10EFB000C8010F94433A892B11F7A0960FB6F89425
:10EFC000DEBF0FBECDBFDF91CF911F910F91FF909C
:10EFD000EF9008950F931F93CF93DF93CDB7DEB7D4
:10EFE0006B970FB6F894DEBF0FBECDBF8C0188E1E2
:10EFF00095E10E94839B8BE1E8E1F5E1DE0111964A
:10F0000001900D928A95E1F7B801CE0101960E9418
:10F01000AF77CE0101960E94B99C6B960FB6F8941B
:10F02000DEBF0FBECDBFDF91CF911F910F9108952D
:10F03000DF92EF92FF920F931F93CF93DF93CDB7A1
:10F04000DEB727970FB6F894DEBF0FBECDBF209175
:10F05000EB1723FF37C1F42EE62E8C010E94CA5114
:10F06000882309F480C0FF2009F48BC08091E21747
:10F07000882351F00F944C1784E49BE10F9467169A
:10F0800080E090E00E9414FB80ED9BE09E838D83E6
:10F090008FE28093CF0B81E08F83CE0105969A8318
:10F0A000898302969C838B83F12C9BE1D92E8091DE
:10F0B000E117F81658F4DF9CB00111246D52794E17
:10F0C000CE0101960E94F073F394F1CF8F818B35BE
:10F0D00058F46AED74E1CE0101960E94F0738D81BF
:10F0E0009E8101979E838D83ED81FE811082E09148
:10F0F000E21784E0E89FF0011124E553F44F80917A
:10F10000E7179091E817A091E917B091EA1780836B
:10F110009183A283B3830F945017B8018BE29BE1D4
:10F120000F9439176091E21789E6689FB0011124A6
:10F130006153744F80E29BE10F9439174091E717B8
:10F140005091E8176091E9177091EA178AE19BE105
:10F150000F94FD168AE00E942A548091E2178F5F77
:10F160008093E21726C0FF2039F00F9450178AE0F1
:10F170009BE10F9467161DC01092E21782E0F82EF3
:10F1800002C0FF24F3940F94501785E09BE10F9485
:10F19000671681E0F81609F492C081EF9AE10F94A6
:10F1A0006716B8018DEF9AE10F9439178AE00E9433
:10F1B0002A540E94BB74B801CE0101960E947BFCC8
:10F1C0008C01009709F47EC069817A81EE2009F4F0
:10F1D0004DC021E0AC018AED94E10E94B3A08823E8
:10F1E000E9F18091EB149091EC14A091ED14B091A1
:10F1F000EE148093E3179093E417A093E517B09370
:10F20000E6171092E7171092E8171092E91710927C
:10F21000EA17B80183EE9AE10F9439174091E3178A
:10F220005091E4176091E5177091E6178BED9AE124
:10F230000F94FD168AE00E942A548CEC9AE10F94F8
:10F240006716C8010E94EA778091E10F811102C020
:10F25000C80102C081EE9FE060E02EC0B80188EBDB
:10F260009AE10F94391785EB9AE10FC026E5AC01BE
:10F270008AED94E10E94B3A081110AC0B80181EA2D
:10F280009AE10F9439178EE99AE10F9467161AC024
:10F290008091EB1781608093EB17C8010E94EA7799
:10F2A0001092D116B8018CE89AE10F9439178AE0D0
:10F2B0000E942A5460E0C8010F94A91A03C087EF86
:10F2C0009AE16DCF27960FB6F894DEBF0FBECDBF83
:10F2D000DF91CF911F910F91FF90EF90DF900895F4
:10F2E000CF92DF92EF92FF92CF936B017C01C42FFC
:10F2F0008091D60F9091D70FA091D80FB091D90FD0
:10F300008C159D05AE05BF05D1F00E943D9C811175
:10F3100002C080E018C026ED3DE0B701A601809153
:10F32000DF0F9091E00F0E94BF9C882391F3C09261
:10F33000D60FD092D70FE092D80FF092D90F81E07C
:10F34000C1118093DE0FCF91FF90EF90DF90CF90AF
:10F3500008954F925F926F927F928F929F92AF9299
:10F36000BF92CF92DF92EF92FF920F931F93CF93B2
:10F37000DF93EC01423051056105710510F480E026
:10F3800069C089859A85AB85BC850196A11DB11D93
:10F3900084179507A607B70790F38F89803149F442
:10F3A000852E962EA72EBB248B899C89AD89BE897C
:10F3B0000FC0803221F78B889C88AD88BE88DB0126
:10F3C000CA01E7E0B695A79597958795EA95D1F795
:10F3D000880E991EAA1EBB1E280139016A017B01F5
:10F3E00041E0C501B4010E947079882341F29F89F0
:10F3F000903161F4DD24EE24FF249601220F331FA7
:10F40000F901EA52F24F5182408211C0E894C7F8E4
:10F41000DD24EE24FF249601220F331F220F331F19
:10F42000F901EA52F24F40825182628273829A89D4
:10F43000923080F04D815E816F817885840E951EBB
:10F44000A61EB71E8092DA0F9092DB0FA092DC0FFF
:10F45000B092DD0FDF91CF911F910F91FF90EF9050
:10F46000DF90CF90BF90AF909F908F907F906F90E4
:10F470005F904F900895CF92DF92EF92FF920F939B
:10F480001F93CF93DF93FC0181859285A385B4857B
:10F490000196A11DB11D84179507A607B70710F4A3
:10F4A00080E061C08789803149F4BB27A72F962F60
:10F4B000852FC388D488E588F6880FC0803281F70D
:10F4C00083899489A589B6896A017B01C7E0F6948E
:10F4D000E794D794C794CA95D1F78C0D9D1DAE1DA6
:10F4E000BF1DE9016A017B018F014091D60F509148
:10F4F000D70F6091D80F7091D90F84179507A60781
:10F50000B70739F040E0BC01CD010E947079882333
:10F5100039F2F8018789803179F4B701A6015527BE
:10F5200066277727440F551FFA01EA52F24F808170
:10F530009181A0E0B0E012C0B701A6014F77552736
:10F5400066277727440F551F440F551FFA01EA52CB
:10F55000F24F80819181A281B381BF7088839983AA
:10F56000AA83BB8381E0DF91CF911F910F91FF9020
:10F57000EF90DF90CF9008954F925F926F927F92BD
:10F58000AF92BF92CF92DF92EF92FF920F931F93B1
:10F59000CF93DF9300D01F92CDB7DEB78C014983A4
:10F5A0005A836B837C835901C12CD12C7601412C69
:10F5B00082E0582E612C712C49815A816B817C81AB
:10F5C0009E012F5F3F4FC8010E943B7A882341F183
:10F5D000D301C201F801058404C0880F991FAA1F36
:10F5E000BB1F0A94D2F7C80ED91EEA1EFB1E498122
:10F5F0005A816B817C818789803139F481E0483F71
:10F600005F4F6105710538F4D7CF81E0483F5F4F08
:10F610006F4F7F4088F2F501C082D182E282F3828F
:10F620000F900F900F900F90DF91CF911F910F913E
:10F63000FF90EF90DF90CF90BF90AF907F906F9052
:10F640005F904F9008952F923F924F925F926F92EA
:10F650007F928F929F92AF92BF92CF92DF92EF9262
:10F66000FF921F93CF93DF9300D01F92CDB7DEB7E9
:10F670004A011901FC014080518062807380FB01C6
:10F68000C080D180E280F3802091B90D3091BA0D15
:10F690004091BB0D5091BC0DC301B2010F941830C5
:10F6A00081110EC011E0A70196016091BD0D70910E
:10F6B000BE0D8091BF0D9091C00D0F941830811137
:10F6C00010E080E1E9EBFDE0A5E8BDE001900D92DE
:10F6D0008A95E1F7F40180809180A280B380209127
:10F6E0004402309145024091460250914702C501C3
:10F6F000B4010F941830882379F180928D0D909287
:10F700008E0DA0928F0DB092900D80924402909237
:10F710004502A0924602B092470220E030E040E06D
:10F720005FE360917F0B7091800B8091810B9091D2
:10F73000820B0F947E3069837A838B839C83CE0106
:10F7400001960E94B9C780E1E9EBFDE0A5E8BDE0C4
:10F7500001900D928A95E1F74092850D5092860DA9
:10F760006092870D7092880DC092890DD0928A0D9B
:10F77000E0928B0DF0928C0DF1012081318142815C
:10F7800053816091910D7091920D8091930D9091A4
:10F79000940D0F940E376093910D7093920D80939A
:10F7A000930D9093940D112379F02AEF3EE74AE2EE
:10F7B0005FE36091830B7091840B8091850B909136
:10F7C000860B0F947E3004C060E070E080EA91E424
:10F7D00069837A838B839C83CE0101960E94B9C78B
:10F7E00080E1E9EBFDE0A5E8BDE001900D928A958E
:10F7F000E1F70F900F900F900F90DF91CF911F9135
:10F80000FF90EF90DF90CF90BF90AF909F908F9040
:10F810007F906F905F904F903F902F9008950F933F
:10F820001F93CF93DF93CDB7DEB728970FB6F89429
:10F83000DEBF0FBECDBF8C010E945AE11D821E8229
:10F840001F82188620E030E040E05FE36091C10D48
:10F850007091C20D8091C30D9091C40D0F940E371D
:10F8600069837A838B839C839E012B5F3F4FAE011C
:10F870004F5F5F4F6DEB7DE089EB9DE00E94237B46
:10F880001D821E821F82188620E030E040E05FE388
:10F89000F80160857185828593850F940E376983A1
:10F8A0007A838B839C83B8016C5F7F4F9E012B5FB3
:10F8B0003F4FAE014F5F5F4FC8010E94237B2896E8
:10F8C0000FB6F894DEBF0FBECDBFDF91CF911F9171
:10F8D0000F9108952F923F924F925F926F927F9275
:10F8E0008F929F92AF92BF92CF92DF92EF92FF9250
:10F8F0000F931F93CF93DF93CDB7DEB7A0970FB6CB
:10F90000F894DEBF0FBECDBF8C011B014090B90D36
:10F910005090BA0D6090BB0D7090BC0D8090BD0DE5
:10F920009090BE0DA090BF0DB090C00DDC018D91E8
:10F930009D910D90BC91A02D8D879E87AF87B88B30
:10F940009C01AD01C301B2010F940D376B017C0125
:10F95000D80114968D919D910D90BC91A02D898B0D
:10F960009A8BAB8BBC8B9C01AD01C501B4010F948C
:10F970000D376D8B7E8B8F8B988FD1018D919D91E3
:10F980000D90BC91A02D8D839E83AF83B8879C0181
:10F99000AD01C301B2010F940D37698F7A8F8B8F40
:10F9A0009C8FD10114968D919D910D90BC91A02DAD
:10F9B00089879A87AB87BC879C01AD01C501B401DB
:10F9C0000F940D376D8F7E8F8F8F98A3A7019601AF
:10F9D000C701B6010F947E306B017C012D893E89F1
:10F9E0004F89588DCA01B9010F947E309B01AC013B
:10F9F000C701B6010F940E374B015C012D853E8582
:10FA00004F8558896D817E818F8198850F940D3740
:10FA10002B013C0129893A894B895C8969857A8562
:10FA20008B859C850F940D376B017C01A30192019E
:10FA3000C301B2010F947E302B013C01A701960156
:10FA4000C701B6010F947E309B01AC01C301B20126
:10FA50000F940E370F94BC396B017C01298D3A8DC0
:10FA60004B8D5C8DCA01B9010F947E302B013C0196
:10FA70002D8D3E8D4F8D58A1CA01B9010F947E3056
:10FA80009B01AC01C301B2010F940E379B01AC0185
:10FA9000C501B4010F946E391816E4F420E030E08B
:10FAA000A901C701B6010F946E3987FF04C0C701D1
:10FAB000B601905802C0C701B60120E030E040EA2C
:10FAC00050E40F946E3918162CF4B801C1010E944D
:10FAD0006A7C46C020E030E040E050E4C501B4015B
:10FAE0000F946E3918161CF4C8010E940F7C1982FD
:10FAF0001A821B821C82A801485F5F4FB8016C5FAD
:10FB00007F4F9E012F5F3F4FC8010E94237B2DEC4A
:10FB10003CEC4CEC5CE3C701B6010F947E309B01DA
:10FB2000AC016091600C7091610C8091620C9091BD
:10FB3000630C0F947E3069837A838B839C838091DE
:10FB4000950D81110E9486E1A101485F5F4FB101CF
:10FB50006C5F7F4F9E012F5F3F4FC1010E94237B4F
:10FB6000A0960FB6F894DEBF0FBECDBFDF91CF9148
:10FB70001F910F91FF90EF90DF90CF90BF90AF90CB
:10FB80009F908F907F906F905F904F903F902F90BD
:10FB900008958C3891051CF02CE880E002C0282FD5
:10FBA000892F20937E0980937F090C94C9718091DD
:10FBB000451890914618892B39F00E94EDCB91E0C1
:10FBC000811103C090E001C091E0892F0895CF9387
:10FBD000DF93C82FD62F0E9485CC882321F0DF9198
:10FBE000CF910C94D77D8C2F0E943CCC811101C009
:10FBF0008D2FDF91CF9108952F923F924F925F9278
:10FC00006F927F928F929F92AF92BF92CF92DF922C
:10FC1000EF92FF920F931F93CF93DF93CDB7DEB791
:10FC2000CB56D1090FB6F894DEBF0FBECDBF84EF1F
:10FC30009DE10F9467160E94C8DE81110C947688AE
:10FC400084E50E9485CC882329F00E9401CC60E0E5
:10FC50000E94956B80E090E0A0E8BFE38093600C89
:10FC60009093610CA093620CB093630C8093810D10
:10FC70009093820DA093830DB093840D8DEC9CEC3A
:10FC8000ACE4BEE380935C0C90935D0CA0935E0C9F
:10FC9000B0935F0C80E090E0A0E2B1E48093580C58
:10FCA0009093590CA0935A0CB0935B0C8CE390E0AA
:10FCB0009093570C8093560C8DEC90E09093550CDC
:10FCC0008093540C1092530C4AE959E969E97EE398
:10FCD0008FE40E94ECA329966CAF7DAF8EAF9FAFEF
:10FCE000299760E083E40E94E77DA5968FAFA597F2
:10FCF00060E08BE40E94E77DA6968FAFA69782E432
:10FD00000E9485CC8823C9F00E9405CC0F947A38D4
:10FD10007093570C6093560C6115710571F0685221
:10FD200071096536710548F06CE870E086EC9DE17C
:10FD30000F942C1781EC9DE1B0C18CE40E9485CC1E
:10FD4000882301F10E9405CC6B017C0160935C0C5F
:10FD500070935D0C80935E0C90935F0C20E030E01C
:10FD6000A9010F946E3987FD0AC020E030E040E021
:10FD700050E4C701B6010F94183018161CF489E935
:10FD80009DE18BC181E50E943CCC882351F180919B
:10FD9000451890914618892B09F10E9405CC6B01FA
:10FDA0007C016093810D7093820D8093830D9093FD
:10FDB000840D2DEC3CEC4CE45DE30F946E3987FD33
:10FDC0000AC020E030E040E751E4C701B6010F94DB
:10FDD0001830181634F488E69DE15FC18DE39DE18B
:10FDE0005CC183E50E9485CC8823C9F00E9405CCC4
:10FDF0004B015C012DEC3CEC4CEC5DE30F946E3957
:10FE000087FD0AC020E030E040E050E4C501B401C5
:10FE10000F941830181654F486E19DE13EC1ADEC04
:10FE20008A2EACEC9A2EA92CAEE3BA2E80E50E9465
:10FE30003CCC882371F18091451890914618892B0C
:10FE400019F48EED9CE129C18091530C8F5F809352
:10FE5000530C0E9405CC6B017C016093580C70938D
:10FE6000590C80935A0C90935B0C20E030E0A90170
:10FE70000F946E3987FD0AC020E030E048EC51E471
:10FE8000C701B6010F94183018161CF486EB9CE1DC
:10FE900004C186E40E9485CC8823C9F00E9405CC69
:10FEA0006B017C0120E030E040E85FE30F946E39A5
:10FEB00087FD0AC020E030E040E850E4C701B60109
:10FEC0000F94183018164CF48DE89CE1E6C0C12C54
:10FED000D12CF0EEEF2EFFE3FF2EA7019601C70114
:10FEE000B6010F947E309B01AC0160E070E084E4C9
:10FEF00090E40F9408382091600C3091610C40918F
:10FF0000620C5091630C0F947E302B013C01A501D3
:10FF10009401C501B4010F947E30A70196010F949E
:10FF20007E302CEE31E548EB5DE30F9408389B0101
:10FF3000AC01C301B2010F947E306093600C7093EA
:10FF4000610C8093620C9093630C88E40E9485CCD2
:10FF5000882381F00E9405CC0F947A387093550C59
:10FF60006093540C655A71096838710518F08FE573
:10FF70009CE193C085E50E943CCC8823F1F00F946E
:10FF8000E21F611571058105910511F00F94A92BF0
:10FF90008091451890914618892B19F00E9405CC44
:10FFA00004C060E070E088E492E460934F0C7093CA
:10FFB000500C8093510C9093520C82E50E943CCCE3
:10FFC000811103C08BE29CE168C08091451890913B
:10FFD0004618892B61F00E9401CC6B969FAF8EAFC3
:10FFE0006B97181619064CF087EF9BE156C02AE173
:10FFF00030E06B963FAF2EAF6B9789E50E9485CCC2
:020000021000EC
:10000000882379F00E9405CC20919A0D30919B0DA8
:1000100040919C0D50919D0D0F940D376B017C010B
:1000200008C0C090BD0DD090BE0DE090BF0DF09007
:10003000C00D88E50E9485CC882369F00E9405CC1C
:100040002091960D3091970D4091980D5091990DFA
:100050000F940D3708C06091B90D7091BA0D809161
:10006000BB0D9091BC0D6093470C7093480C80932E
:10007000490C90934A0CC0924B0CD0924C0CE092DD
:100080004D0CF0924E0CB701A60187E49CE00F9452
:100090005C1E811106C08DEC9BE10F9467160C94D9
:1000A000768884E40E943CCC91E089270E9447D264
:1000B00020E030E040EA50E46091C10D7091C20D43
:1000C0008091C30D9091C40D0F94183087FF1CC010
:1000D000198A1A8A1B8A1C8A80E090E0A0EAB0E4A0
:1000E00089839A83AB83BC83BE016F5E7F4FCE0151
:1000F00001960E9426C980E1E5E8FDE0A9EBBDE09C
:1001000001900D928A95E1F730913418A7963FAF90
:10011000A797109234180F948B028CEA9BE10F94EE
:1001200067168091560C9091570C8A31910574F4A2
:100130008091540C9091550C0E94A4A161E0809193
:10014000B80D0E94146A811109C00DC50E94C97DB5
:1001500081E00E9495688111EBCF05C51092C50D15
:100160001092C60D1092C70D1092C80D85EC9DE03F
:100170000E949DFF8091530C882309F455C020E014
:1001800030E040E751E46091830B7091840B8091E3
:10019000850B9091860B0F94083869837A838B8343
:1001A0009C8380E1E9EBFDE0A5E8BDE001900D92C4
:1001B0008A95E1F72091580C3091590C40915A0CD6
:1001C00050915B0C6091910D7091920D8091930D07
:1001D0009091940D0F940E376093910D7093920D42
:1001E0008093930D9093940DCE0101960E94B9C710
:1001F0002091580C3091590C40915A0C50915B0C45
:100200006091910D7091920D8091930D9091940D4C
:100210000F940D376093910D7093920D8093930D11
:100220009093940D0E945AE185E0E2E4FCE0DF0146
:10023000282F1D922A95E9F7EDE3FCE0DF01282F36
:100240001D922A95E9F7E8E3FCE0DF011D928A950B
:10025000E9F780E1E9EBFDE0A5E8BDE001900D9252
:100260008A95E1F780915C0C90915D0CA0915E0CF9
:10027000B0915F0C80938D0D90938E0DA0938F0D98
:10028000B093900D19821A821B821C829E012F5FEF
:100290003F4F4DE85DE069E87DE085E89DE00E9424
:1002A000237B9E012B5B3F4F4DE85DE069E87DE0DD
:1002B00085E89DE00E94237BA596BFADA597BB2353
:1002C000B9F02091B90D3091BA0D4091BB0D50910C
:1002D000BC0D2E962CAF3DAF4EAF5FAF2E978091E9
:1002E000BD0D9091BE0DA091BF0DB091C00D16C077
:1002F0002091470C3091480C4091490C50914A0C88
:100300002E962CAF3DAF4EAF5FAF2E9780914B0C2A
:1003100090914C0CA0914D0CB0914E0C69968CAF05
:100320009DAFAEAFBFAF6997212C312C9FEF2A96BE
:100330009FAF2A97AFEF6596AFAF6597BFEF6C960B
:10034000BFAF6C97EFE4A096EFAFA097F3ECA29647
:10035000FFAFA29727E4A3962FAFA39781E090E089
:10036000A0E0B0E0022C04C0880F991FAA1FBB1F99
:100370000A94D2F7AB968CAF9DAFAEAFBFAFAB9741
:10038000A2E4BCE06496BFAFAEAF649700E010E0BB
:10039000AC962FAEAC976496EEADFFAD64978191AD
:1003A0006496FFAFEEAF649790E0A0E0B0E0AB964C
:1003B0002CAD3DAD4EAD5FADAB9782239323A4230F
:1003C000B523892B8A2B8B2B09F004C180915813FC
:1003D00090915913289EB001299E700D389E700D82
:1003E00011248091350D9091360D680F791F072EDD
:1003F000000C880B990B0F941F3062966CAF7DAF89
:100400008EAF9FAF629780915A1390915B13089FB4
:10041000B001099F700D189F700D11248091370D48
:100420009091380D680F791F072E000C880B990BDF
:100430000F941F306B017C0162962CAD3DAD4EAD2B
:100440005FAD62972E966CAD7DAD8EAD9FAD2E9754
:100450000F940D372B013C01A701960169966CADF5
:100460007DAD8EAD9FAD69970F940D374B015C014B
:10047000A3019201C301B2010F947E302B013C0114
:10048000A5019401C501B4010F947E309B01AC011C
:10049000C301B2010F940E370F94BC394B015C01BC
:1004A00062962CAD3DAD4EAD5FAD62976091470C4D
:1004B0007091480C8091490C90914A0C0F940D3723
:1004C0002B013C01A701960160914B0C70914C0CE3
:1004D00080914D0C90914E0C0F940D376B017C0167
:1004E000A3019201C301B2010F947E302B013C01A4
:1004F000A7019601C701B6010F947E309B01AC01A4
:10050000C301B2010F940E370F94BC3920E030E0E4
:1005100040E751E40F940838A50194010F940E3779
:100520006B017C0180904F0C9090500CA090510C6E
:10053000B090520C20E030E040E85FE3C501B40128
:100540000F946E391816FCF4C501B4010F947A3873
:100550004B015C0116161706180619063CF40F9499
:100560005B2BA50194010F94903603C060E070E00E
:10057000CB010F941F309B01AC01B601C7010F9452
:100580000E376B017C016C962FAD6C97A0963FAD3A
:10059000A097A2964FADA297A3965FADA397B60181
:1005A000C7010F94183087FF15C02A960FAF2A97FE
:1005B000AC963FADAC9765963FAF65976C96CFAE66
:1005C0006C97A096DFAEA097A296EFAEA297A396E7
:1005D000FFAEA3970F5F1F4F0530110509F0DBCE6B
:1005E0004FEF241A340A55E02516310409F0B6CE2F
:1005F00065968FAD6597E82FF0E0EE5BF34F81E0F5
:1006000090E02A960FAC2A9702C0880F991F0A948F
:10061000E2F79081892B808365969FAD65979F3F18
:1006200009F487C22A96AFAD2A97AF3F09F481C279
:10063000209158133091591365964FAD6597420339
:10064000B001439F700D11248091350D9091360DAE
:10065000680F791F072E000C880B990B0F941F3021
:10066000162F072F382E292E862F902FA32DB22D2F
:1006700021968CAF9DAFAEAFBFAF219720915A139B
:1006800030915B132A965FAD2A975203B001539FB6
:10069000700D11248091370D9091380D680F791FDE
:1006A000072E000C880B990B0F941F306B017C01F7
:1006B00025966CAF7DAF8EAF9FAF2597AB01BC0188
:1006C000CE01CD960F945C1E882309F436C220E03B
:1006D00030E040EA50E4612F702F832D922D0F946B
:1006E0000E374B015C01FE01B9968CE0DF011D92D3
:1006F0008A95E9F7C401D50189A79AA7ABA7BCA73A
:10070000CDA6DEA6EFA6F8AA6596BFAD6597B11196
:10071000B2C22A96EFAD2A97E1118EC220E030E0F6
:1007200040EA50E4C701B6010F940E376B017C011B
:100730002A96FFAD2A97FF2309F417C32A963FADE7
:100740002A9734300CF011C3E2ED4E2EE3E55E2E15
:10075000EBE76E2EE1E47E2E89A49AA4ABA4BCA4A0
:100760002DA53EA54FA558A92E962CAF3DAF4EAF57
:100770005FAF2E9725966CAD7DAD8EAD9FAD259765
:100780000F940D3762966CAF7DAF8EAF9FAF6297BF
:10079000A501940121966CAD7DAD8EAD9FAD2197E5
:1007A0000F940D376DAB7EAB8FAB98AF62968CAD6F
:1007B0009DADAEADBFAD629789AF9AAFABAFBCAFE9
:1007C000A50194016091B90D7091BA0D8091BB0D96
:1007D0009091BC0D0F940D374B015C012E962CAD02
:1007E0003DAD4EAD5FAD2E976091BD0D7091BE0DCC
:1007F0008091BF0D9091C00D0F940D372E966CAF68
:100800007DAF8EAF9FAF2E97812F902FA32DB22D4E
:1008100089839A83AB83BC83CD82DE82EF82F886A4
:10082000C0905C0CD0905D0CE0905E0CF0905F0C82
:10083000C986DA86EB86FC862DEC3CEC4CEC5CE35E
:10084000C301B2010F947E302091600C3091610C95
:100850004091620C5091630C0F947E302091C50D35
:100860003091C60D4091C70D5091C80D0F940E37B1
:100870006D877E878F87988BA5019401C501B40190
:100880000F947E304B015C012E962CAD3DAD4EADEC
:100890005FAD2E97CA01B9010F947E309B01AC0168
:1008A000C501B4010F940E3720E030E040E050E481
:1008B0000F946E39181684F420E030E040E05FE3D6
:1008C000C701B6010F940E3769AB7AAB8BAB9CAB0B
:1008D000CE0189960E940F7C80915C0C90915D0CFA
:1008E000A0915E0CB0915F0C89AB9AABABABBCAB8B
:1008F000198A1A8A1B8A1C8A9E012F5E3F4FAE01FD
:100900004F5C5F4FBE01635D7F4FCE0189960E94B1
:10091000237B8091950D81110E9486E140905B02BE
:1009200050905C0260905D0270905E02E0907B0BE4
:10093000F0907C0B00917D0B10917E0BA090770BBB
:10094000B090780BC090790BD0907A0B9501A601EE
:10095000B701C8010F946E39181614F47501860199
:100960002DEC3CEC4CEC5DE3B701C8010F947E30FC
:1009700060935B0270935C0280935D0290935E02D1
:1009800040E0BE016B5C7F4FCE0101960E942DF4CA
:1009900040925B0250925C0260925D0270925E0235
:1009A00080E1E9EBFDE0A5E8BDE001900D928A95BC
:1009B000E1F780915C0C90915D0CA0915E0CB09180
:1009C0005F0C898F9A8FAB8FBC8F8DA39EA3AFA333
:1009D000B8A7CC24C394D12CD60111976796BFAF8A
:1009E000AEAF6797812C912C5401839466960FAC1F
:1009F000669704C0880C991CAA1CBB1C0A94D2F7E9
:100A000081E090E0A0E0B0E00C2C04C0880F991FBA
:100A1000AA1FBB1F0A94D2F79C01AD0128293929CE
:100A20004A295B296F962CAF3DAF4EAF5FAF6F97F2
:100A300081E066960FAC669701C0880F0A94EAF7CA
:100A4000A2968FAFA29748E35CE064965FAF4EAF8B
:100A500064978DE39CE02C969FAF8EAF2C97A2E419
:100A6000BCE06096BFAFAEAF6097212C312CA19651
:100A70003FAE2EAEA1976096EEADFFAD6097A49607
:100A8000FFAFEEAFA497FFEF2F1A3F0A6096AEAD0F
:100A9000BFAD60978C9190E0A0E0B0E06F962CAD78
:100AA0003DAD4EAD5FAD6F9782239323A423B52355
:100AB00082179307A407B50709F47BC16096EEADD2
:100AC000FFAD609731966096FFAFEEAF6097A4964A
:100AD000AEADBFADA4978C9190E0A0E0B0E08821CE
:100AE0009921AA21BB21892B8A2B8B2B09F053C179
:100AF00064962EAD3FAD64972F5F3F4F64963FAF36
:100B00002EAF64972C964EAD5FAD2C974F5F5F4F25
:100B10002C965FAF4EAF2C9755E02516310409F0A7
:100B2000A6CF8FEFC81AD80A96E0C916D10409F0EB
:100B300053CF8091AA0C8093AB0C6B96AEADBFAD3A
:100B40006B9711976B96BFAFAEAF6B97AB2B59F00E
:100B50006596BFAD6597BF3F31F02A96EFAD2A97F6
:100B6000EF3F09F0A9CB6FEF81EC9BE10F944E1A98
:100B70000E945AE180E090E0A0EAB0E480938D0DFD
:100B800090938E0DA0938F0DB093900D19821A82C1
:100B90001B821C829E012F5F3F4F4DE85DE069E89C
:100BA0007DE085E89DE00E94237B80914B0C909135
:100BB0004C0CA0914D0CB0914E0C4091470C5091B3
:100BC000480C6091490C70914A0C4093850D5093EC
:100BD000860D6093870D7093880D8093890D909397
:100BE0008A0DA0938B0DB0938C0D19821A821B82F3
:100BF0001C829E012F5F3F4F4DE85DE069E87DE07C
:100C000085E89DE00E94237BA796FFADA797F09310
:100C100034180F948B02A6962FADA697211166C2A9
:100C200010927F0910927E090E94C9718091B80DBF
:100C300090E00E94A4A15AC2812F902FA32DB22D23
:100C400089A79AA7ABA7BCA720E030E040EA50E410
:100C5000C701B6010F940D376DA77EA78FA798AB7C
:100C60002A962FAD2A9724300CF458CD182D092D33
:100C70003A2C2B2C7AC065964FAD659744300CF416
:100C80004CC02A965FAD2A9754307CF020E030E0CB
:100C900040EA50E4612F702F832D922D0F940D3771
:100CA00069A77AA78BA79CA728C0812F902FA32D77
:100CB000B22D89A79AA7ABA7BCA720E030E040EAF5
:100CC00050E4C701B6010F940E376DA77EA78FA71A
:100CD00098AB2A968FAD2A9781110FC020E030E0A3
:100CE00040EA50E4612F702F832D922D0F940D3721
:100CF000162F072F382E292E38C020E030E040EA8A
:100D000050E4C701B6010F940D376B017C012A96A0
:100D10009FAD2A9794304CF517CD2A96AFAD2A9700
:100D2000A1110DC020E030E040E251E4B401C50162
:100D30000F940D37162F072F382E292E05CD2A9602
:100D4000BFAD2A97B430D4F020E030E040E251E467
:100D5000B401C5010F940D3769A77AA78BA79CA78B
:100D6000182D092D3A2C2B2CEFCC72ED472E73E564
:100D7000572E7BEF672E70E4772EEECC182D092DC1
:100D80003A2C2B2C62ED462E63E5562E6BEF662E29
:100D900061E4762EE1CC808190E0A0E0B0E0882193
:100DA0009921AA21BB21892B8A2B8B2B09F0D0C03A
:100DB0009FCE2C96AEADBFAD2C978C9190E0A0E06D
:100DC000B0E088219921AA21BB21892B8A2B8B2B6A
:100DD00009F074CE0091350D1091360DE090581346
:100DE000F090591367964EAD5FAD6797E49EB001E2
:100DF000E59E700DF49E700D1124600F711F072E7B
:100E0000000C880B990B0F941F3020E030E040E07D
:100E100050E40F940E376D8F7E8F8F8F98A3CE9CEA
:100E2000B001CF9C700DDE9C700D1124600F711FFE
:100E3000072E000C880B990B0F941F3020E030E038
:100E400040E050E40F940D37698B7A8B8B8B9C8B31
:100E50004AE351E061E070E0CE014D960F94430902
:100E600080915A1390915B13A196AEADBFADA1973F
:100E7000A89FB001A99F700DB89F700D112480919B
:100E8000370D9091380D680F791F072E000C880BD5
:100E9000990B0F941F302B013C0120E030E040E81B
:100EA0005FE30F94183087FD12C020E030E849E975
:100EB00053E4C301B2010F946E39181674F4412C37
:100EC00030E8532E39E9632E33E4732E06C0412CEB
:100ED000512C20E8622E2FE3722E4D8A5E8A6F8A93
:100EE000788E49A25AA26BA27CA24AE351E061E04B
:100EF00070E0CE0141960F94430949A15AA16BA11C
:100F00007CA1CE014D960F945C1E882351F04D8933
:100F10005E896F89788DCE0141960F945C1E811198
:100F20000FC02C96EEADFFAD2C978081A296FFAD41
:100F3000A2978F2B2C96AEADBFAD2C978C93BECDC8
:100F4000BE016F5E7F4FCE014D960E946A7CE9CF55
:100F50006496EEADFFAD6497808190E0A0E0B0E0D4
:100F600088219921AA21BB21892B8A2B8B2B09F05F
:100F7000BFCD0091370D1091380DE0905A13F090CD
:100F80005B13A196EEADFFADA197EE9DB001EF9D75
:100F9000700DFE9D700D1124600F711F072E000C47
:100FA000880B990B0F941F3020E030E040E050E4B4
:100FB0000F940E3769A37AA38BA39CA32E9CB00138
:100FC0002F9C700D3E9C700D1124600F711F072E19
:100FD000000C880B990B0F941F3020E030E040E0AC
:100FE00050E40F940D376D8B7E8B8F8B988F809193
:100FF00058139091591367962EAD3FAD6797289F70
:10100000B001299F700D389F700D11248091350D0E
:101010009091360D680F791F072E000C880B990BE5
:101020000F941F302B013C0120E030E040E85FE3EB
:101030000F94183087FD11C020E030E04DE953E4F3
:10104000C301B2010F946E3918166CF4412C512C67
:101050009DE9692E93E4792E06C0412C512C80E83D
:10106000682E8FE3782E498A5A8A6B8A7C8A4D8E45
:101070005E8E6F8E78A243E351E061E070E0CE01B6
:1010800081960F94430943E351E061E070E0CE01A3
:1010900045960F94430949A15AA16BA17CA1CE01A9
:1010A0004D960F945C1E882351F04D895E896F899F
:1010B000788DCE0141960F945C1E81110FC064960D
:1010C000AEADBFAD64978C91A296BFADA2978B2BAE
:1010D0006496EEADFFAD649780830ACDBE016F5E6E
:1010E0007F4FCE014D960E946A7CE9CFC559DF4FF4
:1010F0000FB6F894DEBF0FBECDBFDF91CF911F9129
:101100000F91FF90EF90DF90CF90BF90AF909F90A6
:101110008F907F906F905F904F903F902F900895A9
:101120002F923F924F925F926F927F928F929F92F7
:10113000AF92BF92CF92DF92EF92FF920F931F93E5
:10114000CF93DF93CDB7DEB7CD57D1090FB6F89463
:10115000DEBF0FBECDBF3B014A015901EBA66F9622
:10116000DFAECEAE6F97DC012D913D914D915C913C
:10117000A5962CAF3DAF4EAF5FAFA5972091670B03
:101180003091680B4091690B50916A0BA5966CAD3C
:101190007DAD8EAD9FADA5970F947E300F947B39BA
:1011A000E5966CAF7DAF8EAF9FAFE597D3012D91E4
:1011B0003D914D915C91A9962CAF3DAF4EAF5FAF85
:1011C000A99720916B0B30916C0B40916D0B509156
:1011D0006E0BA9966CAD7DAD8EAD9FADA9970F94AA
:1011E0007E300F947B39E9966CAF7DAF8EAF9FAFA9
:1011F000E997D4012D913D914D915C91AD962CAF25
:101200003DAF4EAF5FAFAD9720916F0B3091700B3C
:101210004091710B5091720BAD966CAD7DAD8EAD62
:101220009FADAD970F947E300F947B39ED966CAFE8
:101230007DAF8EAF9FAFED97D5012D913D914D9133
:101240005C9169962CAF3DAF4EAF5FAF699720912F
:10125000730B3091740B4091750B5091760B69961E
:101260006CAD7DAD8EAD9FAD69970F947E300F94C0
:101270007B396D966CAF7DAF8EAF9FAF6D978091D0
:10128000A20B83FF1CC06D962CAD3DAD4EAD5FAD86
:101290006D972093F3153093F4154093F515509303
:1012A000F61569968CAD9DADAEADBFAD69978093D7
:1012B000E3159093E415A093E515B093E61580919E
:1012C000510B9091520B892B09F079C3D801BC9135
:1012D000BBABF801F181FFAFD8011296BC91249607
:1012E000BFAF2497F801F3812A96FFAF2A97809128
:1012F000C1159091C215891B8F708F3021F480E049
:101300000E945655F4CF2091C115EE962FAFEE975F
:101310008091C115282E312C34E6839FC001112401
:10132000AC014E54574E29965FAF4EAF299780912E
:10133000E7159091E815A091E915B091EA15E596A9
:101340008CAC9DACAEACBFACE597881A990AAA0AE2
:10135000BB0A8091EB159091EC15A091ED15B09121
:10136000EE15E9964CAC5DAC6EAC7FACE997481AD3
:10137000590A6A0A7B0A8091EF159091F015A091A5
:10138000F115B091F215ED962CAD3DAD4EAD5FADC2
:10139000ED97281B390B4A0B5B0B2FAB38AF49AFCE
:1013A0005AAF8091F3159091F415A091F515B09175
:1013B000F6156D962CAD3DAD4EAD5FAD6D97281B0E
:1013C000390B4A0B5B0B2BA33CA34DA35EA3232B32
:1013D000242B252B09F49BC08091A10B81113CC0CB
:1013E00020E030E0A9016091630970916409809167
:1013F0006509909166090F940E370F947A38209101
:101400004202309143026217730734F56D968CAD3A
:101410009DADAEADBFAD6D978093F3159093F41570
:10142000A093F515B093F61569962CAD3DAD4EAD74
:101430005FAD69972093E3153093E4154093E5156C
:101440005093E6150F94501784E29EE10F946716AF
:101450001BA21CA21DA21EA24BA534E0439F80012B
:101460001124085B1D4F6BA17CA18DA19EA10F943F
:101470001F30D8012D913D914D915C910F947E309C
:101480006B017C0120E030E0A9010F946E3987FFE9
:1014900004C0F7FAF094F7F8F09420E030E04AEF57
:1014A00053E46091730B7091740B8091750B909164
:1014B000760B0F947E30A70196010F94183087FFAA
:1014C00026C06D962CAD3DAD4EAD5FAD6D972093B2
:1014D000F3153093F4154093F5155093F61569966E
:1014E0008CAD9DADAEADBFAD69978093E315909384
:1014F000E415A093E515B093E6150F94501785E019
:101500009EE10F9467161BA21CA21DA21EA2D5016C
:10151000C4018827B7FD83959927AA27BB278FA3E6
:1015200077FE03C0E82FE260EFA32FA938AD49ADE5
:101530005AAD57FF03C03FA134603FA38BA19CA1CC
:10154000ADA1BEA1B7FF03C09FA198609FA3BBA59B
:10155000A4E0BA9F80011124085B1D4F6BA17CA100
:101560008DA19EA10F941F30F8012081318142810D
:1015700053810F947E306B017C0120E030E0A901A3
:101580000F946E3987FF04C0C701B601905802C09E
:10159000C701B60120E030E040E05FE30F940E3772
:1015A0000F9481386FA778AB89AB9AAB84E6829DA4
:1015B000F001839DF00D1124EE54F74E1082EA5B8A
:1015C000FF4F2FA120838FA998ADA9ADBAAD619629
:1015D0008CAF9DAFAEAFBFAF6197B7FF0DC0B095F9
:1015E000A095909581959F4FAF4FBF4F61968CAF5F
:1015F0009DAFAEAFBFAF61974BAE5CAE6DAE7EAE92
:1016000077FE0BC022273327A90124193509460983
:1016100057092BAF3CAF4DAF5EAF8FA298A6A9A6DE
:10162000BAA6B7FE0BC088279927DC01881999094B
:10163000AA09BB098FA398A7A9A7BAA72FA138A564
:1016400049A55AA52996AEADBFAD299755962D93BC
:101650003D934D935C9358972BAD3CAD4DAD5EAD36
:1016600059962D933D934D935C935C9761962CAD69
:101670003DAD4EAD5FAD61975D962D933D934D931E
:101680005C939097C501B4010F941F302091880C92
:101690003091890C40918A0C50918B0C0F947E30C4
:1016A00065966CAF7DAF8EAF9FAF6597698B7A8B78
:1016B0008B8B9C8BC301B2010F941F3020918C0C3B
:1016C00030918D0C40918E0C50918F0C0F947E3088
:1016D0002B013C016D8B7E8B8F8B988F6FA978AD22
:1016E00089AD9AAD0F941F302091900C3091910CE0
:1016F0004091920C5091930C0F947E304B015C0101
:10170000698F7A8F8B8F9C8F2091940C3091950CE0
:101710004091960C5091970CC701B6010F947E3002
:101720006B017C016D8F7E8F8F8F98A32FA138A5C1
:1017300049A55AA52630310541055105BCF58BADAB
:101740009CADADADBEAD0697A105B1057CF561962A
:101750002CAD3DAD4EAD5FAD6197263031054105F5
:10176000510524F520E030E0A901C701B6010F942E
:101770006E3987FF04C0F7FAF094F7F8F09484E626
:10178000829D8001839D100D11240E54174E20E080
:1017900030E0A901C701B6010F940E37D8011D969C
:1017A0006D937D938D939C93509752C06F96EEAD41
:1017B000FFAD6F97C080D180E280F38020E030E001
:1017C000A901C701B6010F941830882369F084E697
:1017D000829DF001839DF00D1124EE54F74EC586D5
:1017E000D686E786F08A34C065962CAD3DAD4EAD09
:1017F0005FAD6597CA01B9010F947E306B017C0122
:10180000A3019201C301B2010F947E309B01AC0190
:10181000C701B6010F940E376B017C01A50194013D
:10182000C501B4010F947E309B01AC01C701B60124
:101830000F940E370F94BC3924E6229DF001239DAE
:10184000F00D1124EE54F74E658776878787908BCD
:1018500084E6829DF001839DF00D1124EE54F74E35
:101860002FA538A949A95AA921A332A343A354A358
:1018700061968CAD9DADAEADBFAD61972BAD3CAD6E
:101880004DAD5EAD82179307A407B50710F4DA01DA
:10189000C9012FA138A549A55AA582179307A40706
:1018A000B50710F4DA01C9012FA538A949A95AA929
:1018B00082179307A407B50710F4DA01C90124E6DB
:1018C000229DF001239DF00D1124EE54F74E85A3C7
:1018D00096A3A7A3B0A70697A105B10510F40C9491
:1018E000AB98DF01AE59BF4F8091B00D8C9311962C
:1018F0008091B10D8C933BA531A78FA198A5A9A587
:10190000BAA5892B8A2B8B2B09F05F9884E6829DE0
:10191000F001839DF00D1124EE54F74E818D928DD0
:10192000A38DB48D892B8A2B8B2B09F08A9884E6A2
:10193000829DF001839DF00D1124EE54F74E858DAC
:10194000968DA78DB0A1892B8A2B8B2B29F08091A6
:1019500008018170809306012FA538A949A95AA9C9
:10196000232B242B252B71F18091A80C882319F0AF
:1019700081508093A80C8091A90C882389F0815014
:101980008093A90C3BA5332319F0313071F023C0AB
:10199000811101C0479A129880E28093A80C1BC065
:1019A000FBA5FF23B9F3F130B1F48091A80C8111AC
:1019B00001C0129A479880E28093A90C0CC080E085
:1019C0000C942A99E090970BF090980B0091990B4A
:1019D00010919A0B08C0E090930BF090940B00913B
:1019E000950B1091960B9701A8016BA97FAD2496DA
:1019F0008FAD24972A969FAD2A970F94183087FFB2
:101A000008C0EBAAFFAE24960FAF24972A961FAF0B
:101A10002A9784E6829DF001839DF00D1124EE54F7
:101A2000F74E4584568467847088A301920160E074
:101A300070E080E89FE30F9408386BA77CA78DA720
:101A40009EA72BA93FAD24964FAD24972A965FAD54
:101A50002A970F947E306B017C018091C115909183
:101A6000BF15891B8F708FAFA701960160E074E2EC
:101A700084E799E40F9408380F947B394B015C019B
:101A80008FAD82508630B0F58091630B9091640BDE
:101A9000A091650BB091660B88169906AA06BB0645
:101AA00048F588199909AA09BB09BC01CD01660F3F
:101AB000771F881F991F4FAD042F10E020E030E002
:101AC000A90198010F946E36CA01B9010F941D3017
:101AD0000F947B39680D791D8A1D9B1D0F941D3055
:101AE0009B01AC0160E074E284E799E40F9408384C
:101AF0006B017C01A7019601C301B2010F947E30F6
:101B00009B01AC010F947E302D966CAF7DAF8EAFF4
:101B10009FAF2D9784E6829D8001839D100D112437
:101B20000E54174E2D968CAD9DADAEADBFAD2D971D
:101B3000F80181839283A383B48325A136A147A1B1
:101B400050A52FA338A749A75AA7CA01B9010F94D6
:101B50001D306FAB78AF89AF9AAF9B01AC01C70165
:101B6000B6010F947E300F94EC370F948138619654
:101B70006CAF7DAF8EAF9FAF6197F801EE5AFF4F0C
:101B80006083718382839383FE0171962596FFAFF4
:101B9000EEAF259727E73BE063963FAF2EAF639705
:101BA000AE014F5D5F4F5AA349A31BAE1BAA00E8CD
:101BB0001FE32596AEADBFAD25972D913D914D917B
:101BC0005D912596BFAFAEAF2597C701B6010F94C3
:101BD0007E304B015C0120E030E0A9010F946E39AA
:101BE00087FF04C0B7FAB094B7F8B0946396EEAD2F
:101BF000FFAD639741905190619071906396FFAFF4
:101C0000EEAF6397A5019401C301B2010F941830A0
